:020000040000FA
:061000008FEF74F01200F6
:021006001200D6
:061008001CEF08F01200CD
:0610180055EF09F0120083
:02101E000200CE
:101020002EEA0000600000008100000050E900008E
:0810300000010000DE000000D9
:08103800DACFE4FFE2CFDAFF9A
:10104000E9CFE4FFEACFE4FFF6CFE4FFF7CFE4FF18
:10105000F5CFE4FFF3CFE4FFF4CFE4FFFACFE4FFF2
:1010600000EE48F0140EE80403E3EECFE4FFFBD7F4
:1010700000EE00F0480EE80403E3EECFE4FFFBD7F8
:10108000E6529EAA96D09E9AAFCF80FA0A01A9BBDB
:101090005CD0240E0A01805D0EE10101A66B010106
:1010A000A651EA6A000FE96E0A0EEA2280CAEFFF33
:1010B0000101A62BD6D00101A651EA6A000FE96E04
:1010C0000A0EEA2280CAEFFF0101A62B2A0E0A01AE
:1010D000805D18E1520E0A01035D14E14D0E0A0114
:1010E000045D10E1430E0A01055D0CE10101A66BF0
:1010F0000A01A3810101A72B0101BF2B000EC02310
:10110000C123C223540E0A01035D10E1580E0A01E7
:10111000045D0CE1540E0A01055D08E10101A66BB6
:101120000A01036B0A01046B0A01056B0101A65158
:101130005C6E5D6A5D3404E25C507F08000E5D54B5
:1011400002E20101A66B8DD034D0240E0A01805D2D
:101150000EE10101A66B0101A651EA6A000FE96EDA
:101160000A0EEA2280CAEFFF0101A62B7AD0010104
:10117000A6515C6E5D6A5D3404E25C507F08000E2F
:101180005D5402E20101A66B0101A651EA6A000F5B
:10119000E96E0A0EEA2280CAEFFF0101A62B240E97
:1011A0000A01005D06E10A0E0A01805D02E10A0102
:1011B000A9879EA41ED09E940A01AAB71AD00A013C
:1011C000AA870A01AA83BBCFA0F1BCCFA1F101017C
:1011D000A26BA36BCF6ACE6A0A01AA910A01AA93F5
:1011E0000A01AA8BA396A496010E786E5D0E776E07
:1011F000A3869EA00DD09E90CF6ACE6A0101A42B3B
:10120000100E0101A45D04E10A01AA810101A46B91
:10121000A1A215D0A1920101D22B0101D32B0A0169
:10122000DD810101D42B000ED5230101092B000E15
:101230000A230101052B000E062307230823A4A679
:1012400008D0A496010E786E5D0E776E9E940A010A
:10125000AA97A4BAA49A020E0201585D02E122ECF8
:101260004CF0E55200EE47F0480EE80403E3E5CF0A
:10127000EDFFFBD700EE5BF0140EE80403E3E5CFCF
:10128000EDFFFBD7E5CFFAFFE5CFF4FFE5CFF3FFA6
:10129000E5CFF5FFE5CFF7FFE5CFF6FFE5CFEAFFB6
:1012A000E5CFE9FFE5CFDAFF1100D8CFE4FFE0CFCB
:1012B000E4FFE46EDACFE4FFE2CFDAFFE652E55274
:1012C000E5CFDAFFE550E5CFE0FFE5CFD8FF10002E
:1012D000BDCB4EF0BECB4FF0BFCB50F0C0CB51F0EA
:1012E000EDEC63F04FC004F050C005F051C006F0C3
:1012F00052C007F004C0E6FF05C0E6FF06C0E6FFE7
:1013000007C0E6FF6FEC73F0E552E552E552E55297
:101310004EC000F04FC001F050C002F051C003F0C9
:10132000546A556A7A0E566E440E576E00C04FF0DE
:1013300001C050F002C051F003C052F09DEC64F0C7
:10134000B8EC65F050C0BAFB51C0BBFBBDCB4EF052
:10135000BECB4FF0BFCB50F0C0CB51F0EDEC63F003
:101360004FC004F050C005F051C006F052C007F065
:1013700004C0E6FF05C0E6FF06C0E6FF07C0E6FFC3
:101380006FEC73F0E552E552E552E5524EC000F0C5
:101390004FC001F050C002F051C003F0BACB0CF0C6
:1013A000BBCB0DF00E6A0F6AE80E536E030E546E3F
:1013B000556A566A0CC04EF00DC04FF00EC050F08A
:1013C0000FC051F037EC73F04AC00CF04BC00DF079
:1013D0004CC00EF04DC00FF00CC04EF00DC04FF0E1
:1013E0000EC050F00FC051F0EDEC63F04FC008F0AC
:1013F00050C009F051C00AF052C00BF008C054F0C0
:1014000009C055F00AC056F00BC057F000C04FF0AD
:1014100001C050F002C051F003C052F006EC64F07D
:10142000B8EC65F050C0B8FB51C0B9FB3C0E006E83
:10143000016ABACB50F0BBCB51F000C055F001C0EF
:1014400056F035EC74F050C0BCFB3C0E0B01BC03F5
:10145000F350006E016A00500B01BA5D0B01BA6FC8
:1014600001500B01BB590B01BB6F12009EAAFED7A6
:101470009E9AAF5000D01200D9CFE6FFE1CFD9FF3E
:10148000ADA2FED7FE0EDB50AE6EE552E7CFD9FF20
:101490001200D9CFE6FFE1CFD9FFA8A2FED7FE0EFA
:1014A000DB50A96EE552E7CFD9FF1200D9CFE6FF96
:1014B000E1CFD9FFE652DF6ADF50E76EFD0EDBCFEA
:1014C000E9FFFE0EDBCFEAFFE750E926000EEA2235
:1014D000EF5012E0DF50E76EFD0EDBCFE9FFFE0EAE
:1014E000DBCFEAFFE750E926000EEA22EF50E66E76
:1014F000D0DFE552DF2AE0D7E552E552E7CFD9FF4A
:101500001200D9CFE6FFE1CFD9FFE652DF6ADF5004
:10151000E76EFD0EDBCFE9FFFE0EDBCFEAFFE75003
:10152000E926000EEA22EF5012E0DF50E76EFD0ED2
:10153000DBCFE9FFFE0EDBCFEAFFE750E926000E26
:10154000EA22EF50E66E98DFE552DF2AE0D7E55257
:10155000E552E7CFD9FF1200D9CFE6FFE1CFD9FF9F
:10156000020EE126100EDE6E270EDD6E8150010B9D
:1015700019E10A010A01AA51200B14E10A010A012A
:10158000A351010B0FE1D9CFE9FFDACFEAFF000E3B
:10159000D880EE54000EED5405E2DF06010E01E2A4
:1015A000DB06E4D781A005D01E0EE66E6FEC74F06A
:1015B000E552020EE15C02E2E16AE552E16EE552BB
:1015C000E7CFD9FF1200D9CFE6FFE1CFD9FFE6522E
:1015D000ACA205D0AC98AF50DF6EAC8802D0AF5053
:1015E000DF6EDF5000D0E552E552E7CFD9FF1200A1
:1015F000D9CFE6FFE1CFD9FFE6520A0EDF6EF3EC5A
:1016000055F00A0EDF6E100EDF5C0EE2DFCFE6FF54
:10161000B0EC56F0E5522DEC55F0320EE66E1EECB5
:1016200074F0E552DF2AEFD7E552E552E7CFD9FF54
:1016300012000A01AAB387D00A01AAB17FD0020121
:101640005D6B5E6B02011A0E5D5D000E5E591FE25E
:101650005DC2E9FF5EC2EAFF020ED890E936EA36C3
:10166000E806FBE1610EE926020EEA22EE500201D5
:101670005927EE5002015A23EE5002015B23EE502F
:1016800002015C2302015D2B000E5E23DBD7910E6D
:10169000006E790E016E0B0E026E4F0E036E8DCA38
:1016A0000CF00D6A0E6A0F6A0CC04EF00DC04FF0C0
:1016B0000EC050F00FC051F059C253F05AC254F04E
:1016C0005BC255F05CC256F037EC73F04AC008F0CC
:1016D0004BC009F04CC00AF04DC00BF008C04EF0F2
:1016E00009C04FF00AC050F00BC051F0EBEC63F0B2
:1016F0004FC004F050C005F051C006F052C007F0D2
:1017000004C054F005C055F006C056F007C057F0AD
:1017100000C04FF001C050F002C051F003C052F0C1
:101720009DEC64F0B8EC65F050C05FF251C060F21F
:101730000201596B5A6B5B6B5C6B03D002015F6BF0
:10174000606B0A01AA8500D01200200E926E300E46
:10175000936EB40E946E410E956EFD0E966E8C9A3D
:10176000898EBA6AF00EBA140409BA6E9F84BC6AF4
:10177000BB6ACD9ECD9CCD82CD8ACD889A6A0F0161
:10178000010E526FCF6ACE6ACD80976A799E799C9E
:101790007982799A798879800F01526B7668A5866B
:1017A000A386A2827B6A7A6AD08E9D84A082829868
:1017B000829C839083948396C26AC280C29EC29C9C
:1017C000C16AC18EC186C188C18AC190C182C184EB
:1017D0000F01EF0E486F0F014969F296F28CF28EFD
:1017E0008C8E8A808A828A848A868B82898C8B807E
:1017F00012000B0EE66EE66AE66AF40EE66E0A0E5C
:10180000E66E29EC72F0006E050EE15E00501200EB
:10181000D9CFE6FFE1CFD9FFE652DF6ADF50006E95
:10182000016A800E005C000E015809E2DF50EA6A8E
:10183000000FE96E0A0EEA22EF6ADF2AEFD70101F4
:10184000A66B00D0E552E552E7CFD9FF12000101A7
:10185000B36B0201306B4D0E0A01045D01E049D308
:10186000430E0A01055D01E044D302013051EA6AEA
:10187000000FE96E0A0EEA22EF502C0803E0020185
:10188000302BF3D70201302B02013051EA6A000FEE
:10189000E96E0A0EEA22EF502C0803E00201302B19
:1018A000F3D70201302B02013051EA6A000FE96ED2
:1018B0000A0EEA22EFCFB3F1410E0101B35D05E15B
:1018C0000A01DE810201518504D00A01DE91020184
:1018D000519502013051EA6A000FE96E0A0EEA22C0
:1018E000EF502C0803E00201302BF3D70201302B1C
:1018F00002011F6B040E02011F5D0CE202011F5169
:10190000EA6A200FE96E020EEA22780EEF6E0201FB
:101910001F2BF0D702013051EA6A000FE96E0A0E60
:10192000EA22EFCF20F202013029EA6A000FE96EC5
:101930000A0EEA22EFCF21F2200EE66E020EE66ECC
:1019400065EC6AF0E552E5524EC0DFFA4FC0E0FAAE
:1019500050C0E1FA51C0E2FA400E536E420E546E8E
:101960000F0E556E566ADFCA4EF0E0CA4FF0E1CA5C
:1019700050F0E2CA51F037EC73F04AC0DFFA4BC0C6
:10198000E0FA4CC0E1FA4DC0E2FA020E0201302743
:1019900002011F6B090E02011F5D0CE202011F51C3
:1019A000EA6A200FE96E020EEA22780EEF6E02015B
:1019B0001F2BF0D702013051EA6A000FE96E0A0EC0
:1019C000EA22EFCF20F202013029EA6A000FE96E25
:1019D0000A0EEA22EFCF21F2030E02013025EA6A55
:1019E000000FE96E0A0EEA22EFCF22F2040E020186
:1019F0003025EA6A000FE96E0A0EEA22EFCF23F2E1
:101A0000050E02013025EA6A000FE96E0A0EEA228D
:101A1000EFCF24F2060E02013025EA6A000FE96ECC
:101A20000A0EEA22EFCF25F20201300E266F0201E4
:101A3000300E276F200EE66E020EE66E65EC6AF041
:101A4000E552E5524EC02CF24FC02DF250C02EF29E
:101A500051C02FF22CC22CF22DC22DF22EC22EF22A
:101A60002FC22FF23C0E536E546A556A566A2CC22E
:101A70004EF02DC24FF02EC250F02FC251F05DEC4F
:101A800065F04EC02CF24FC02DF250C02EF251C066
:101A90002FF202012C510A01DF2702012D510A0108
:101AA000E02302012E510A01E12302012F510A0114
:101AB000E22302013051EA6A000FE96E0A0EEA22BF
:101AC000EF502C0803E00201302BF3D70201302B3A
:101AD00002013051EA6A000FE96E0A0EEA22EFCFE6
:101AE000B3F14E0E0101B35D03E10A01DE9702D0AE
:101AF0000A01DE8702013051EA6A000FE96E0A0E20
:101B0000EA22EF502C0803E00201302BF3D7020148
:101B1000302B02011F6B050E02011F5D0CE202015A
:101B20001F51EA6A200FE96E020EEA22780EEF6E6C
:101B300002011F2BF0D702013051EA6A000FE96E53
:101B40000A0EEA22EFCF20F202013029EA6A000FE2
:101B5000E96E0A0EEA22EFCF21F2020E02013025D1
:101B6000EA6A000FE96E0A0EEA22EFCF22F2200E97
:101B7000E66E020EE66E65EC6AF0E552E5524EC086
:101B8000E3FA4FC0E4FA50C0E5FA51C0E6FA400E5D
:101B9000536E420E546E0F0E556E566AE3CA4EF0E7
:101BA000E4CA4FF0E5CA50F0E6CA51F037EC73F0E2
:101BB0004AC0E3FA4BC0E4FA4CC0E5FA4DC0E6FA7D
:101BC000030E0201302702011F6B090E02011F5D87
:101BD0000CE202011F51EA6A200FE96E020EEA22AE
:101BE000780EEF6E02011F2BF0D702013051EA6A26
:101BF000000FE96E0A0EEA22EFCF20F2020130292F
:101C0000EA6A000FE96E0A0EEA22EFCF21F2030E14
:101C100002013025EA6A000FE96E0A0EEA22EFCFD0
:101C200022F2040E02013025EA6A000FE96E0A0E64
:101C3000EA22EFCF23F2050E02013025EA6A000FF7
:101C4000E96E0A0EEA22EFCF24F2060E02013025D9
:101C5000EA6A000FE96E0A0EEA22EFCF25F20201CE
:101C6000300E266F0201300E276F200EE66E020E38
:101C7000E66E65EC6AF0E552E5524EC02CF24FC0BC
:101C80002DF250C02EF251C02FF22CC22CF22DC2D8
:101C90002DF22EC22EF22FC22FF23C0E536E546A3A
:101CA000556A566A2CC24EF02DC24FF02EC250F02B
:101CB0002FC251F05DEC65F04EC02CF24FC02DF2FA
:101CC00050C02EF251C02FF202012C510A01E3271D
:101CD00002012D510A01E42302012E510A01E523DC
:101CE00002012F510A01E62302013051EA6A000F76
:101CF000E96E0A0EEA22EF502C0803E00201302BB5
:101D0000F3D70201302B02013051EA6A000FE96E6D
:101D10000A0EEA22EFCFB3F1450E0101B35D03E1F4
:101D20000A01DE9502D00A01DE8502013051EA6A1D
:101D3000000FE96E0A0EEA22EF502C0803E00201C0
:101D4000302BF3D70201302B02013051016A000F12
:101D5000006E0A0E012200C0E6FF01C0E6FF03ECA0
:101D60006EF0E552E5524EC0C5F14FC0C6F150C00D
:101D7000C7F151C0C8F1546A556A180E566E430E29
:101D8000576EC5C14FF0C6C150F0C7C151F0C8C1B0
:101D900052F027EC66F0010A3EE1546A556AC80E1B
:101DA000566E420E576EC5C14FF0C6C150F0C7C146
:101DB00051F0C8C152F0F0EC64F0B8EC65F050C0DE
:101DC000E9FA51C0EAFA560E546E0E0E556EED0E3B
:101DD000566E3F0E576EC5C14FF0C6C150F0C7C119
:101DE00051F0C8C152F0F0EC64F04FC0C5F150C0E2
:101DF000C6F151C0C7F152C0C8F1C5C14FF0C6C14C
:101E000050F0C7C151F0C8C152F0B8EC65F050C0F5
:101E1000E7FA51C0E8FA0A01A4930A01140EE75D3B
:101E2000000EE85910E20A01A4830101AE2B000E56
:101E3000AF230101580ED880AE55020EAF5502E215
:101E40000A01A4810AD00A01A4910101AE6BAF6B13
:101E50000101056B066B076B086B02013051EA6AE2
:101E6000000FE96E0A0EEA22EF502C0803E002018F
:101E7000302BF3D70201302B02013051016A000FE1
:101E8000006E0A0E012200C0E6FF01C0E6FF03EC6F
:101E90006EF0E552E5524EC0C5F14FC0C6F150C0DC
:101EA000C7F151C0C8F1546A556AC80E566E420E49
:101EB000576EC5C14FF0C6C150F0C7C151F0C8C17F
:101EC00052F0F0EC64F04FC0C5F150C0C6F151C003
:101ED000C7F152C0C8F1C5C14FF0C6C150F0C7C16B
:101EE00051F0C8C152F0B8EC65F050C0EBFA51C0E7
:101EF000ECFA0A010A01A651040B01E198D00A018B
:101F00000A01A351400B01E092D00A010A01A3513A
:101F1000080B01E08CD001010151021107E0010121
:101F20000107000E025B0A01A39781D062DC020167
:101F3000306B02013051EA6A000FE96E0A0EEA22A4
:101F4000EF502C0803E00201302BF3D70201302BB5
:101F50000101016B026B0101040E015D000E0259CB
:101F60001BE202013051EA6A000FE96E0A0EEA2212
:101F7000EF50E66EF40E01010125E96E0A0E010133
:101F80000221EA6EE552E750EF6E0101012B000ECF
:101F900002230201302BDFD7F40E01010125E96E87
:101FA0000A0E01010221EA6E2C0EEF6E0101012BD7
:101FB000000E02230201206B0201306B090E0201A8
:101FC000205D0FE00201302B02013051EA6A000F60
:101FD000E96E0A0EEA22EF502C0802E10201202BE2
:101FE000EDD70201302B01010B0E015D000E0259ED
:101FF0001BE202013051EA6A000FE96E0A0EEA2282
:10200000EF50E66EF40E01010125E96E0A0E0101A2
:102010000221EA6EE552E750EF6E0101012B000E3E
:1020200002230201302BDFD70A01A38703D008EC7B
:102030000CF000D01200D9CFE6FFE1CFD9FFFC0EA3
:10204000DBCFE9FFFD0EDBCFEAFF000EE926080E2D
:10205000EA22EF502C0806E0FC0EDB2AFD0E01E31D
:10206000DB2AEDD7FC0EDB2AFD0E01E3DB2AFE0E98
:10207000DB500C0A01E15CD3060A01E116D3030A26
:1020800001E1B2D1010A01E19AD10F0A01E182D145
:10209000010A01E110D1030A01E19ED0010A2DE0FD
:1020A000070A16E0010A10E0020A01E056D3FC0E0E
:1020B000DBCFE9FFFD0EDBCFEAFF000EE926080EBD
:1020C000EA22EFCF8BFA49D30A01010E8E6F45D376
:1020D000FC0EDBCF00F0FD0EDBCF01F0000E002682
:1020E000080E012200C0E6FF01C0E6FFF0EC69F037
:1020F000E552E552F3CF8DFA30D3FC0EDBCF00F082
:10210000FD0EDBCF01F0000E0026080E012200C0FC
:10211000E6FF01C0E6FFF0EC69F0E552E552F3CFCF
:1021200096FAFC0EDBCFE9FFFD0EDBCFEAFF000ED7
:10213000E926080EEA22EF502C0806E0FC0EDB2A06
:10214000FD0E01E3DB2AEDD7FC0EDB2AFD0E01E3D9
:10215000DB2AFC0EDBCF00F0FD0EDBCF01F0000E22
:102160000026080E012200C0E6FF01C0E6FFF0ECE9
:1021700069F0E552E552F3CF98FAF4CF99FAFC0EE4
:10218000DBCFE9FFFD0EDBCFEAFF000EE926080EEC
:10219000EA22EF502C0806E0FC0EDB2AFD0E01E3DC
:1021A000DB2AEDD7FC0EDB2AFD0E01E3DB2AFC0E59
:1021B000DBCF00F0FD0EDBCF01F0000E0026080E95
:1021C000012200C0E6FF01C0E6FFF0EC69F0E55235
:1021D000E552F3CF97FAC1D2FC0EDBCF00F0FD0E33
:1021E000DBCF01F0000E0026080E012200C0E6FF42
:1021F00001C0E6FFF0EC69F0E552E552F3CF9AFA40
:10220000FC0EDBCFE9FFFD0EDBCFEAFF000EE92677
:10221000080EEA22EF502C0806E0FC0EDB2AFD0E29
:1022200001E3DB2AEDD7FC0EDB2AFD0E01E3DB2AFE
:10223000FC0EDBCF00F0FD0EDBCF01F0000E002620
:10224000080E012200C0E6FF01C0E6FFF0EC69F0D5
:10225000E552E552F3CF9CFAF4CF9DFAFC0EDBCFAA
:10226000E9FFFD0EDBCFEAFF000EE926080EEA22A9
:10227000EF502C0806E0FC0EDB2AFD0E01E3DB2A02
:10228000EDD7FC0EDB2AFD0E01E3DB2AFC0EDBCFD3
:1022900000F0FD0EDBCF01F0000E0026080E01223B
:1022A00000C0E6FF01C0E6FFF0EC69F0E552E55240
:1022B000F3CF9BFA52D2FC0EDBCF00F0FD0EDBCF4A
:1022C00001F0000E0026080E012200C0E6FF01C04A
:1022D000E6FFF0EC69F0E552E552F3CF9EFAFC0E12
:1022E000DBCFE9FFFD0EDBCFEAFF000EE926080E8B
:1022F000EA22EF502C0806E0FC0EDB2AFD0E01E37B
:10230000DB2AEDD7FC0EDB2AFD0E01E3DB2AFC0EF7
:10231000DBCF00F0FD0EDBCF01F0000E0026080E33
:10232000012200C0E6FF01C0E6FFF0EC69F0E552D3
:10233000E552F3CFA0FAF4CFA1FAFC0EDBCFE9FF10
:10234000FD0EDBCFEAFF000EE926080EEA22EF5071
:102350002C0806E0FC0EDB2AFD0E01E3DB2AEDD79C
:10236000FC0EDB2AFD0E01E3DB2AFC0EDBCF00F0C6
:10237000FD0EDBCF01F0000E0026080E012200C08A
:10238000E6FF01C0E6FFF0EC69F0E552E552F3CF5D
:102390009FFAE3D1FC0EDBCF00F0FD0EDBCF01F0A6
:1023A000000E0026080E012200C0E6FF01C0E6FF75
:1023B000F0EC69F0E552E552F3CF90FACED1FC0E85
:1023C000DBCF00F0FD0EDBCF01F0000E0026080E83
:1023D000012200C0E6FF01C0E6FFF0EC69F0E55223
:1023E000E552F3CF91FAB9D102011F6B0F0E020132
:1023F0001F5D2CE202011F51E96EEA6AD890E936AE
:10240000EA36240EE9260B0EEA22EE6AED6A020194
:102410001F51E96EEA6AD890E936EA363C0EE926A1
:102420000B0EEA22EE6AED6A02011F51040DF3CF92
:10243000E9FFF4CFEAFF540EE9260B0EEA22EE6A1A
:10244000EE6AEE6AEE6A02011F2BD0D70B011A6BFF
:10245000FC0EDBCF00F0FD0EDBCF01F0000E0026FE
:10246000080E012200C0E6FF01C0E6FF65EC6AF03D
:10247000E552E5524EC020FB4FC021FB50C022FB6D
:1024800051C023FBFC0EDBCFE9FFFD0EDBCFEAFFE3
:10249000000EE926080EEA22EF502C0806E0FC0E9A
:1024A000DB2AFD0E01E3DB2AEDD7FC0EDB2AFD0E55
:1024B00001E3DB2AFC0EDBCF00F0FD0EDBCF01F0E9
:1024C000000E0026080E012200C0E6FF01C0E6FF54
:1024D00065EC6AF0E552E5524EC01CFB4FC01DFB97
:1024E00050C01EFB51C01FFBFC0EDBCFE9FFFD0EF1
:1024F000DBCFEAFF000EE926080EEA22EF502C0897
:1025000006E0FC0EDB2AFD0E01E3DB2AEDD7FC0E14
:10251000DB2AFD0E01E3DB2AFC0EDBCF00F0FD0E13
:10252000DBCF01F0000E0026080E012200C0E6FFFE
:1025300001C0E6FF97EC69F0E552E5520B011A6F16
:1025400002011F6B0B011A5102011F5D01E37DD0D7
:10255000FC0EDBCFE9FFFD0EDBCFEAFF000EE92624
:10256000080EEA22EF502C0806E0FC0EDB2AFD0ED6
:1025700001E3DB2AEDD7FC0EDB2AFD0E01E3DB2AAB
:10258000FC0EDBCF02F0FD0EDBCF03F0000E0226C7
:10259000080E032202C0E6FF03C0E6FFF0EC69F07C
:1025A000E552E552F3CF00F0F4CF01F002011F51E4
:1025B000E96EEA6AD890E936EA36240EE9260B0E6F
:1025C000EA2200C0EEFF01C0EDFFFC0EDBCFE9FF09
:1025D000FD0EDBCFEAFF000EE926080EEA22EF50DF
:1025E0002C0806E0FC0EDB2AFD0E01E3DB2AEDD70A
:1025F000FC0EDB2AFD0E01E3DB2AFC0EDBCF02F032
:10260000FD0EDBCF03F0000E0226080E032202C0EF
:10261000E6FF03C0E6FFF0EC69F0E552E552F3CFC8
:1026200000F0F4CF01F002011F51E96EEA6AD89080
:10263000E936EA363C0EE9260B0EEA2200C0EEFF30
:1026400001C0EDFF02011F2B7DD7FC0EDBCFE9FFA0
:10265000FD0EDBCFEAFF000EE926080EEA22EF505E
:102660002A0806E0FC0EDB2AFD0E01E3DB2AEDD78B
:10267000D950FC0FE96EFF0EDA20EA6EEE06000E6E
:10268000ED5A0B01020E1B6FFC0EDBCFE9FFFD0EB6
:10269000DBCFEAFF000EE926080EEA22EF503108F0
:1026A00003E10B01010E1B6F58D0FC0EDBCF00F0D5
:1026B000FD0EDBCF01F0000E0026080E012200C047
:1026C000E6FF01C0E6FFF0EC69F0E552E552F3CF1A
:1026D00092FAFC0EDBCFE9FFFD0EDBCFEAFF000E26
:1026E000E926080EEA22EF502C0806E0FC0EDB2A51
:1026F000FD0E01E3DB2AEDD7FC0EDB2AFD0E01E324
:10270000DB2AFC0EDBCF00F0FD0EDBCF01F0000E6C
:102710000026080E012200C0E6FF01C0E6FFF0EC33
:1027200069F0E552E552F3CF93FAF4CF94FA15D05D
:10273000FC0EDBCF00F0FD0EDBCF01F0000E00261B
:10274000080E012200C0E6FF01C0E6FFF0EC69F0D0
:10275000E552E552F3CF95FA00D0E552E7CFD9FF25
:102760001200D9CFE6FFE1CFD9FF020EE126DE6AE3
:10277000DD6AE66A020EE66EE668000EE66E080E98
:10278000E66E29EC72F0006E050EE15E0050ACECD6
:102790000AF0000EE66E080EE66EB8EC5AF0E5524E
:1027A000E552000901E09AD00B0EE66EE66ADB0EF8
:1027B000006EDE0E016E026A00C0E6FF01C0E6FF99
:1027C00002C0E6FFDECF03F0DDCF04F0000E0326EB
:1027D000080E042203C0E6FF04C0E6FF06EC72F018
:1027E000056E070EE15E05500B0EDE26000EDD22A3
:1027F000020EE66EE66AD30E006EDF0E016E026A0E
:1028000000C0E6FF01C0E6FF02C0E6FFDECF03F036
:10281000DDCF04F0000E0326080E042203C0E6FFFD
:1028200004C0E6FF06EC72F0056E070EE15E05508F
:10283000020EDE26000EDD22110EE66EE66AE70EBF
:10284000006EDE0E016E026A00C0E6FF01C0E6FF08
:1028500002C0E6FFDECF03F0DDCF04F0000E03265A
:10286000080E042203C0E6FF04C0E6FF06EC72F087
:10287000056E070EE15E0550110EDE26000EDD220C
:10288000020EE66EE66AD30E006EDF0E016E026A7D
:1028900000C0E6FF01C0E6FF02C0E6FFDECF03F0A6
:1028A000DDCF04F0000E0326080E042203C0E6FF6D
:1028B00004C0E6FF06EC72F0056E070EE15E0550FF
:1028C000020EDE26000EDD22ACEC0AF0000EE66EF3
:1028D000080EE66E00EC5BF0E552E5520A01460E8A
:1028E0008B6F0A01280E8C6F0A01A3890A018D6B78
:1028F0000A018E6B0B011B6B0A01916B0A01906B35
:102900000A01926B0A01936B946B0A01956B0A01A1
:10291000976B0A01966B0A01986B996B0A019B6B86
:102920000A019A6B0A019C6B9D6B0A019F6B0A015D
:102930009E6B0A01A06BA16B0B011A6BDE6ADD6A4C
:10294000DECF00F0DDCF01F0000E005C020E01587A
:1029500033E2DECFE9FFDDCFEAFF000EE926080E05
:10296000EA22EF50240823E1DECFE6FFDDCFE6FFC9
:10297000DECF00F0DDCF01F0000E0026080E0122B0
:10298000010E0026000E012200C0E6FF01C0E6FF96
:10299000F0EC69F0E552E552F350E66E1BEC10F0F6
:1029A000E552E552E552DF2A010E01E3DB2ADF2A78
:1029B000010E01E3DB2AC4D70A018D5102E1BA6A94
:1029C00000D00A018F6B0101B40508E0020E01017D
:1029D000B45D04E0030E0101B45D03E10A01960E4B
:1029E0008F6F0B010E0E176F0A018D5103E0020E5F
:1029F0000B0117270A018E5103E0090E0B0117275F
:102A0000960E0101C36FC46B0B011B0505E10101AB
:102A10002C0EC36F010EC46F0A01A3970A01A69181
:102A2000020EE15C02E2E16AE552E16EE552E7CFB7
:102A3000D9FF1200D9CFE6FFE1CFD9FF040EE1267E
:102A4000DE6ADD6A020EDB6A030EDB6AE66A020EEC
:102A5000E66EE668000EE66E060EE66E29EC72F093
:102A6000006E050EE15E0050E66A020EE66EE66854
:102A7000000EE66E080EE66E29EC72F0006E050E92
:102A8000E15E0050ACEC0AF0000EE66E060EE66E5B
:102A9000B8EC5AF0E552E552DE6ADD6ADECF00F0AE
:102AA000DDCF01F0000E005C020E015801E39DD164
:102AB000DECFE9FFDDCFEAFF000EE926060EEA22AF
:102AC000EF5024085BE1DECFE9FFDDCFEAFF010E26
:102AD000E926000EEA22000EE926060EEA22EF5051
:102AE00030084CE1DECFE9FFDDCFEAFF020EE92638
:102AF000000EEA22000EE926060EEA22EF502C080C
:102B00003DE1DECFE9FFDDCFEAFF000EE926060E4C
:102B1000EA22EF500A0821E0DECFE9FFDDCFEAFF2D
:102B2000000EE926060EEA22EF50E66E020EDBCF1B
:102B3000E9FF030EDBCFEAFF000EE926080EEA22CA
:102B4000E552E750EF6EDF2A010E01E3DB2A020EA9
:102B5000DB2A030E01E3DB2AD4D7020EDBCFE9FF29
:102B6000030EDBCFEAFF000EE926080EEA220A0E6A
:102B7000EF6E020EDB2A030E01E3DB2ADECFE9FF54
:102B8000DDCFEAFF000EE926060EEA22EF50240808
:102B90005BE1DECFE9FFDDCFEAFF010EE926000EA3
:102BA000EA22000EE926060EEA22EF5031084CE137
:102BB000DECFE9FFDDCFEAFF020EE926000EEA22B2
:102BC000000EE926060EEA22EF502C083DE1DECF8A
:102BD000E9FFDDCFEAFF000EE926060EEA22EF50FC
:102BE0000A0821E0DECFE9FFDDCFEAFF000EE9268B
:102BF000060EEA22EF50E66E020EDBCFE9FF030E6F
:102C0000DBCFEAFF000EE926080EEA22E552E75084
:102C1000EF6EDF2A010E01E3DB2A020EDB2A030E30
:102C200001E3DB2AD4D7020EDBCFE9FF030EDBCFB3
:102C3000EAFF000EE926080EEA220A0EEF6E020EE7
:102C4000DB2A030E01E3DB2ADECFE9FFDDCFEAFF5B
:102C5000000EE926060EEA22EF5024085BE1DECFE3
:102C6000E9FFDDCFEAFF010EE926000EEA22000EA1
:102C7000E926060EEA22EF5032084CE1DECFE9FFEA
:102C8000DDCFEAFF020EE926000EEA22000EE92659
:102C9000060EEA22EF502C083DE1DECFE9FFDDCF42
:102CA000EAFF000EE926060EEA22EF500A0821E0AC
:102CB000DECFE9FFDDCFEAFF000EE926060EEA22AD
:102CC000EF50E66E020EDBCFE9FF030EDBCFEAFF2B
:102CD000000EE926080EEA22E552E750EF6EDF2AE1
:102CE000010E01E3DB2A020EDB2A030E01E3DB2ADD
:102CF000D4D7020EDBCFE9FF030EDBCFEAFF000ED5
:102D0000E926080EEA220A0EEF6E020EDB2A030EF7
:102D100001E3DB2ADECFE9FFDDCFEAFF000EE92683
:102D2000060EEA22EF5024085BE1DECFE9FFDDCF9B
:102D3000EAFF010EE926000EEA22000EE926060E41
:102D4000EA22EF5033084CE1DECFE9FFDDCFEAFFA6
:102D5000020EE926000EEA22000EE926060EEA22FD
:102D6000EF502C083DE1DECFE9FFDDCFEAFF000E9A
:102D7000E926060EEA22EF500A0821E0DECFE9FF3D
:102D8000DDCFEAFF000EE926060EEA22EF50E66EDE
:102D9000020EDBCFE9FF030EDBCFEAFF000EE926D0
:102DA000080EEA22E552E750EF6EDF2A010E01E33A
:102DB000DB2A020EDB2A030E01E3DB2AD4D7020E44
:102DC000DBCFE9FF030EDBCFEAFF000EE926080E9A
:102DD000EA220A0EEF6E020EDB2A030E01E3DB2A63
:102DE000DF2A010E01E3DB2A59D6040EE15C02E280
:102DF000E16AE552E16EE552E7CFD9FF1200D9CF83
:102E0000E6FFE1CFD9FFE652DF6ADF50006E016ACC
:102E1000100E005C000E015814E2EA6ADF34FE0B6B
:102E2000EA36E96EBB0EE9260A0EEA22EE6AED6A80
:102E3000DF50EA6AAB0FE96E0A0EEA22EF6ADF2A78
:102E4000E4D70A01DB6BE552E552E7CFD9FF120068
:102E5000D9CFE6FFE1CFD9FFE6520A01AAB947D0A0
:102E60000A01DB5132E0DF6ADF50006E016A100EAA
:102E7000005C000E015828E20A01DB51026E036A71
:102E8000EA6ADF34FE0BEA36E96EBB0EE9260A0E6B
:102E9000EA22EECF00F0EFCF01F000C050F001C009
:102EA00051F002C055F003C056F035EC74F05050AC
:102EB000E66EDF50EA6AAB0FE96E0A0EEA22E552CF
:102EC000E750EF6EDF2AD0D712D0DF6ADF50006EF6
:102ED000016A100E005C000E015809E2DF50EA6A38
:102EE000AB0FE96E0A0EEA22EF6ADF2AEFD7E5524E
:102EF000E552E7CFD9FF1200D9CFE6FFE1CFD9FFE6
:102F00000101000EAC5D020EAD590BE2000E010195
:102F1000AC25E96E060E0101AD21EA6EFE0EDBCF97
:102F2000EFFF0101AC2B000EAD23E552E7CFD9FF37
:102F300012000A01AA9B0101A45121E0A4C14EF094
:102F40004F6A506A516A53685468556A566A37EC3A
:102F500073F04A500101A0250101A06F4B500101FF
:102F6000A1210101A16F4C500101A2210101A26F19
:102F70004D500101A3210101A36F0101A46B0201C6
:102F8000C951040DF3CFE9FFF4CFEAFF610EE92642
:102F9000020EEA22A0C1EEFFA1C1EEFFA2C1EEFF28
:102FA000A3C1EEFF0201C92B1A0E0201C95D02E1A5
:102FB0000201C96B0101A46B1200D9CFE6FFE1CF7A
:102FC000D9FFE6520A018D5104E102015F6B606B8B
:102FD00002D019EC0BF05FC20CFB60C20DFB0A01C2
:102FE0008D510EE002015F510C01315D0201605113
:102FF0000C01325904E25FC231FC60C232FC0DD0D8
:103000000A01E7510C01315D0A01E8510C01325906
:1030100004E2E7CA31FCE8CA32FC0C0160B115D009
:103020000A018E0512E1ABCA0EFBACCA0FFBADCA9A
:1030300010FBAECA11FBAFCA12FBB0CA13FBB1CA78
:1030400014FBB2CA15FBB3CA16FB0A01A3A309D02D
:103050000A01A3938B82898C8B80010EE66E84DA41
:10306000E5520A01DE930A01A3A92CD00A01A3AB01
:103070000FD08B92899C8B90020EE66E75DAE5522A
:103080000A01A3830A01A3990A01DE830A01A39B13
:103090000A018C51360DF3CF00F0F4CF01F00B0193
:1030A0000851005C095101580DE28B92899C8B906C
:1030B000020EE66E59DAE5520A01A3830A01A399CA
:1030C0000A01DE83DECAFFFA0C0160A17CD00A018E
:1030D000FF810B01002B000E012302230323E3CA0F
:1030E00004FBE4CA05FBE5CA06FBE6CA07FB640E5F
:1030F0000B010827000E0B01092308CBE7FA09CBC7
:10310000E8FA0B01200E085D4E0E095904E3140E77
:103110000B01086F096B640E0B010A27000E0B01EF
:103120000B230ACB00F00BCB01F0026AD8900250BF
:10313000000A06E6A00E005C8C0E0158000E025834
:1031400003E30B010A6B0B6B0A01A5830B01940EC1
:10315000F56F810EF66FD70EF76FF86B0B01390E16
:10316000F96F300EFA6FFB6BFC6B0B01320EFD6FCB
:10317000090EFE6F010EFF6F006B0C01400E016F18
:10318000E20E026F010E036F046B0C01FA0E056F65
:10319000920E066F030E076F086B0A018E0512E18F
:1031A000ABCA0EFBACCA0FFBADCA10FBAECA11FB1B
:1031B000AFCA12FBB0CA13FBB1CA14FBB2CA15FBEB
:1031C000B3CA16FB18D0E3CA04FBE4CA05FBE5CA80
:1031D00006FBE6CA07FBDFCA00FBE0CA01FBE1CA47
:1031E00002FBE2CA03FBE9CA08FBEACA09FBEBCA15
:1031F0000AFBECCA0BFB0101AC6BAD6BDF6ADF5065
:10320000006E016A0D0E005C000E01580DE2DF50E9
:103210000101EA6AB925E96EBA51EA22EF50E66E79
:103220006BDEE552DF2AEBD70A018D5116E0DF6A2B
:10323000DF50006E016A020E005C000E01580DE2C4
:10324000DF500101EA6ABD25E96EBE51EA22EF5066
:10325000E66E52DEE552DF2AEBD70A018E0516E153
:10326000DF6ADF50006E016A090E005C000E015833
:103270000DE2DF500101EA6ABB25E96EBC51EA228A
:10328000EF50E66E39DEE552DF2AEBD70A01A58161
:10329000E552E552E7CFD9FF1200D9CFE6FFE1CFE3
:1032A000D9FF020EE126DE6ADD6A0A019651030AA1
:1032B0000FE0010A08E0030A01E00FD0E7CADEFFD1
:1032C000E8CADDFF0AD00CCBDEFF0DCBDDFF05D059
:1032D0000C012A51DE6EDD6A00D0DECF00F0DDCFBA
:1032E00001F00A019851005C9951015805E2010171
:1032F0000A0EA96F8B8014D00A01970502E18B900A
:103300000FD0020E0A01975D07E10101A95104E007
:103310008B700101A90703D00101A96B8B8000D03C
:10332000020EE15C02E2E16AE552E16EE552E7CFAE
:10333000D9FF1200D9CFE6FFE1CFD9FF020EE12677
:10334000DE6ADD6A0A01A2990A019A51040A4EE076
:10335000010A3AE0060A27E0010A14E0030A01E044
:103360004CD0E7CADEFFE8CADDFFDECF00F0DDCFDC
:1033700001F00A019C51005C9D51015802E20A01D2
:10338000A2893BD00CCBDEFF0DCBDDFFDECF00F002
:10339000DDCF01F00A019C51005C9D51015802E211
:1033A0000A01A2892AD00C012A51DE6EDD6ADECF25
:1033B00000F0DDCF01F00A019C51005C9D510158E5
:1033C00002E20A01A28919D00C015235000E5219ED
:1033D00009E6D880000E4F55000E5055000E51558D
:1033E000000E525502E20A01A28907D00C01800E9C
:1033F000521502E00A01A28900D00A01A2B906D042
:1034000001010A0EAA6F898C8C8617D00A019B05D0
:1034100003E1899C8C9611D0020E0A019B5D08E1A4
:103420000101AA5105E0897C8C760101AA0704D02C
:103430000101AA6B898C8C8600D0020EE15C02E24D
:10344000E16AE552E16EE552E7CFD9FF1200D9CF2C
:10345000E6FFE1CFD9FF020EE126DE6ADD6A0A014E
:10346000A29B0A019E51040A4EE0010A3AE0060AB4
:1034700027E0010A14E0030A01E04CD0E7CADEFFAE
:10348000E8CADDFFDECF00F0DDCF01F00A01A05178
:10349000005CA151015802E20A01A28B3BD00CCB87
:1034A000DEFF0DCBDDFFDECF00F0DDCF01F00A0146
:1034B000A051005CA151015802E20A01A28B2AD05E
:1034C0000C012A51DE6EDD6ADECF00F0DDCF01F0A7
:1034D0000A01A051005CA151015802E20A01A28B2D
:1034E00019D00C015235000E521909E6D880000E91
:1034F0004F55000E5055000E5155000E525502E228
:103500000A01A28B07D00C01800E521502E00A01BD
:10351000A28B00D00A01A2BB06D001010A0EAB6F3C
:103520008B828C8417D00A019F0503E18B928C94C7
:1035300011D0020E0A019F5D08E10101AB5105E0C7
:103540008B728C740101AB0704D00101AB6B8B82D1
:103550008C8400D0020EE15C02E2E16AE552E16E89
:10356000E552E7CFD9FF1200D9CFE6FFE1CFD9FF6F
:10357000FE0EDB50020A45E0030A36E0010A01E0D4
:1035800045D00C015BAD2FD00C015E2B140E0C014D
:103590005E5D1AE18A868A840C015BB78A960C010B
:1035A0005BBB8A940C015B9D0C015E6B0C015BAFF5
:1035B0000AD08A828A800C015BB58A920C015BB9C1
:1035C0008A900C015B9F0FD00C015BB78A760C01CF
:1035D0005BBB8A740C015BAF06D00C015BB58A72D1
:1035E0000C015BB98A7012D08A868A848A828A80AA
:1035F0000C015B950C015B970C015B990C015B9BCB
:1036000005D08A968A948A928A9000D000D0E5529A
:10361000E7CFD9FF12000A01A6930101AC6BAD6B95
:10362000E66A020EE66EE66A000EE66E060EE66ECC
:1036300029EC72F0006E050EE15E0050E66A020EA3
:10364000E66EE66A000EE66E080EE66E29EC72F093
:10365000006E050EE15E0050E3EC5BF04EC0CAF276
:103660004FC0CBF250C0CCF251C0CDF212000A01D3
:10367000A69B010EE66E78DFE5521200D9CFE6FF79
:10368000E1CFD9FF020EE126DF6A0F0E0601001519
:103690000601006F02011EA705D0400E06010011B1
:1036A0000601006F02011EAB05D0200E06010011BD
:1036B0000601006F02011EA905D0100E06010011BF
:1036C0000601006F010EDB6ADF6A0B011705DF5C84
:1036D00010E2DF50EA6A000FE96E060EEA22010EE0
:1036E000DBCFE7FFEF50E71A010EE7CFDBFFDF2A62
:1036F000ECD7DF50EA6A000FE96E060EEA22010EEF
:10370000DBCFEFFF0A01A6B793D017CB00F0016A19
:10371000026A036A00500201CA5F01500201CB5BDA
:1037200002500201CC5B03500201CD5B0101006B32
:10373000DF6A0B011751DF5C2EE2DFCF01F0026A76
:10374000036A046ACA0EE96E020EEA6EEE500126A2
:10375000EE500222EE500322EE50042201C0E6FF9A
:1037600002C0E6FF03C0E6FF04C0E6FF3BEC61F0E9
:10377000E552E552E552E552006EDF50EA6A000F6D
:10378000E96E080EEA22EF50005C03E00101010E31
:10379000006FDF2ACED70101005142E0200EE66E15
:1037A000E66AE66A320EE66E080EE66E29EC72F004
:1037B000006E050EE15E00500B011751E66EE66AE1
:1037C000320EE66E080EE66ECAC2E6FFCBC2E6FF18
:1037D000CCC2E6FFCDC2E6FFE1EC60F0006E080E61
:1037E000E15E00500B0117510201CA27000ECB23E6
:1037F000CC23CD230B011751E66EE66A000EE66E70
:10380000080EE66ECAC2E6FFCBC2E6FFCCC2E6FFF8
:10381000CDC2E6FFE1EC60F0006E080EE15E005004
:103820000B0117510201CA27000ECB23CC23CD2355
:103830000B011751E66EE66A000EE66E060EE66EA6
:10384000CAC2E6FFCBC2E6FFCCC2E6FFCDC2E6FFAE
:10385000E1EC60F0006E080EE15E0050DF6A0B01E3
:103860001751DF5C13E2DF50EA6A000FE96E060EC3
:10387000EA22EF50E66EDF50EA6A000FE96E080EAA
:10388000EA22E552E750EF6EDF2AE9D70B01175124
:103890000201CA27000ECB23CC23CD230A01A59118
:1038A0000A01A697020EE15C02E2E16AE552E16ECE
:1038B000E552E7CFD9FF1200D9CFE6FFE1CFD9FF1C
:1038C000030EE126DF6AD950010FE96EDACFEAFF75
:1038D000F50EEE6E0B0EED6ED880CB0E0201CE55BE
:1038E000FF0ECF551F0ED055000ED15501E2E8D086
:1038F0000A01A6B99AD0340E0201CE5F000E020171
:10390000CF5B000E0201D05B000E0201D15B010112
:10391000006BDF6A340EDF5C33E2DFCF01F0026A56
:10392000036A046ACE0EE96E020EEA6EEE500126BC
:10393000EE500222EE500322EE50042201C0E6FFB8
:1039400002C0E6FF03C0E6FF04C0E6FF3BEC61F007
:10395000E552E552E552E552006EDF50E96EEA6A43
:10396000800EE926000EEA22000EE926080EEA2261
:10397000EF50005C03E00101010E006FDF2ACAD79F
:103980000101005146E0340EE66EE66AE66A800EFA
:10399000E66E080EE66E29EC72F0006E050EE15E32
:1039A0000050340EE66EE66A800EE66E080EE66E95
:1039B000CEC2E6FFCFC2E6FFD0C2E6FFD1C2E6FF2D
:1039C000E1EC60F0006E080EE15E0050340E020182
:1039D000CE27000E0201CF23000E0201D023000EDD
:1039E0000201D123340EE66EE66A010EDBCFE6FF5C
:1039F000020EDBCFE6FFCEC2E6FFCFC2E6FFD0C2AB
:103A0000E6FFD1C2E6FFE1EC60F0006E080EE15E79
:103A10000050340E0201CE27000E0201CF23000E0B
:103A20000201D023000E0201D123340EE66EE66AB5
:103A3000010EDBCFE6FF020EDBCFE6FFCEC2E6FFD4
:103A4000CFC2E6FFD0C2E6FFD1C2E6FFE1EC60F0F4
:103A5000006E080EE15E0050DF6A340EDF5C1EE28D
:103A6000DF50E76E010EDBCFE9FF020EDBCFEAFF8E
:103A7000E750E926000EEA22EF50E66EDF50E96ECD
:103A8000EA6A800EE926000EEA22000EE926080EF8
:103A9000EA22E552E750EF6EDF2ADFD7340E02014B
:103AA000CE27000E0201CF23000E0201D023000E0C
:103AB0000201D1230A01A5930A01A699DEEC24F0A4
:103AC000030EE15C02E2E16AE552E16EE552E7CF06
:103AD000D9FF1200DEEC5CF04EC0CEF24FC0CFF248
:103AE00050C0D0F251C0D1F23BEC5FF00A01A69B6E
:103AF0000C012E6B0C012F6B306B0C012A6B0A0131
:103B0000A6890A01A593DEEC24F01200D9CFE6FFC6
:103B1000E1CFD9FF020EE126DE6ADD6AE3EC5BF05D
:103B20004EC0CAF24FC0CBF250C0CCF251C0CDF261
:103B30001AEC15F00101AC6BAD6BE66A020EE66E95
:103B4000E66A000EE66E060EE66E29EC72F0006E76
:103B5000050EE15E0050240EE66E7CEC17F0E55297
:103B6000DE6ADD6ADECF00F0DDCF01F0020E005C20
:103B7000000E015812E2DECFE9FFDDCFEAFFD70EDB
:103B8000E926010EEA22EF50E66E7CEC17F0E552D2
:103B9000DF2A010E01E3DB2AE5D72C0EE66E7CEC72
:103BA00017F0E552DE6ADD6ADECF00F0DDCF01F00E
:103BB000020E005C000E015813E2DECFF6FFDDCFEF
:103BC000F7FFD80EF626DE0EF7220800F550E66E57
:103BD0007CEC17F0E552DF2A010E01E3DB2AE4D783
:103BE0002C0EE66E7CEC17F0E552DE6ADD6ADECF65
:103BF00000F0DDCF01F0020E005C000E015812E271
:103C0000DECFE9FFDDCFEAFFDA0EE926010EEA2278
:103C1000EF50E66E7CEC17F0E552DF2A010E01E36F
:103C2000DB2AE5D72A0EE66E7CEC17F0E5520D0E86
:103C3000E66E7CEC17F0E5520A0EE66E7CEC17F0AF
:103C4000E552DE6ADD6ADECFE9FFDDCFEAFF000E76
:103C5000E926080EEA22EF50FF0812E0DECFE9FF66
:103C6000DDCFEAFF000EE926080EEA22EF50E66EED
:103C70007CEC17F0E552DF2A010E01E3DB2AE3D7E3
:103C8000240EE66E7CEC17F0E552540EE66E7CECEA
:103C900017F0E5522C0EE66E7CEC17F0E5520C01A5
:103CA00060B11ED0DE6ADD6ADECF00F0DDCF01F04C
:103CB0000B0E005C000E015812E2DECFE9FFDDCFF3
:103CC000EAFFF40EE9260A0EEA22EF50E66E7CECDB
:103CD00017F0E552DF2A010E01E3DB2AE5D720D0F9
:103CE000DE6ADD6ADECFF6FFDDCFF7FF3B0EF6269C
:103CF000E00EF7220800F55013E0DECFF6FFDDCF2F
:103D0000F7FF3B0EF626E00EF7220800F550E66EB0
:103D10007CEC17F0E552DF2A010E01E3DB2AE2D743
:103D20000D0EE66E7CEC17F0E5520A0EE66E7CECAA
:103D300017F0E552DE6ADD6ADECFF6FFDDCFF7FF72
:103D4000D50EF626DF0EF7220800F55013E0DECF81
:103D5000F6FFDDCFF7FFD50EF626DF0EF7220800BF
:103D6000F550E66E7CEC17F0E552DF2A010E01E318
:103D7000DB2AE2D70D0EE66E7CEC17F0E5520A0E58
:103D8000E66E7CEC17F0E552240EE66E7CEC17F044
:103D9000E5522C0EE66E7CEC17F0E55217CBE6FFF1
:103DA0007CEC17F0E5520D0EE66E7CEC17F0E55258
:103DB0000A0EE66E7CEC17F0E552ACEC0AF0ACC1F2
:103DC000E6FFADC1E6FF000EE66E060EE66E78EC8D
:103DD0005BF0E552E552E552E5520A01A6830A017D
:103DE000A5910A01A39B0A01A6870A01A3930A01D0
:103DF000A3890101BF6BC06BC16BC26B0101A86BD2
:103E0000E66A020EE66EE66A000EE66E080EE66EE2
:103E100029EC72F0006E050EE15E0050020EE15CCE
:103E200002E2E16AE552E16EE552E7CFD9FF120006
:103E30000C0160A102D0010E59D00A01DEA122D0EE
:103E40000A01A6810201518501010351041110E00C
:103E500001010307000E045B0A01A6950A01A3975E
:103E60000101580E016F020E026F000E3FD009D003
:103E70000A01A6850A01A3B704D00A01A899000E79
:103E800035D011D00A01A691020151950101080E09
:103E9000036F070E046F0A01A6950A01A3970A0192
:103EA000A899000E23D0460E0A018B5D02E1010E97
:103EB0001DD0500E0A018B5D17E10A01140ED88047
:103EC000E755000EE85502E2010E10D00A01A8A93C
:103ED00007D00A01A89984B4FED7010E07D004D0F8
:103EE0000A01A899000E02D0000E00D01200D9CF0E
:103EF000E6FFE1CFD9FF020EE126DE6ADD6A0401AA
:103F0000E05103E035EC4BF0FAD7DECF00F0DDCF27
:103F100001F0000E005C020E015823E235EC4BF07C
:103F20000401E0511DE1FD0EDBCF00F0FE0EDBCF02
:103F300001F0DE50000100240401E16FDD500001BA
:103F400001200401E26F0401400EE56F0401010E3F
:103F5000E66F0401010EE06F400EDE26000EDD224A
:103F6000D4D7020EE15C02E2E16AE552E16EE5526D
:103F7000E7CFD9FF1200E3EC5BF04EC0D2F24FC0A6
:103F8000D3F250C0D4F251C0D5F20201CA6B200E58
:103F9000CB6FCC6BCD6B0401E05103E035EC4BF003
:103FA000FAD7CA0EE96E020EEA6E0201D251EE5C39
:103FB0000201D351EE580201D451EE580201D551FD
:103FC000EE581EE235EC4BF00401E05118E162ECD2
:103FD0005BF0000EE66E060EE66E89DFE552E552F6
:103FE000020E0201CB27000E0201CC23000E0201BB
:103FF000CD230401E05103E035EC4BF0FAD7D1D7E3
:10400000CBEC48F012000201D269EF0ED36F1F0E05
:10401000D46FD56B0201CA6B100ECB6FCC6BCD6B1E
:104020000401E05103E035EC4BF0FAD7CA0EE96E1B
:10403000020EEA6E0201D251EE5C0201D351EE583B
:104040000201D451EE580201D551EE581EE235EC72
:104050004BF00401E05118E162EC5BF0000EE66EFB
:10406000060EE66E44DFE552E552020E0201CB2752
:10407000000E0201CC23000E0201CD230401E05109
:1040800003E035EC4BF0FAD7D1D7CBEC48F0120077
:10409000D9CFE6FFE1CFD9FF020EE126DE6ADD6A65
:1040A000000EE66E060EE66EB8EC5AF0E552E552EA
:1040B000DECF00F0DDCF01F0000E005C020E0158F3
:1040C0001DE235EC4BF00401E05117E1DECFE1F4E5
:1040D000DDCFE2F4000E0401E127060E0401E22325
:1040E0000401080EE56F0401010EE66F0401010EE4
:1040F000E06F080EDE26000EDD22DAD7020EE15C4C
:1041000002E2E16AE552E16EE552E7CFD9FF120023
:10411000D9CFE6FFE1CFD9FF020EE126DE6ADD6AE4
:10412000E66A020EE66EE668000EE66E060EE66EC3
:1041300029EC72F0006E050EE15E0050E66A020E98
:10414000E66EE668000EE66E080EE66E29EC72F08A
:10415000006E050EE15E005001019B6B9C6B01013E
:104160009D6B9E6B0101FF0E9B5D010E9C593AE217
:1041700035EC4BF0400EE66E000EE66E080EE66E75
:10418000C9EC67F0E552E552E55200092AE0040166
:10419000DF5101019D6F9E6B01019F6B01019D51DC
:1041A00001019F5D000E01019E551BE201019F511F
:1041B000EA6A000FE96E080EEA22EF50E66E000E82
:1041C00001019B25E96E060E01019C21EA6EE55274
:1041D000E750EF6E01019B2B000E9C2301019F2BEA
:1041E000DDD7C0D7DE68010EDD6EDECFE9FFDDCFA3
:1041F000EAFF000EE926060EEA22EF502A080EE03A
:10420000DECFE9FFDDCFEAFF000EE926060EEA2247
:10421000EF68DF06010E01E2DB06E7D700D0020EF1
:10422000E15C02E2E16AE552E16EE552E7CFD9FFD7
:104230001200500EE66EE66AE66A4B0EE66E010E5E
:10424000E66E29EC72F0006E050EE15E0050010191
:104250009B6B9C6B01019F6B01019D6B9E6B120020
:10426000470E01014C5D12E1500E01014D5D0EE162
:10427000430E01014E5D0AE14F0E01014F5D06E163
:104280004E0E0101505D02E1040E79D1470E01018D
:104290004C5D12E1450E01014D5D0EE1440E010140
:1042A0004E5D0AE1410E01014F5D06E1540E010130
:1042B000505D02E1050E63D1470E01014C5D12E134
:1042C000450E01014D5D0EE1430E01014E5D0AE117
:1042D0004E0E01014F5D06E1460E0101505D02E107
:1042E000060E4DD1530E01014C5D12E1450E010148
:1042F0004D5D0EE1430E01014E5D0AE14E0E0101DE
:104300004F5D06E1460E0101505D02E1070E37D117
:10431000470E01014C5D12E1450E01014D5D0EE1BC
:10432000430E01014E5D0AE14C0E01014F5D06E1B5
:104330004F0E0101505D02E1080E21D1530E010123
:104340004C5D12E1450E01014D5D0EE1430E010190
:104350004E5D0AE14C0E01014F5D06E1520E010176
:10436000505D02E10A0E0BD1530E01014C5D12E1CA
:10437000450E01014D5D0EE1430E01014E5D0AE166
:10438000410E01014F5D06E14C0E0101505D02E15D
:10439000130EF5D0470E01014C5D12E1450E0101EF
:1043A0004D5D0EE14D0E01014E5D0AE1450E01012C
:1043B0004F5D06E14D0E0101505D02E10B0EDFD0B5
:1043C000470E01014C5D12E1450E01014D5D0EE10C
:1043D0004D0E01014E5D0AE1450E01014F5D06E102
:1043E000540E0101505D02E1200EC9D0470E0101BB
:1043F0004C5D12E1450E01014D5D0EE1430E0101E0
:104400004E5D0AE1540E01014F5D06E1450E0101CA
:10441000505D02E1210EB3D0470E01014C5D12E167
:10442000450E01014D5D0EE1410E01014E5D0AE1B7
:10443000440E01014F5D06E1530E0101505D02E1A2
:104440000E0E9DD0470E01014C5D12E1450E01019B
:104450004D5D0EE1520E01014E5D0AE1410E01017A
:104460004F5D06E1570E0101505D02E1100E87D04D
:10447000470E01014C5D12E1450E01014D5D0EE15B
:10448000560E01014E5D0AE1450E01014F5D06E148
:10449000520E0101505D02E1140E71D0530E010164
:1044A0004C5D12E1450E01014D5D0EE1560E01011C
:1044B0004E5D0AE1450E01014F5D06E1520E01011C
:1044C000505D02E1230E5BD0530E01014C5D12E101
:1044D000450E01014D5D0EE1550E01014E5D0AE1F3
:1044E000500E01014F5D06E14C0E0101505D02E1ED
:1044F000120E45D0530E01014C5D12E1450E010133
:104500004D5D0EE1430E01014E5D0AE14C0E0101CD
:104510004F5D06E14D0E0101505D02E11A0E2FD0F4
:10452000530E01014C5D12E1450E01014D5D0EE19E
:10453000430E01014E5D0AE14C0E01014F5D06E1A3
:10454000540E0101505D02E11F0E19D0470E01010A
:104550004C5D12E1450E01014D5D0EE14D0E010174
:104560004E5D0AE1560E01014F5D06E1540E010158
:10457000505D02E1250E03D05CDE000E00D012007B
:104580000A01A7950A01A7910A01A79384A004D064
:104590008D920A01A78564D00A01B351006E016AA9
:1045A000013404E200508008000E01540EE20A01BA
:1045B000A7810101B051B11102E18D9205D0010135
:1045C000B007000EB15B8D8203D08D820A01A783F4
:1045D0000101B251006E016AD890015004E6800ECC
:1045E000005C000E015802E2020151816E0E0101D1
:1045F000B25D36E2010EE66EB4EC1AF0E5528B8045
:10460000898C8B82020151810201519302015195E3
:10461000F3EC55F0E66ACDEC54F0E55202015D6B27
:104620005E6B02010A0E5D5D000E5E5917E202012B
:104630005171020151730DEC5AF02DEC55F001014E
:10464000D46BD56B0101640ED45D000ED55901E227
:10465000F9D702015D2B000E5E23E3D761EC3DF03C
:1046600012000A01B551006E016A013404E20050E3
:104670008008000E015405E28450040B02E0190E7C
:10468000A5D00A01B651006E016A013404E200505F
:104690008008000E01540DE20A01B751026E036A50
:1046A000033404E202508008000E035402E2220E9A
:1046B0008DD00A01B651006E016A013404E2005047
:1046C0008008000E015409E20A010A01A851010BF9
:1046D00004E10A01A881150E79D00A01B751006ED4
:1046E000016A013404E200508008000E015409E21E
:1046F0000A010A01A851020B04E10A01A883160E5F
:1047000065D00A01B551006E016A013404E200501F
:104710008008000E015409E20A010A01A851040BA5
:1047200004E10A01A885170E51D08450040B09E159
:104730000A010A01A851080B04E10A01A887180E12
:1047400045D00A01B651006E016AD890015004E6C6
:10475000800E005C000E015807E20A010A01A85110
:10476000010B02E00A01A8910A01B751006E016A2B
:10477000D890015004E6800E005C000E015807E25C
:104780000A010A01A851020B02E00A01A8930A01DA
:10479000B551006E016AD890015004E6800E005CAD
:1047A000000E015807E20A010A01A851040B02E0B9
:1047B0000A01A8958450040B07E00A010A01A851D8
:1047C000080B02E00A01A897000E00D012000A01AF
:1047D000AA898D82C280C46AC36A899E0F014899E2
:1047E000928AF00E89140909896E640EE66E9DECBA
:1047F00074F0E552640EE66E9DEC74F0E552640EC2
:10480000E66E9DEC74F0E552640EE66E9DEC74F07D
:10481000E552640EE66E9DEC74F0E552640EE66EB1
:104820009DEC74F0E552C30EC2141009C26EC28230
:10483000C2B2FED7050EE66E9DEC74F0E552040E92
:10484000006E016AC3CF50F0C4CF51F000C055F0E4
:1048500001C056F035EC74F050C0B2F1898EC290B0
:104860000A01AA991200D9CFE6FFE1CFD9FFE6529B
:104870000A01AA890A01A3B38ED0899A928A0F01EC
:104880004899C280C46AC36A899E0A01DC6B100E13
:104890000A01DC5D34E2F00E89140A01DC11896E34
:1048A000050EE66E9DEC74F0E552C30EC2141009BD
:1048B000C26EC282C2B2FED7050EE66E9DEC74F0E7
:1048C000E552C3CF00F0C4CF01F0020E0F0B05E09C
:1048D000D89001320032E806FBE10A01DC51E96EB2
:1048E000EA6AD890E936EA36BB0EE9260A0EEA22D1
:1048F0000050EE260150ED220A01DC2BC8D7898E2C
:10490000C2900A01DB2B080E0A01DB5D43E1DF6A7E
:10491000DF50006E016A100E005C000E015833E299
:104920000A01DB51026E036AEA6ADF34FE0BEA36E3
:10493000E96EBB0EE9260A0EEA22EECF00F0EFCFB9
:1049400001F000C050F001C051F002C055F003C0AA
:1049500056F035EC74F05050E66EDF50EA6AAB0F5B
:10496000E96E0A0EEA22E552E750EF6EEA6ADF349A
:10497000FE0BEA36E96EBB0EE9260A0EEA22EE6A63
:10498000ED6ADF2AC5D70A01DB6B0A01A7A302D0B3
:10499000B4CAB2F10CD0899EF00E89140D09896E4B
:1049A0000F014889929A898A0101100EB66F0A0197
:1049B000AA99E552E552E7CFD9FF1200D9CFE6FF19
:1049C000E1CFD9FFE652DF6A0B011A51DF5C10E23A
:1049D000DF50040DF3CFE9FFF4CFEAFFF50EE9262F
:1049E0000B0EEA22EE6AEE6AEE6AEE6ADF2AECD776
:1049F000E552E552E7CFD9FF1200D9CFE6FFE1CF6C
:104A0000D9FFE6520B0118690C01296B0C012A6BC6
:104A1000DF6A0D0EDF5C10E2DF50040DF3CFE9FF1B
:104A2000F4CFEAFFF50EE9260B0EEA22EE6AEE6AF3
:104A3000EE6AEE6ADF2AEDD70C013F6B406B416BEB
:104A4000426B0C01436B446B456B466B0C013B6B3B
:104A50003C6B3D6B3E6B0C014B6B4C6B4D6B4E6B73
:104A60000C01476B486B496B4A6B0C014F6B506BE9
:104A7000516B526B0C01536B546B556B566B0C01A5
:104A8000576B586B596B5A6B010EE66EB4EC1AF00B
:104A9000E5528B808B82898C0C012E6B0C012F6B65
:104AA000306B0C01C00E336F270E346F090E356F5B
:104AB000366B0C01C00E376F270E386F090E396F39
:104AC0003A6B0B01BD6BBE6BBF6BC06B0C01576BC0
:104AD000586B596B5A6B0C01536B546B556B566B7F
:104AE00068EC09F01FEC58F077EC57F00A01F06B16
:104AF000F16BF26BF36BE552E552E7CFD9FF120091
:104B0000D9CFE6FFE1CFD9FFE652DF6A0B0118519A
:104B100001E01DD1FB0EDBCF43FCFC0EDBCF44FCE0
:104B2000FD0EDBCF45FCFE0EDBCF46FCFB0EDB5063
:104B30000C013F27FC0EDB500C014023FD0EDB5027
:104B40000C014123FE0EDB500C0142233FCC3BFC09
:104B500040CC3CFC41CC3DFC42CC3EFC0C01292B22
:104B60000B011A510C01295D12E20C01292B0C01D9
:104B70002951040DF3CFE9FFF4CFEAFFF50EE92642
:104B80000B0EEA22EE6AEE6AEE6AEE6AE9D70C01D3
:104B90002951040DF3CFE9FFF4CFEAFFF50EE92622
:104BA0000B0EEA2243CCEEFF44CCEEFF45CCEEFFE9
:104BB00046CCEEFF3FCCF5FB40CCF6FB41CCF7FBFF
:104BC00042CCF8FB0A01A5830C012A2B0C013F6B98
:104BD000406B416B426B0C012951040DF3CFE9FF8F
:104BE000F4CFEAFFC10EE9260B0EEA22EE500C01CB
:104BF000435D0C014B6FEE500C0144590C014C6F9E
:104C0000EE500C0145590C014D6FEE500C01465908
:104C10000C014E6FC10EE96E0B0EEA6EEE500C01E8
:104C20003B5D0C01476FEE500C013C590C01486F85
:104C3000EE500C013D590C01496FEE500C013E59EC
:104C40000C014A6F47CC4FFC48CC50FC49CC51FC7E
:104C50004ACC52FCC10EE96E0B0EEA6EEE500C010E
:104C60003B5DEE500C013C59EE500C013D59EE50AD
:104C70000C013E592CE2DF6A0B011A51D880DF5437
:104C800026E3DF50040DF3CFE9FFF4CFEAFFF50E82
:104C9000E9260B0EEA22EECF00F0EECF01F0EECFC8
:104CA00002F0EFCF03F0DF50040DF3CFE9FFF4CFB4
:104CB000EAFFC10EE9260B0EEA2200C0EEFF01C09A
:104CC000EEFF02C0EEFF03C0EEFFDF2AD5D73B0E9A
:104CD000E96E0C0EEA6E0C013351EE5C0C0134519E
:104CE000EE580C013551EE580C013651EE580AE2DF
:104CF0003BCC33FC3CCC34FC3DCC35FC3ECC36FCD0
:104D00002ACC2DFC3B0EE96E0C0EEA6E0C013751DD
:104D1000EE5C0C013851EE580C013951EE580C0183
:104D20003A51EE5811E23BCC37FC3CCC38FC3DCC40
:104D300039FC3ECC3AFC31CC2FFC32CC30FC2ACCB6
:104D40002EFC0C01316B326B0C01296B95D00B01E1
:104D50001A510C01D880295503E2000E0CD3F7D765
:104D6000FB0EDBCF43FCFC0EDBCF44FCFD0EDBCFA8
:104D700045FCFE0EDBCF46FCFB0EDB500C013F2753
:104D8000FC0EDB500C014023FD0EDB500C014123D7
:104D9000FE0EDB500C0142230C01292B0C01295182
:104DA000040DF3CFE9FFF4CFEAFFF50EE9260B0E71
:104DB000EA2243CCEEFF44CCEEFF45CCEEFF46CCDE
:104DC000EEFF0C012951040DF3CFE9FFF4CFEAFF08
:104DD000C10EE9260B0EEA22EE500C01435D0C01D8
:104DE0004B6FEE500C0144590C014C6FEE500C010E
:104DF00045590C014D6FEE500C0146590C014E6F98
:104E00000C014F6B506B516B526B010EDF6E0C013E
:104E10002951D880DF5418E3DF50040DF3CFE9FFA8
:104E2000F4CFEAFFC10EE9260B0EEA22EE500C0188
:104E30004F27EE500C015023EE500C015123EE5041
:104E40000C015223DF2AE3D74F0EE96E0C0EEA6EF7
:104E5000EE500C013F5D0C014F6FEE500C014059BC
:104E60000C01506FEE500C0141590C01516FEE5086
:104E70000C0142590C01526F0B01185101E02BD16A
:104E80000A019151050A01E1B1D0010A6CE0070A5B
:104E900027E0010A14E0030A01E0EBD03BCCBDFBA4
:104EA0003CCCBEFB3DCCBFFB3ECCC0FB47CC57FC53
:104EB00048CC58FC49CC59FC4ACC5AFCDAD043CCFB
:104EC000BDFB44CCBEFB45CCBFFB46CCC0FB4BCCB2
:104ED00057FC4CCC58FC4DCC59FC4ECC5AFCC9D09C
:104EE0004BCC4EF04CCC4FF04DCC50F04ECC51F062
:104EF000EDEC63F04FC004F050C005F051C006F077
:104F000052C007F004C0E6FF05C0E6FF06C0E6FF9A
:104F100007C0E6FF6FEC73F0E552E552E552E5524B
:104F20004EC000F04FC001F050C002F051C003F07D
:104F300000C04FF001C050F002C051F003C052F069
:104F4000E7EC65F04EC0BDFB4FC0BEFB50C0BFFBE1
:104F500051C0C0FB4BCC57FC4CCC58FC4DCC59FC41
:104F60004ECC5AFC86D047CC4EF048CC4FF049CCC2
:104F700050F04ACC51F0EDEC63F04FC004F050C05B
:104F800005F051C006F052C007F004C0E6FF05C0AE
:104F9000E6FF06C0E6FF07C0E6FF6FEC73F0E552E0
:104FA000E552E552E5524EC000F04FC001F050C04E
:104FB00002F051C003F000C04FF001C050F002C039
:104FC00051F003C052F0E7EC65F04EC0BDFB4FC09E
:104FD000BEFB50C0BFFB51C0C0FB47CC57FC48CC08
:104FE00058FC49CC59FC4ACC5AFC43D04FCC4EF02B
:104FF00050CC4FF051CC50F052CC51F0EDEC63F06E
:105000004FC004F050C005F051C006F052C007F088
:1050100004C0E6FF05C0E6FF06C0E6FF07C0E6FFE6
:105020006FEC73F0E552E552E552E5524EC000F0E8
:105030004FC001F050C002F051C003F000C04FF06B
:1050400001C050F002C051F003C052F0E7EC65F02F
:105050004EC0BDFB4FC0BEFB50C0BFFB51C0C0FB2C
:105060004FCC57FC50CC58FC51CC59FC52CC5AFC7C
:1050700000D00C015A35000E5A1909E6D880000EEE
:105080005755000E5855000E5955000E5A5506E357
:105090000C015B950C015B898A828A900C015A3560
:1050A000000E5A1909E6D880000E5755000E5855C3
:1050B000000E5955000E5A5506E20C015B850C0195
:1050C0005B998A928A800C015B8F0C015E6B68ECA5
:1050D00009F01FEC58F00A019051040A01E19ED03A
:1050E000070A59E0010A14E0030A01E0DAD043CCD0
:1050F000BDFB44CCBEFB45CCBFFB46CCC0FB4BCC80
:1051000053FC4CCC54FC4DCC55FC4ECC56FCC9D079
:105110004BCC4EF04CCC4FF04DCC50F04ECC51F02F
:10512000EDEC63F04FC004F050C005F051C006F044
:1051300052C007F004C0E6FF05C0E6FF06C0E6FF68
:1051400007C0E6FF6FEC73F0E552E552E552E55219
:105150004EC000F04FC001F050C002F051C003F04B
:1051600000C04FF001C050F002C051F003C052F037
:10517000E7EC65F04EC0BDFB4FC0BEFB50C0BFFBAF
:1051800051C0C0FB4BCC53FC4CCC54FC4DCC55FC1B
:105190004ECC56FC86D047CC4EF048CC4FF049CC94
:1051A00050F04ACC51F0EDEC63F04FC004F050C029
:1051B00005F051C006F052C007F004C0E6FF05C07C
:1051C000E6FF06C0E6FF07C0E6FF6FEC73F0E552AE
:1051D000E552E552E5524EC000F04FC001F050C01C
:1051E00002F051C003F000C04FF001C050F002C007
:1051F00051F003C052F0E7EC65F04EC0BDFB4FC06C
:10520000BEFB50C0BFFB51C0C0FB47CC53FC48CCD9
:1052100054FC49CC55FC4ACC56FC43D04FCC4EF004
:1052200050CC4FF051CC50F052CC51F0EDEC63F03B
:105230004FC004F050C005F051C006F052C007F056
:1052400004C0E6FF05C0E6FF06C0E6FF07C0E6FFB4
:105250006FEC73F0E552E552E552E5524EC000F0B6
:105260004FC001F050C002F051C003F000C04FF039
:1052700001C050F002C051F003C052F0E7EC65F0FD
:105280004EC0BDFB4FC0BEFB50C0BFFB51C0C0FBFA
:105290004FCC53FC50CC54FC51CC55FC52CC56FC5A
:1052A00000D068EC09F077EC57F00A019A51040A33
:1052B00007E0010A01E008D001010A0EAA6F04D03C
:1052C00001010A0EAA6F00D00A019E51040A07E0EC
:1052D000010A01E008D001010A0EAB6F04D0010100
:1052E0000A0EAB6F00D0010EE66E57CCE6FF58CC2D
:1052F000E6FF59CCE6FF5ACCE6FF53CCE6FF54CC90
:10530000E6FF55CCE6FF56CCE6FF2BEC5AF0006EDC
:10531000090EE15E00500C015635000E561909E6E3
:10532000D880000E5355000E5455000E5555000EF2
:10533000565506E30C015B970C015B8B8A868A94B9
:105340000C015635000E561909E6D880000E53554B
:10535000000E5455000E5555000E565506E20C0130
:105360005B870C015B9B8A968A840C015B8D0C0128
:105370005E6B010E00D0E552E552E7CFD9FF120077
:105380000B0118690B0119690101C56B500EC66F3D
:10539000C30EC76F470EC86F02011F6B0B011A5176
:1053A00002011F5D01E3CAD196CB50F097CB51F0BB
:1053B000D6EC63F04FC010F050C011F051C012F0A5
:1053C00052C013F002011F51E96EEA6AD890E93623
:1053D000EA36240EE9260B0EEA22EECF18F0EFCFC4
:1053E00019F018C050F019C051F0D6EC63F04FC05E
:1053F00014F050C015F051C016F052C017F014C090
:1054000054F015C055F016C056F017C057F010C034
:105410004FF011C050F012C051F013C052F006EC22
:1054200064F04FC00CF050C00DF051C00EF052C0EF
:105430000FF096CB50F097CB51F0D6EC63F04FC005
:105440001EF050C01FF051C020F052C021F00201E8
:105450001F51E96EEA6AD890E936EA36240EE92649
:105460000B0EEA22EECF26F0EFCF27F026C050F049
:1054700027C051F0D6EC63F04FC022F050C023F0AB
:1054800051C024F052C025F022C054F023C055F082
:1054900024C056F025C057F01EC04FF01FC050F07A
:1054A00020C051F021C052F006EC64F04FC01AF059
:1054B00050C01BF051C01CF052C01DF01AC054F077
:1054C0001BC055F01CC056F01DC057F00CC04FF06B
:1054D0000DC050F00EC051F00FC052F0F0EC64F06F
:1054E0004FC008F050C009F051C00AF052C00BF094
:1054F00090CB50F091CB51F0D6EC63F04FC030F030
:1055000050C031F051C032F052C033F002011F518F
:10551000E96EEA6AD890E936EA363C0EE9260B0EC7
:10552000EA22EECF38F0EFCF39F038C050F039C072
:1055300051F0D6EC63F04FC034F050C035F051C09C
:1055400036F052C037F034C054F035C055F036C094
:1055500056F037C057F030C04FF031C050F032C075
:1055600051F033C052F006EC64F04FC02CF050C044
:105570002DF051C02EF052C02FF090CB50F091CBB7
:1055800051F0D6EC63F04FC03EF050C03FF051C038
:1055900040F052C041F002011F51E96EEA6AD89012
:1055A000E936EA363C0EE9260B0EEA22EECF46F04B
:1055B000EFCF47F046C050F047C051F0D6EC63F053
:1055C0004FC042F050C043F051C044F052C045F0CB
:1055D00042C054F043C055F044C056F045C057F0A7
:1055E0003EC04FF03FC050F040C051F041C052F0BB
:1055F00006EC64F04FC03AF050C03BF051C03CF0B4
:1056000052C03DF03AC054F03BC055F03CC056F09B
:105610003DC057F02CC04FF02DC050F02EC051F0BF
:105620002FC052F0F0EC64F04FC028F050C029F0C9
:1056300051C02AF052C02BF028C054F029C055F0B8
:105640002AC056F02BC057F008C04FF009C050F0E8
:105650000AC051F00BC052F007EC64F04FC004F0E8
:1056600050C005F051C006F052C007F004C0E6FF7C
:1056700005C0E6FF06C0E6FF07C0E6FFE2EC6BF000
:10568000E552E552E552E5524EC000F04FC001F040
:1056900050C002F051C003F002011F51040DF3CFBE
:1056A000E9FFF4CFEAFF540EE9260B0EEA2200C010
:1056B000EEFF01C0EEFF02C0EEFF03C0EEFF0201ED
:1056C0001F51040DF3CFE9FFF4CFEAFF540EE92692
:1056D0000B0EEA22EECF00F0EECF01F0EECF02F09B
:1056E000EFCF03F0C5C154F0C6C155F0C7C156F0A5
:1056F000C8C157F000C04FF001C050F002C051F0D7
:1057000003C052F027EC66F0010A15E102011F51B7
:10571000040DF3CFE9FFF4CFEAFF540EE9260B0E98
:10572000EA22EECFC5F1EECFC6F1EECFC7F1EFCF53
:10573000C8F11FC219FB02011F2B30D696CB50F0C7
:1057400097CB51F0D6EC63F04FC00CF050C00DF089
:1057500051C00EF052C00FF00B011951E96EEA6A08
:10576000D890E936EA36240EE9260B0EEA22EECF6F
:1057700014F0EFCF15F014C050F015C051F0D6EC76
:1057800063F04FC010F050C011F051C012F052C081
:1057900013F010C054F011C055F012C056F013C0F1
:1057A00057F00CC04FF00DC050F00EC051F00FC0BC
:1057B00052F006EC64F04FC008F050C009F051C040
:1057C0000AF052C00BF096CB50F097CB51F0D6ECCC
:1057D00063F04FC01AF050C01BF051C01CF052C013
:1057E0001DF00B011951E96EEA6AD890E936EA36E4
:1057F000240EE9260B0EEA22EECF22F0EFCF23F0A3
:1058000022C050F023C051F0D6EC63F04FC01EF020
:1058100050C01FF051C020F052C021F01EC054F003
:105820001FC055F020C056F021C057F01AC04FF0ED
:105830001BC050F01CC051F01DC052F006EC64F0CB
:105840004FC016F050C017F051C018F052C019F0F8
:1058500016C054F017C055F018C056F019C057F0D4
:1058600008C04FF009C050F00AC051F00BC052F010
:10587000F0EC64F04FC004F050C005F051C006F0E9
:1058800052C007F090CB50F091CB51F0D6EC63F0C2
:105890004FC02CF050C02DF051C02EF052C02FF050
:1058A0000B011951E96EEA6AD890E936EA363C0EE6
:1058B000E9260B0EEA22EECF34F0EFCF35F034C0FC
:1058C00050F035C051F0D6EC63F04FC030F050C00E
:1058D00031F051C032F052C033F030C054F031C01A
:1058E00055F032C056F033C057F02CC04FF02DC0E9
:1058F00050F02EC051F02FC052F006EC64F04FC0B3
:1059000028F050C029F051C02AF052C02BF090CBA3
:1059100050F091CB51F0D6EC63F04FC03AF050C04C
:105920003BF051C03CF052C03DF00B011951E96E03
:10593000EA6AD890E936EA363C0EE9260B0EEA22EE
:10594000EECF42F0EFCF43F042C050F043C051F0F1
:10595000D6EC63F04FC03EF050C03FF051C040F075
:1059600052C041F03EC054F03FC055F040C056F028
:1059700041C057F03AC04FF03BC050F03CC051F02E
:105980003DC052F006EC64F04FC036F050C037F026
:1059900051C038F052C039F036C054F037C055F01D
:1059A00038C056F039C057F028C04FF029C050F029
:1059B0002AC051F02BC052F0F0EC64F04FC024F03C
:1059C00050C025F051C026F052C027F024C054F03A
:1059D00025C055F026C056F027C057F004C04FF040
:1059E00005C050F006C051F007C052F007EC64F05B
:1059F0004FC000F050C001F051C002F052C003F09F
:105A000000C0E6FF01C0E6FF02C0E6FF03C0E6FFFC
:105A1000E2EC6BF0E552E552E552E5524EC084FBF4
:105A20004FC085FB50C086FB51C087FBC3C150F0FF
:105A3000C4C151F0D6EC63F04FC000F050C001F08B
:105A400051C002F052C003F000C054F001C055F044
:105A500002C056F003C057F088CB4FF089CB50F00E
:105A60008ACB51F08BCB52F01EEC66F0010A02E1BA
:105A700022EF35F084CB54F085CB55F086CB56F031
:105A800087CB57F088CB4FF089CB50F08ACB51F0C1
:105A90008BCB52F027EC66F0010A02E022EF35F0E2
:105AA0008CCB54F08DCB55F08ECB56F08FCB57F07E
:105AB00088CB4FF089CB50F08ACB51F08BCB52F092
:105AC00027EC66F0010A02E022EF35F08CCB54F0AF
:105AD0008DCB55F08ECB56F08FCB57F084CB4FF05B
:105AE00085CB50F086CB51F087CB52F01EEC66F0A0
:105AF000010A01E1C9D398CB50F099CB51F0D6EC13
:105B000063F04FC00CF050C00DF051C00EF052C009
:105B10000FF096CB50F097CB51F0D6EC63F04FC01E
:105B200010F050C011F051C012F052C013F010C06C
:105B300054F011C055F012C056F013C057F00CC00D
:105B40004FF00DC050F00EC051F00FC052F006ECF7
:105B500064F04FC008F050C009F051C00AF052C0C4
:105B60000BF098CB50F099CB51F0D6EC63F04FC0CE
:105B700018F050C019F051C01AF052C01BF096CB6B
:105B800050F097CB51F0D6EC63F04FC01CF050C0F2
:105B90001DF051C01EF052C01FF01CC054F01DC0BB
:105BA00055F01EC056F01FC057F018C04FF019C076
:105BB00050F01AC051F01BC052F006EC64F04FC018
:105BC00014F050C015F051C016F052C017F014C0B8
:105BD00054F015C055F016C056F017C057F008C065
:105BE0004FF009C050F00AC051F00BC052F0F0EC79
:105BF00064F04FC004F050C005F051C006F052C030
:105C000007F092CB50F093CB51F0D6EC63F04FC03D
:105C100028F050C029F051C02AF052C02BF090CB90
:105C200050F091CB51F0D6EC63F04FC02CF050C047
:105C30002DF051C02EF052C02FF02CC054F02DC0CA
:105C400055F02EC056F02FC057F028C04FF029C095
:105C500050F02AC051F02BC052F006EC64F04FC057
:105C600024F050C025F051C026F052C027F092CB4E
:105C700050F093CB51F0D6EC63F04FC034F050C0ED
:105C800035F051C036F052C037F090CB50F091CB88
:105C900051F0D6EC63F04FC038F050C039F051C02D
:105CA0003AF052C03BF038C054F039C055F03AC019
:105CB00056F03BC057F034C04FF035C050F036C0FE
:105CC00051F037C052F006EC64F04FC030F050C0D5
:105CD00031F051C032F052C033F030C054F031C016
:105CE00055F032C056F033C057F024C04FF025C0F5
:105CF00050F026C051F027C052F0F0EC64F04FC0D5
:105D000020F050C021F051C022F052C023F020C03A
:105D100054F021C055F022C056F023C057F004C003
:105D20004FF005C050F006C051F007C052F007EC2C
:105D300064F04FC000F050C001F051C002F052C0FA
:105D400003F000C0E6FF01C0E6FF02C0E6FF03C0AB
:105D5000E6FFE2EC6BF0E552E552E552E5524EC04B
:105D6000C9F14FC0CAF150C0CBF151C0CCF188CBC2
:105D700054F089CB55F08ACB56F08BCB57F084CBBF
:105D80004FF085CB50F086CB51F087CB52F007EC2B
:105D900064F04FC014F050C015F051C016F052C05E
:105DA00017F0C9C154F0CAC155F0CBC156F0CCC1EF
:105DB00057F014C04FF015C050F016C051F017C086
:105DC00052F006EC64F04FC010F050C011F051C01A
:105DD00012F052C013F088CB54F089CB55F08ACB27
:105DE00056F08BCB57F084CB4FF085CB50F086CB61
:105DF00051F087CB52F006EC64F04FC01CF050C05D
:105E00001DF051C01EF052C01FF0C9C154F0CAC1EC
:105E100055F0CBC156F0CCC157F01CC04FF01DC09F
:105E200050F01EC051F01FC052F007EC64F04FC09C
:105E300018F050C019F051C01AF052C01BF018C031
:105E400054F019C055F01AC056F01BC057F010C0DE
:105E50004FF011C050F012C051F013C052F0F0ECEE
:105E600064F04FC00CF050C00DF051C00EF052C0A5
:105E70000FF0546A556A800E566EBF0E576E84CB73
:105E80004FF085CB50F086CB51F087CB52F0F0EC41
:105E900064F04FC028F050C029F051C02AF052C021
:105EA0002BF088CB54F089CB55F08ACB56F08BCBB6
:105EB00057F028C04FF029C050F02AC051F02BC035
:105EC00052F007EC64F04FC024F050C025F051C0F0
:105ED00026F052C027F0C9C154F0CAC155F0CBC159
:105EE00056F0CCC157F024C04FF025C050F026C06A
:105EF00051F027C052F007EC64F04FC020F050C0C2
:105F000021F051C022F052C023F020C054F021C033
:105F100055F022C056F023C057F00CC04FF00DC012
:105F200050F00EC051F00FC052F0F0EC64F04FC0D2
:105F300008F050C009F051C00AF052C00BF088CBF5
:105F400054F089CB55F08ACB56F08BCB57F084CBED
:105F50004FF085CB50F086CB51F087CB52F007EC59
:105F600064F04FC030F050C031F051C032F052C038
:105F700033F0C9C154F0CAC155F0CBC156F0CCC101
:105F800057F030C04FF031C050F032C051F033C044
:105F900052F007EC64F04FC02CF050C02DF051C00F
:105FA0002EF052C02FF02CC054F02DC055F02EC052
:105FB00056F02FC057F008C04FF009C050F00AC08B
:105FC00051F00BC052F0F0EC64F04FC004F050C040
:105FD00005F051C006F052C007F004C0E6FF05C04E
:105FE000E6FF06C0E6FF07C0E6FFE2EC6BF0E55215
:105FF000E552E552E5524EC000F04FC001F050C0EE
:1060000002F051C003F0546A556A566A400E576E4A
:1060100000C04FF001C050F002C051F003C052F078
:106020009DEC64F04FC0CDF150C0CEF151C0CFF126
:1060300052C0D0F1C9C154F0CAC155F0CBC156F01D
:10604000CCC157F0CDC14FF0CEC150F0CFC151F00F
:10605000D0C152F09DEC64F04FC0CDF150C0CEF1F4
:1060600051C0CFF152C0D0F188CB54F089CB55F05C
:106070008ACB56F08BCB57F088CB4FF089CB50F0C2
:106080008ACB51F08BCB52F0F0EC64F04FC004F0AF
:1060900050C005F051C006F052C007F0CDC154F019
:1060A000CEC155F0CFC156F0D0C157F0CDC14FF0A1
:1060B000CEC150F0CFC151F0D0C152F0F0EC64F03D
:1060C0004FC008F050C009F051C00AF052C00BF0A8
:1060D00008C054F009C055F00AC056F00BC057F084
:1060E00004C04FF005C050F006C051F007C052F098
:1060F00006EC64F04FC000F050C001F051C002F057
:1061000052C003F000C0E6FF01C0E6FF02C0E6FF98
:1061100003C0E6FFE2EC6BF0E552E552E552E552D2
:106120004EC0C5F14FC0C6F150C0C7F151C0C8F153
:10613000CDC154F0CEC155F0CFC156F0D0C157F00B
:1061400088CB4FF089CB50F08ACB51F08BCB52F0FB
:1061500006EC64F04FC004F050C005F051C006F0EA
:1061600052C007F004C0E6FF05C0E6FF06C0E6FF28
:1061700007C0E6FF6FEC73F0E552E552E552E552D9
:106180004EC000F04FC001F050C002F051C003F00B
:106190006F0E546E120E556E830E566E3A0E576E7B
:1061A00000C04FF001C050F002C051F003C052F0E7
:1061B00027EC66F0010A05E10101C56BC66BC76BF0
:1061C000C86B19CB18FBA0CB4EF0A1CB4FF0A2CBE4
:1061D00050F0A3CB51F0EBEC63F04FC000F050C097
:1061E00001F051C002F052C003F0546A556AC80E63
:1061F000566E420E576EC5C14FF0C6C150F0C7C1B2
:1062000051F0C8C152F0F0EC64F04FC008F050C03B
:1062100009F051C00AF052C00BF0C9C154F0CAC114
:1062200055F0CBC156F0CCC157F008C04FF009C0B3
:1062300050F00AC051F00BC052F09DEC64F04FC01A
:1062400004F050C005F051C006F052C007F004C081
:1062500054F005C055F006C056F007C057F000C016
:106260004FF001C050F002C051F003C052F007ECF3
:1062700064F0E7EC65F04EC0B4FB4FC0B5FB50C016
:10628000B6FB51C0B7FBDFD384CB54F085CB55F0C0
:1062900086CB56F087CB57F08CCB4FF08DCB50F0A0
:1062A0008ECB51F08FCB52F027EC66F0010A01E063
:1062B000C9D398CB50F099CB51F0D6EC63F04FC0D6
:1062C0000CF050C00DF051C00EF052C00FF09ACB40
:1062D00050F09BCB51F0D6EC63F04FC010F050C0A3
:1062E00011F051C012F052C013F010C054F011C0A0
:1062F00055F012C056F013C057F00CC04FF00DC04F
:1063000050F00EC051F00FC052F006EC64F04FC0D8
:1063100008F050C009F051C00AF052C00BF098CB01
:1063200050F099CB51F0D6EC63F04FC018F050C04C
:1063300019F051C01AF052C01BF09ACB50F09BCB11
:1063400051F0D6EC63F04FC01CF050C01DF051C0AE
:106350001EF052C01FF01CC054F01DC055F01EC0EE
:1063600056F01FC057F018C04FF019C050F01AC0B7
:1063700051F01BC052F006EC64F04FC014F050C056
:1063800015F051C016F052C017F014C054F015C0EB
:1063900055F016C056F017C057F008C04FF009C0AE
:1063A00050F00AC051F00BC052F0F0EC64F04FC056
:1063B00004F050C005F051C006F052C007F092CB77
:1063C00050F093CB51F0D6EC63F04FC028F050C0A2
:1063D00029F051C02AF052C02BF094CB50F095CB4D
:1063E00051F0D6EC63F04FC02CF050C02DF051C0EE
:1063F0002EF052C02FF02CC054F02DC055F02EC0FE
:1064000056F02FC057F028C04FF029C050F02AC0D6
:1064100051F02BC052F006EC64F04FC024F050C095
:1064200025F051C026F052C027F092CB50F093CB0C
:1064300051F0D6EC63F04FC034F050C035F051C08D
:1064400036F052C037F094CB50F095CB51F0D6ECEB
:1064500063F04FC038F050C039F051C03AF052C02C
:106460003BF038C054F039C055F03AC056F03BC04C
:1064700057F034C04FF035C050F036C051F037C03F
:1064800052F006EC64F04FC030F050C031F051C013
:1064900032F052C033F030C054F031C055F032C049
:1064A00056F033C057F024C04FF025C050F026C03E
:1064B00051F027C052F0F0EC64F04FC020F050C013
:1064C00021F051C022F052C023F020C054F021C06E
:1064D00055F022C056F023C057F004C04FF005C05D
:1064E00050F006C051F007C052F007EC64F04FC006
:1064F00000F050C001F051C002F052C003F000C0E3
:10650000E6FF01C0E6FF02C0E6FF03C0E6FFE2ECE3
:106510006BF0E552E552E552E5524EC0C9F14FC06D
:10652000CAF150C0CBF151C0CCF188CB54F089CB2B
:1065300055F08ACB56F08BCB57F08CCB4FF08DCBF0
:1065400050F08ECB51F08FCB52F007EC64F04FC07F
:1065500014F050C015F051C016F052C017F0C9C168
:1065600054F0CAC155F0CBC156F0CCC157F014C09D
:106570004FF015C050F016C051F017C052F006ECA5
:1065800064F04FC010F050C011F051C012F052C072
:1065900013F088CB54F089CB55F08ACB56F08BCBD7
:1065A00057F08CCB4FF08DCB50F08ECB51F08FCB82
:1065B00052F006EC64F04FC01CF050C01DF051C00A
:1065C0001EF052C01FF0C9C154F0CAC155F0CBC172
:1065D00056F0CCC157F01CC04FF01DC050F01EC08B
:1065E00051F01FC052F007EC64F04FC018F050C0DB
:1065F00019F051C01AF052C01BF018C054F019C065
:1066000055F01AC056F01BC057F010C04FF011C023
:1066100050F012C051F013C052F0F0EC64F04FC0D3
:106620000CF050C00DF051C00EF052C00FF0546A83
:10663000556A800E566EBF0E576E8CCB4FF08DCBC9
:1066400050F08ECB51F08FCB52F0F0EC64F04FC095
:1066500028F050C029F051C02AF052C02BF088CB4E
:1066600054F089CB55F08ACB56F08BCB57F028C02D
:106670004FF029C050F02AC051F02BC052F007EC67
:1066800064F04FC024F050C025F051C026F052C035
:1066900027F0C9C154F0CAC155F0CBC156F0CCC1E6
:1066A00057F024C04FF025C050F026C051F027C04D
:1066B00052F007EC64F04FC020F050C021F051C000
:1066C00022F052C023F020C054F021C055F022C067
:1066D00056F023C057F00CC04FF00DC050F00EC064
:1066E00051F00FC052F0F0EC64F04FC008F050C011
:1066F00009F051C00AF052C00BF088CB54F089CB9E
:1067000055F08ACB56F08BCB57F08CCB4FF08DCB1E
:1067100050F08ECB51F08FCB52F007EC64F04FC0AD
:1067200030F050C031F051C032F052C033F0C9C126
:1067300054F0CAC155F0CBC156F0CCC157F030C0AF
:106740004FF031C050F032C051F033C052F007EC7E
:1067500064F04FC02CF050C02DF051C02EF052C04C
:106760002FF02CC054F02DC055F02EC056F02FC085
:1067700057F008C04FF009C050F00AC051F00BC0EC
:1067800052F0F0EC64F04FC004F050C005F051C07E
:1067900006F052C007F004C0E6FF05C0E6FF06C0E1
:1067A000E6FF07C0E6FFE2EC6BF0E552E552E5528A
:1067B000E5524EC000F04FC001F050C002F051C091
:1067C00003F0546A556A566A400E576E00C04FF087
:1067D00001C050F002C051F003C052F09DEC64F0D3
:1067E0004FC0CDF150C0CEF151C0CFF152C0D0F169
:1067F000C9C154F0CAC155F0CBC156F0CCC157F055
:10680000CDC14FF0CEC150F0CFC151F0D0C152F048
:106810009DEC64F04FC0CDF150C0CEF151C0CFF12E
:1068200052C0D0F188CB54F089CB55F08ACB56F0CA
:106830008BCB57F088CB4FF089CB50F08ACB51F0FF
:106840008BCB52F0F0EC64F04FC004F050C005F078
:1068500051C006F052C007F0CDC154F0CEC155F082
:10686000CFC156F0D0C157F0CDC14FF0CEC150F0DE
:10687000CFC151F0D0C152F0F0EC64F04FC008F03D
:1068800050C009F051C00AF052C00BF008C054F0DB
:1068900009C055F00AC056F00BC057F004C04FF0C5
:1068A00005C050F006C051F007C052F006EC64F08D
:1068B0004FC000F050C001F051C002F052C003F0D0
:1068C00000C0E6FF01C0E6FF02C0E6FF03C0E6FF2E
:1068D000E2EC6BF0E552E552E552E5524EC0C5F1EF
:1068E0004FC0C6F150C0C7F151C0C8F1CDC154F07E
:1068F000CEC155F0CFC156F0D0C157F088CB4FF084
:1069000089CB50F08ACB51F08BCB52F006EC64F07F
:106910004FC004F050C005F051C006F052C007F05F
:1069200004C0E6FF05C0E6FF06C0E6FF07C0E6FFBD
:106930006FEC73F0E552E552E552E5524EC000F0BF
:106940004FC001F050C002F051C003F06F0E546E02
:10695000120E556E830E566E3A0E576E00C04FF0F3
:1069600001C050F002C051F003C052F027EC66F0B5
:10697000010A05E10101C56BC66BC76BC86B19CB7A
:1069800018FBA0CB4EF0A1CB4FF0A2CB50F0A3CB85
:1069900051F0EBEC63F04FC000F050C001F051C07B
:1069A00002F052C003F0546A556AC80E566E420E89
:1069B000576EC5C14FF0C6C150F0C7C151F0C8C134
:1069C00052F0F0EC64F04FC008F050C009F051C034
:1069D0000AF052C00BF0C9C154F0CAC155F0CBC186
:1069E00056F0CCC157F008C04FF009C050F00AC0B3
:1069F00051F00BC052F09DEC64F04FC004F050C059
:106A000005F051C006F052C007F004C054F005C0B4
:106A100055F006C056F007C057F000C04FF001C057
:106A200050F002C051F003C052F006EC64F0E7EC05
:106A300065F04EC0B4FB4FC0B5FB50C0B6FB51C0B3
:106A4000B7FB01D000D01200D9CFE6FFE1CFD9FFCC
:106A5000FE0EDB5001E198D0FE0EDBCFE6FF00EC2E
:106A60005EF0E552FE0EDBCFE6FFDDEC58F0E552BE
:106A7000F5CBBDFBF6CBBEFBF7CBBFFBF8CBC0FB2A
:106A800068EC09F01FEC58F0C10EE96E0B0EEA6ECF
:106A9000EE500B01F55D0C01476FEE500B01F659FE
:106AA0000C01486FEE500B01F7590C01496FEE5085
:106AB0000B01F8590C014A6F47CC4EF048CC4FF00F
:106AC00049CC50F04ACC51F0EDEC63F04FC004F0EB
:106AD00050C005F051C006F052C007F004C0E6FFF8
:106AE00005C0E6FF06C0E6FF07C0E6FF6FEC73F0E7
:106AF000E552E552E552E5524EC000F04FC001F0BC
:106B000050C002F051C003F000C04FF001C050F07F
:106B100002C051F003C052F0E7EC65F04EC0BDFB7F
:106B20004FC0BEFB50C0BFFB51C0C0FB68EC09F0BA
:106B300077EC57F047CC53FC48CC54FC49CC55FC7F
:106B40004ACC56FC47CC57FC48CC58FC49CC59FCA5
:106B50004ACC5AFC010EE66E57CCE6FF58CCE6FF55
:106B600059CCE6FF5ACCE6FF53CCE6FF54CCE6FF07
:106B700055CCE6FF56CCE6FF2BEC5AF0006E090E22
:106B8000E15E00502DEC55F0E552E7CFD9FF120041
:106B9000D9CFE6FFE1CFD9FFFE0EDBCFE6FF16EC43
:106BA00059F0E552FE0EDB50040DF3CFE9FFF4CFB0
:106BB000EAFFF50EE9260B0EEA22EECF00F0EECF4B
:106BC00001F0EECF02F0EFCF03F0FE0EDB50040D2C
:106BD000F3CFE9FFF4CFEAFFC10EE9260B0EEA225C
:106BE000EE50005C0C014B6FEE5001580C014C6FE5
:106BF000EE5002580C014D6FEE5003580C014E6FD1
:106C0000C10EE96E0B0EEA6EEE500B01F55D0C0144
:106C1000476FEE500B01F6590C01486FEE500B0117
:106C2000F7590C01496FEE500B01F8590C014A6FEE
:106C3000FD0EDB0413E1FE0EDB50040DF3CFE9FF84
:106C4000F4CFEAFFF50EE9260B0EEA22EECFBDFBEC
:106C5000EECFBEFBEECFBFFBEFCFC0FBFD0EDB5098
:106C600008E14BCCBDFB4CCCBEFB4DCCBFFB4ECCAE
:106C7000C0FB68EC09F077EC57F04BCC53FC4CCCE4
:106C800054FC4DCC55FC4ECC56FC47CC57FC48CC64
:106C900058FC49CC59FC4ACC5AFC010EE66E57CC44
:106CA000E6FF58CCE6FF59CCE6FF5ACCE6FF53CCC2
:106CB000E6FF54CCE6FF55CCE6FF56CCE6FF2BECC6
:106CC0005AF0006E090EE15E00502DEC55F0E552D1
:106CD000E7CFD9FF12003BEC5FF00C012D513EE0F5
:106CE0002DCCE6FFDDEC58F0E552C1CBBDFBC2CBAD
:106CF000BEFBC3CBBFFBC4CBC0FB68EC09F01FECF1
:106D000058F00B01BD6BBE6BBF6BC06B68EC09F03C
:106D100077EC57F00C01536B546B556B566B0C01B1
:106D2000576B586B596B5A6B010EE66E57CCE6FFEA
:106D300058CCE6FF59CCE6FF5ACCE6FF53CCE6FF31
:106D400054CCE6FF55CCE6FF56CCE6FF2BEC5AF0D0
:106D5000006E090EE15E00502DEC55F012002DCCB6
:106D6000E6FFDDEC58F0E552C1CBBDFBC2CBBEFB6C
:106D7000C3CBBFFBC4CBC0FB68EC09F01FEC58F0E1
:106D80000B01BD6BBE6BBF6BC06B68EC09F077ECA1
:106D900057F00C01536B546B556B566B0C01576BD2
:106DA000586B596B5A6B010EE66E57CCE6FF58CC08
:106DB000E6FF59CCE6FF5ACCE6FF53CCE6FF54CCB5
:106DC000E6FF55CCE6FF56CCE6FF2BEC5AF0006E02
:106DD000090EE15E00502DEC55F012000A019251AF
:106DE000020A1DE0030A01E052D0E7CA00F0E8CA37
:106DF00001F0030ED89000360136E806FBE100C032
:106E000050F001C051F093CA55F094CA56F035ECD9
:106E100074F05050E66EC5EC59F0E55238D093CA84
:106E200002F094CA03F0640E556E566A02C050F028
:106E300003C051F035EC74F050C002F051C003F0C3
:106E40000CCB00F00DCB01F0640E556E566A00C0FD
:106E500050F001C051F035EC74F050C000F051C05A
:106E600001F0030ED89000360136E806FBE100C0C1
:106E700050F001C051F002C055F003C056F035EC9F
:106E800074F05050E66EC5EC59F0E55200D0120097
:106E90000A019551030A49E0010A0CE0030A01E0E6
:106EA0004AD0E7CAE6FFE8CAE6FF4FEC59F0E552E0
:106EB000E55241D00B010F0ED8800C55270E0D5511
:106EC0001AE20CCB00F00DCB01F0640E556E566A41
:106ED00000C050F001C051F035EC74F050C000F02B
:106EE00051C001F000C0E6FF01C0E6FF8AEC59F096
:106EF000E552E55219D00CCB00F00DCB01F00A0E93
:106F0000556E566A00C050F001C051F035EC74F077
:106F100050C000F051C001F000C0E6FF01C0E6FF24
:106F20008AEC59F0E552E55206D02ACCE6FFDDECBA
:106F300058F0E55200D012000A01A6BB4BD00B015D
:106F4000BD6BBE6BBF6BC06B68EC09F01FEC58F0FB
:106F50000C01476B486B496B4A6B0B01BD6BBE6BF9
:106F6000BF6BC06B68EC09F077EC57F047CC53FC73
:106F700048CC54FC49CC55FC4ACC56FC47CC57FC79
:106F800048CC58FC49CC59FC4ACC5AFC010EE66E60
:106F900057CCE6FF58CCE6FF59CCE6FF5ACCE6FFCB
:106FA00053CCE6FF54CCE6FF55CCE6FF56CCE6FFCB
:106FB0002BEC5AF0006E090EE15E0050E66ADDEC43
:106FC00058F0E5520A01A3B305D0010EE66EB4EC09
:106FD0001AF0E55212000C012D5101E1FED00A0118
:106FE000A3B305D0010EE66EB4EC1AF0E552010130
:106FF0009F514DE10101010E9F6F2DCCE6FFDDECAD
:1070000058F0E552C1CBBDFBC2CBBEFBC3CBBFFB2F
:10701000C4CBC0FB68EC09F01FEC58F00C01476BC7
:10702000486B496B4A6B0B01BD6BBE6BBF6BC06B92
:1070300068EC09F077EC57F047CC53FC48CC54FC93
:1070400049CC55FC4ACC56FC47CC57FC48CC58FCA4
:1070500049CC59FC4ACC5AFC010EE66E57CCE6FFEF
:1070600058CCE6FF59CCE6FF5ACCE6FF53CCE6FFFE
:1070700054CCE6FF55CCE6FF56CCE6FF2BEC5AF09D
:10708000006E090EE15E00502DEC55F0A6D0010116
:107090009F6B0C012E5101E1A0D00A018D5109E036
:1070A0002FCCE6FF30CCE6FF8AEC59F0E552E552F2
:1070B00008D02FCCE6FF30CCE6FF4FEC59F0E5527C
:1070C000E55237CCBDFB38CCBEFB39CCBFFB3ACC4C
:1070D000C0FB68EC09F01FEC58F0C10EE96E0B0E16
:1070E000EA6EEE500C01375D0C01476FEE500C015B
:1070F00038590C01486FEE500C0139590C01496F99
:10710000EE500C013A590C014A6F47CC4EF048CC76
:107110004FF049CC50F04ACC51F0EDEC63F04FC049
:1071200004F050C005F051C006F052C007F004C092
:10713000E6FF05C0E6FF06C0E6FF07C0E6FF6FEC0E
:1071400073F0E552E552E552E5524EC000F04FC0F3
:1071500001F050C002F051C003F000C04FF001C078
:1071600050F002C051F003C052F0E7EC65F04EC0A1
:10717000BDFB4FC0BEFB50C0BFFB51C0C0FB68ECA5
:1071800009F077EC57F047CC53FC48CC54FC49CC81
:1071900055FC4ACC56FC47CC57FC48CC58FC49CC53
:1071A00059FC4ACC5AFC010EE66E57CCE6FF58CC8F
:1071B000E6FF59CCE6FF5ACCE6FF53CCE6FF54CCB1
:1071C000E6FF55CCE6FF56CCE6FF2BEC5AF0006EFE
:1071D000090EE15E00502DEC55F01200D9CFE6FF0C
:1071E000E1CFD9FFE652DF6A0A01DB6B0A01A69103
:1071F0000A01A6930A01A6950A01A69B0A01A39774
:107200000A01A3910A01A3930A01DE910A01DE9308
:107210000A01E76BE86B0A01E96BEA6B0A01EB6BA9
:10722000EC6B0A01DF6BE06BE16BE26B0A01E36B75
:10723000E46BE56BE66B0201C96B02015F6B606B8F
:107240000A01A39D0A01A385E66A020EE66EE66ABC
:10725000000EE66E060EE66E29EC72F0006E050E6C
:10726000E15E0050E66A020EE66EE66A000EE66E29
:10727000080EE66E29EC72F0006E050EE15E00501D
:107280000101B46B0101BF6BC06BC16BC26B01012B
:10729000D46BD56B0101056B066B076B086B0201A4
:1072A00051910201519302015195010EE66EB4EC29
:1072B0001AF0E552FFEC16F00A01CD69CE6B0A0117
:1072C000B4690A01CB6BCC6B0A01B36B00D0E552F9
:1072D000E552E7CFD9FF1200D9CFE6FFE1CFD9FFC2
:1072E000E6520A01A3A19FD088CB8CFB89CB8DFBF2
:1072F0008ACB8EFB8BCB8FFB92CB94FB93CB95FBF6
:1073000098CB9AFB99CB9BFBA0CBA4FBA1CBA5FB75
:10731000A2CBA6FBA3CBA7FB84CB88FB85CB89FBA9
:1073200086CB8AFB87CB8BFB90CB92FB91CB93FBDD
:1073300096CB98FB97CB99FB9CCBA0FB9DCBA1FB5D
:107340009ECBA2FB9FCBA3FB27EC0CF01C0EE96E9F
:107350000B0EEA6EEE500A01DF5D006EEE500A0180
:10736000E059016EEE500A01E159026EEE500A0139
:10737000E259036E00C090FB01C091FB200EE96E44
:107380000B0EEA6EEE500A01E35D006EEE500A014C
:10739000E459016EEE500A01E559026EEE500A0101
:1073A000E659036E00C096FB01C097FBBFC19CFB72
:1073B000C0C19DFBC1C19EFBC2C19FFB640E536E49
:1073C000546A556A566A9CCB4EF09DCB4FF09ECBCB
:1073D00050F09FCB51F037EC73F04AC09CFB4BC090
:1073E0009DFB4CC09EFB4DC09FFB02011E6B02012A
:1073F0001E8B0A01A3910A0E0C015C5D05E10C01D4
:107400005C6B0C015B8102D00C015C2B050E0C0146
:107410005D5D05E10C015D6B0C015B8302D00C012D
:107420005D2B020E5FD10A01DDA11DD00A01DD91A5
:1074300033EC24F00101B6510FE1C0EC22F031EC45
:1074400023F0DF6EDF5007E00101056B066B076B71
:10745000086BDF5047D107D00A01A8970101B60792
:107460008D820A01A7838450010B20E00A010A01E2
:10747000A351400B1BE10A01A38D0A018AA114D07C
:10748000FC0ED3140009D36E0A0EE66E1EEC74F0E7
:10749000E5520A018A917990976A799E799C79825E
:1074A000799A7988A1927980030E1CD10A010A0188
:1074B000A351400B13E08450010B10E1320EE66E35
:1074C0001EEC74F0E55284B004D00A01A39D090EAD
:1074D00009D10101056B066B076B086B8450010B2A
:1074E00058E0200E0E01005D54E1020E0201585DCD
:1074F00050E1080EE66E000EE66E080EE66EC9EC70
:1075000067F0E552E552E55200093EE00401DF5123
:10751000006E016A005001019D27015001019E2368
:1075200001019F6B01019D5101019F5D000E010151
:107530009E551BE201019F51EA6A000FE96E080E99
:10754000EA22EF50E66E4B0E01019B25E96E010E1B
:1075500001019C21EA6EE552E750EF6E01019B2B81
:10756000000E9C2301019F2BDDD70101070E9D5DBD
:10757000000E9E5909E301019D6B9E6B01019B6BFF
:107580009C6B30EC21F0AED00101056B066B076BF4
:10759000086B0A01AAAB0DD002011E6B02011E8905
:1075A0000A01AA9B0101056B066B076B086B0F0EA6
:1075B00099D00A01A3A504D00A01A395010E92D087
:1075C0000A018AB10CD00101C20ED45D010ED55959
:1075D00005E30101D46BD56B240E84D00BD00101DF
:1075E000260ED45D070ED55905E30101D46BD56B8A
:1075F000240E78D0140E0101D25D04E30101D26B98
:107600001D0E70D03C0E0101D35D04E30101D36B6C
:107610001E0E68D0050E0101A75D04E30101A76BF2
:107620000C0E60D00C015BA104D00C015B911C0E10
:1076300059D00C015BA304D00C015B931B0E52D0FC
:10764000DA0E0101055D420E0659010E0759000EC2
:10765000085901E336DAFF0E0201CA5DEF0ECB597D
:107660001F0ECC59000ECD5902E30D0E3BD0010187
:10767000B40508E0020E0101B45D04E0030E01014F
:10768000B45D0EE10A010A01DE51010B09E00A01B5
:10769000960ED880E755000EE85502E20D0E22D076
:1076A00001019C0E095D6B0E0A590BE30A010A01E8
:1076B000A751010B06E0E7EC23F08D920101096B65
:1076C0000A6B81A00DD00A01AA8F02011E6B0A016C
:1076D000AAAF02D002011E870A01AA9F110E02D092
:1076E000000E00D0E552E552E7CFD9FF12000A01A3
:1076F000DE810A01A6810A01A3870B010A6B0B6BCD
:107700000B01086B096B0B01006B016B026B036BC8
:107710000B01046B056B066B076B0B010C6B0D6BA0
:107720000A01E76BE86B0A01E96BEA6B0A01A685BF
:1077300012004B0E0A01045D63E1300E0A01055D83
:107740005FE1300E0A01065D5BE1310E0A01075D63
:1077500057E1330E0A01095D19E1310E0A010A5D94
:1077600015E1340E0A010B5D11E1330E0A010D5DC6
:107770000DE1330E0A010F5D09E1360E0A01105DBD
:1077800005E10A01A9850A01A9977DD0320E0A01F7
:10779000095D19E1320E0A010A5D15E1300E0A0198
:1077A0000B5D11E1330E0A010D5D0DE1330E0A018F
:1077B0000F5D09E1300E0A01105D05E10A01A983A0
:1077C0000A01A99760D0310E0A01095D19E1360E50
:1077D0000A010A5D15E1310E0A010B5D11E1330E5C
:1077E0000A010D5D0DE1330E0A010F5D09E1360E50
:1077F0000A01105D05E10A01A9890A01A99743D090
:107800004B0E0A01045D2EE1300E0A01055D2AE1EE
:10781000310E0A01065D26E1300E0A01075D22E104
:10782000300E0A01095D0DE1300E0A010A5D09E121
:10783000310E0A010B5D05E10A01A98D0A01A99724
:1078400022D0300E0A01095D0DE1300E0A010A5DF9
:1078500009E1320E0A010B5D05E10A01A98F0A0157
:10786000A99711D0520E0A01035D0DE14D0E0A01D8
:10787000045D09E1430E0A01055D05E10A01A381EA
:107880000A01A99700D01200D9CFE6FFE1CFD9FFB6
:10789000040EE126DE6ADE6ADE6ADD6ADD52DD5252
:1078A0000A01A9970101D46BD56B0A010A01A951FC
:1078B000080B07E10101280ED45D000ED55901E245
:1078C000F4D70A01A9A702D0010E0AD00101280E9F
:1078D000D45D000ED55902E3020E02D0000E00D096
:1078E000006E040EE15C02E2E16AE552E16E0050D6
:1078F000E552E7CFD9FF12000A01A9970A01A99919
:1079000008EC0CF00A01A9970A01A9A7FDD70A0EF5
:10791000E66E1EEC74F0E552300EE66EE00EE66E9A
:1079200021EC49F0E552E5520101D46BD56B010120
:10793000140ED45D000ED55901E2F9D70A01A997BA
:107940000101D46BD56B0101140ED45D000ED55925
:1079500001E2F9D70101010EDD6F0A01A9B7D2D703
:107960001200D9CFE6FFE1CFD9FF020EE1260A01CE
:10797000A3910A01A99D0A01A99FD4EC49F0010134
:10798000D46BD56BE50EE66EDF0EE66E21EC49F0AA
:10799000E552E5520101020EDD6F0A01A9B7C9DE09
:1079A0000101140ED45D000ED559ECE3E50EE66E30
:1079B000DF0EE66E21EC49F0E552E552E50EE66E8B
:1079C000DF0EE66E21EC49F0E552E552E50EE66E7B
:1079D000DF0EE66E21EC49F0E552E552FA0EE66E56
:1079E0001EEC74F0E552E50EE66EDF0EE66E21EC5D
:1079F00049F0E552E55248DF02080EE0E50EE66E7A
:107A0000DF0EE66E21EC49F0E552E5520A0EE66E15
:107A10001EEC74F0E552EFD7EEEC49F0020EE15C9B
:107A200002E2E16AE552E16EE552E7CFD9FF1200CA
:107A30000A018AB117D00A01A98B0A01A9995CDF52
:107A40000A01A99BD380D3820A018A817990976A1F
:107A5000799E798C7982799A7998A19279800101BD
:107A6000D46BD56B12000A018AA120D0FC0ED3146E
:107A70000009D36E0A0EE66E1EEC74F0E5520A01A0
:107A80008A917990976A799E799C7982799A798896
:107A9000A19279800A01A3910A01A98B08EC0CF04C
:107AA00060DF0A01A99B0101D46BD56B12000A01AA
:107AB000A7A306D00A018AB102D0BADF01D0D3DF72
:107AC0001200010EE66EB4EC1AF0E5520A01A7A30B
:107AD0001DD08B92899C8B90F8EC0AF0F3EC55F05A
:107AE0002DEC55F08B82898C8B808D9284B4FED7DF
:107AF0000101A86B100E0101A85D08E2C80EE66E38
:107B00001EEC74F0E5520101A82BF4D70A01A7A1DD
:107B100050D0010EE66EB4EC1AF0E5528B82898CDF
:107B20008B908D92F8EC0AF0F3EC55F02DEC55F0BB
:107B30000101A86B140E0101A85D0DE20101D46BD7
:107B4000D56B0101140ED45D000ED55901E2F9D7B1
:107B50000101A82BEFD784B40BD00101D46BD56BF6
:107B60000101050ED45D000ED55901E2F9D7F3D716
:107B700084A40BD00101D46BD56B0101030ED45D3D
:107B8000000ED55901E2F9D7F3D70101A86B050E14
:107B90000101A85D0DE20101D46BD56B0101050E59
:107BA000D45D000ED55901E2F9D70101A82BEFD71A
:107BB000FF0012000B01BA6BBB6B0B01B86BB96B0A
:107BC0000B01BC6B0B01BD6BBE6BBF6BC06BE66A80
:107BD000DDEC58F0E55277EC57F01FEC58F0E66A10
:107BE000C5EC59F0E5520DEC5AF0E66A010EE66E6E
:107BF000010EE66E2BEC5AF0E552E552E5528B820F
:107C0000898C8B808A808A828A848A862DEC55F0C2
:107C100012000201CA6BCB6BCC6BCD6B62EC5BF0DC
:107C200005C6D7F106C6D8F108C6DAF109C6DBF1F8
:107C30004B0E0101DA5D07E1430E0101DB5D03E15B
:107C40000101010EB46F4B0E0101DA5D07E1470E31
:107C50000101DB5D03E10101020EB46F4B0E010176
:107C6000DA5D07E1520E0101DB5D03E10101030E64
:107C7000B46F410E0101DA5D07E1430E0101DB5DE6
:107C800003E10101040EB46F410E0101DA5D07E169
:107C9000470E0101DB5D03E10101050EB46F410EEA
:107CA0000101DA5D07E1520E0101DB5D03E1010133
:107CB000060EB46F410E0101DA5D07E1530E0101BA
:107CC000DB5D03E10101070EB46F12000E01F29FAC
:107CD000550EA76EAA0EA76EFF91050EDA6F090E5C
:107CE000DB6F0A0EDC6F170EFB6F160EFC6F0D0EAE
:107CF000ED6F130EF66F550EA76EAA0EA76EFF81DD
:107D0000E1EC48F0656A0F01366B0E01006BEEEC9A
:107D100038F0A5EC0BF08D820A01A783800EE66E89
:107D2000080EE66E05EC74F0E552E552C868FEEC0C
:107D300054F0800EE66E080EE66E05EC74F0E55227
:107D4000E552C868FEEC54F0800EE66E080EE66E52
:107D500005EC74F0E552E552C868FEEC54F0800E74
:107D6000E66E080EE66E05EC74F0E552E552C86862
:107D7000FEEC54F0800EE66E080EE66E05EC74F034
:107D8000E552E552C868FEEC54F014DFE66AE66A94
:107D9000E66AC6EC73F0E552E552E552BBEC63F0DF
:107DA0000101100EB66F0C0160910C0160930C0183
:107DB00060950201586B0101B06B020EB16F84B087
:107DC00031D00101DD6B200E0101DD5D05E233ECF8
:107DD00024F00101DD2BF7D731EC23F00101DD6F39
:107DE000150E0101DD5D08E0160E0101DD5D04E008
:107DF000170E0101DD5D0BE10C0160910C01608348
:107E00000C0160950201040E586F0101DD6B0A013F
:107E1000A98B0A01A9950A01A993FCEC49F00A0172
:107E2000A99B01D08D920201CA6B100ECB6FCC6B57
:107E3000CD6B62EC5BF0240E0601005D19E1530E80
:107E40000601015D15E1450E0601025D11E1550EC9
:107E50000601035D0DE1500E0601045D09E14C0EC3
:107E60000601055D05E1B1EC13F0F29E0EEF00F0A6
:107E7000D0DEB1EC13F00A018A910101400EB66F19
:107E80000A01A385F8EC0AF095DE8C848C86020149
:107E90005851030A02E191EF48F0010A02E1D6EFDE
:107EA00043F0050A02E185EF43F0060A01E1CAD278
:107EB000010A01E14FD2060A01E17BD1030A01E187
:107EC000B9D0010A02E0C8EF48F06CEC39F0190AA9
:107ED00001E1ACD01A0A01E1A3D01D0A01E18ED064
:107EE0003A0A01E18AD03C0A01E17CD00F0A76E02F
:107EF000010A22E0030A16E0170A04E0020A01E080
:107F000097D096D0090E0101DD5D0BE18B708B726D
:107F1000897C8A708A728A748A760A01A3910A011E
:107F2000A58386D00101DD6BDDC1E6FF0FEC56F0C5
:107F3000E5522DEC55F07CD0DDC1E6FF0FEC56F09C
:107F4000E5522DEC55F08B808B82898C8A808A8259
:107F50008A848A860101DD5101E18B900101DD05F2
:107F600001E18B92020E0101DD5D01E1899C030EAE
:107F70000101DD5D01E18A90040E0101DD5D01E199
:107F80008A92050E0101DD5D01E18A94060E010170
:107F9000DD5D01E18A96070E0101DD5D09E18B805F
:107FA0008B82898C8A808A828A848A868C948C8649
:107FB000080E0101DD5D09E18B908B92899C8A900E
:107FC0008A928A948A968C848C960101DD2B110EFC
:107FD0000101DD5D02E10101DD6B2AD00101090E25
:107FE000DD6F26D00101080EDD6FDDC1E6FF0FEC6D
:107FF00056F0E5522DEC55F01BD01AD0090E0101B8
:10800000DD5D0DE18B708B72897C8A708A728A7457
:108010008A760A01A3910A01A583F8EC0AF008D038
:108020000201020E586F0A01A38502D04ADD00D07A
:10803000C8EF48F06CEC39F0240A01E1B6D0260A0A
:1080400001E1ABD0200A01E1A3D0210A01E198D0DF
:108050001B0A01E18FD00F0A01E185D0010A76E009
:10806000030A68E0140A4CE01C0A08E0040A04E071
:10807000190A01E09CD09BD024DD99D00C012D5130
:108080000C012A5D38E101019F511BE10101010E44
:108090009F6FE66A57CCE6FF58CCE6FF59CCE6FF67
:1080A0005ACCE6FF53CCE6FF54CCE6FF55CCE6FFB6
:1080B00056CCE6FF2BEC5AF0006E090EE15E005044
:1080C0001AD001019F6B010EE66E57CCE6FF58CC2B
:1080D000E6FF59CCE6FF5ACCE6FF53CCE6FF54CC82
:1080E000E6FF55CCE6FF56CCE6FF2BEC5AF0006ECF
:1080F000090EE15E00500DEC5AF02DEC55F057D012
:1081000097DC7FEC5DF00C012B6F1ACB2CFC6BEC39
:1081100036F001019F6B2DCC2AFCE66ACDEC54F0C1
:10812000E552010EE66EB4EC1AF0E5528B82898CB2
:108130008B803DD00C012A51010802E20C012A0774
:108140002ACCE6FF24EC35F0E55231D00C012B515E
:108150000C012A5D02E20C012A2B2ACCE6FF24EC5A
:1081600035F0E55224D06BEC36F001019F6B2DCC3D
:108170002AFC1DD00201060E586F0A01A38517D0F4
:108180000BEC1BF00201020E586F0A01A3850FD001
:108190000201586B0A01A3850AD00A01A4B304D0D6
:1081A0000201586B0A01A38502D081DC00D0C8EF20
:1081B00048F06CEC39F0240A01E1C7D0260A01E14D
:1081C000BCD0200A01E1B2D0210A01E1A7D01B0AEC
:1081D00001E199D00F0A01E17DD0010A60E0030AB4
:1081E00045E0140A25E01F0A08E0070A04E0190A1E
:1081F00001E0AED0ADD065DCABD001019D519E1148
:108200000AE1010E01019D6F9E6B2ACCE6FFDDECB9
:1082100058F0E55208D001019D6B9E6B29CCE6FF1A
:1082200016EC59F0E5520DEC5AF02DEC55F090D0CB
:1082300018EC3DF001019F6B01019D6B9E6B0C01E1
:10824000010E296F01019F5109E1010EE66E29CC53
:10825000E6FFC8EC35F0E552E55207D0E66A29CCD6
:10826000E6FFC8EC35F0E552E55272D00C01290565
:1082700002E00C01290701019F5109E1010EE66EA0
:1082800029CCE6FFC8EC35F0E552E55207D0E66AA6
:1082900029CCE6FFC8EC35F0E552E55259D00C0187
:1082A0002C510C01295D02E20C01292B01019F5187
:1082B00009E1010EE66E29CCE6FFC8EC35F0E55287
:1082C000E55207D0E66A29CCE6FFC8EC35F0E55266
:1082D000E5523ED001019F510BE10101010E9F6F5C
:1082E000E66A29CCE6FFC8EC35F0E552E5520AD043
:1082F00001019F6B010EE66E29CCE6FFC8EC35F05C
:10830000E552E55225D00201050E586F2ACCE6FF52
:1083100024EC35F0E55201019F6B1AD00BEC1BF0F9
:108320000201020E586F0A01A38512D0F8EC0AF080
:108330000201586B0A01A3850BD00A01A4B304D033
:108340000201586B0A01A38503D057EC3DF000D021
:10835000C8EF48F06CEC39F00D0A67E0150A62E0EE
:108360000F0A5AE0140A50E0010A3DE00E0A25E027
:108370000D0A09E0180A04E0190A01E061D060D092
:1083800061EC3DF05DD033EC3DF08B808B82898CCD
:108390008C848C860101080E036F070E046F0A019E
:1083A000A3970A01A6950A01A899DAEC3DF0010EFF
:1083B000E66ECDEC54F0E55243D00A010A01A65115
:1083C000010B09E00A010A01A351080B04E08B80AC
:1083D0008B72898C03D08B808B82897C0DEC5AF058
:1083E0002DEC55F02DD018EC1FF001080CE1020126
:1083F000010E586F0A01A3858B908B82898C0A012C
:10840000A8870A01A39B1CD00BEC1BF00201020EF3
:10841000586F0A01A38514D00201050E586F0A0196
:10842000A3850ED00A01A8890BD00101010ED66FD9
:108430000201030E586F0A01A3858B928B9000D026
:10844000C8EF48F06CEC39F00D0A01E151D1180A7F
:1084500001E14DD1020A01E140D1140A01E133D119
:10846000010A01E1A8D00E0A5DE01D0A3EE01E0AE5
:1084700028E0170A23E0190A09E0180A04E0190A9B
:1084800001E041D140D161EC3DF03DD133EC3DF014
:108490008B9086EC1DF00A01A69B0B011A5102E09D
:1084A0006AEC1DF08B808B82898CDAEC3DF0E66AF9
:1084B000CDEC54F0E5522DEC55F025D10A01A38BFB
:1084C00022D199EC17F00A010A01A551010B0CE029
:1084D0000A010A01A651020B07E03EEC1BF00A015B
:1084E000A5A302D05CEC1CF00ED10A010A01A55133
:1084F000010B17E00A010A01A651020B12E00C0160
:1085000060B18B901E0EE66E6FEC74F0E5523EEC9F
:108510001BF00A01A5A302D05CEC1CF00C0160B1B9
:108520008B80F1D00DEC5AF00C0160B1ECD00A0157
:108530000A01A351020B06E10A010A01A651200B10
:1085400001E18B700A010A01A451010B12E00A013A
:108550000A01A651200B0DE00BEC1BF037EC1BF0D1
:1085600001019F6BEBEC37F00201070E586F0A0117
:10857000A3850A010A01A451020B07E00A010A01BE
:10858000A651200B02E0EBEC37F00A010A01A451DE
:10859000020B07E10A010A01A651200B02E19CEC43
:1085A00037F00A01A4A306D0EEEC36F048EC37F021
:1085B0002DEC55F0A8D00A01A6A323D00A01A5A14D
:1085C00007D03EEC1BF00A01A5A302D05CEC1CF026
:1085D000DDEC17F00A010A01A351020B12E10A01B6
:1085E0000A01A651200B0DE00C0160B10AD04DEC40
:1085F00019F09AEC19F027EC1AF0E66AB4EC1AF0CC
:10860000E5520B011A5155E00101D151000803E276
:108610000101D1074ED0C0EC29F0FF0E0B01185D0F
:1086200048E001010A0ED16F0A01A6BB10D00B0170
:1086300018510CE10A01A68BFDEC24F0B4CBA8FB89
:10864000B5CBA9FBB6CBAAFBB7CBABFB32D0A80E00
:10865000E96E0B0EEA6EEE500B01B45D0B01AC6FD0
:10866000EE500B01B5590B01AD6FEE500B01B65931
:108670000B01AE6FEE500B01B7590B01AF6FB4CBCE
:10868000A8FBB5CBA9FBB6CBAAFBB7CBABFBACCB5E
:10869000E6FFADCBE6FFAECBE6FFAFCBE6FF80EC6F
:1086A00025F0E552E552E552E552000902E10201EA
:1086B00051830A01A4B306D0EEEC36F048EC37F053
:1086C0002DEC55F020D00BEC1BF037EC1BF0020129
:1086D000020E586F0A01A38516D00201050E586FCD
:1086E0000BEC1BF037EC1BF00A01A3850CD00BD070
:1086F0000201030E586F0101010ED66F0A01A38516
:108700000BEC1BF000D0C8EF48F06CEC39F0030A1A
:108710003DE0210A30E0350A28E0330A23E0260A4A
:1087200013E0030A09E0180A04E0190A01E03CD04A
:108730003BD061EC3DF038D0010EE66ECDEC54F04C
:10874000E55218EC3DF030D00A01A4B30AD0020182
:1087500051910DEC5AF02DEC55F00201586B0A01C5
:10876000A38522D057EC3DF01FD00201050E586FB3
:108770000A01A38519D0020151910DEC5AF02DEC9C
:1087800055F00201586B0A01A3850ED00BEC1BF0CB
:1087900037EC1BF0E66ACDEC54F0E5520201020E14
:1087A000586F0A01A38500D0C8EF48F06CEC39F08F
:1087B000010A02E14AEF48F00F0A01E1B2D3090AC7
:1087C00001E18BD3010A01E180D3150A01E122D333
:1087D0000C0A01E1E0D2050A01E166D2100A01E1CA
:1087E0000ED22A0A01E1B1D1010A01E171D12A0AAE
:1087F00001E10AD1030A01E1CAD01C0A66E0370A86
:1088000044E0310A31E0170A27E0010A12E00D0ABC
:1088100009E0090A02E090EF48F08B9035EC4BF04C
:1088200090EF48F08B828B80F8EC0AF0FF0090EF1D
:1088300048F019EC21F08B920401E05108E1020E9E
:10884000E66EE80EE66E93EC68F0E552E552CBEC8E
:1088500048F08B8290EF48F019EC21F08B92BBEC42
:108860001FF08B8290EF48F019EC21F08B9288EC8E
:1088700020F0000EE66E060EE66E00EC5BF0E552B0
:10888000E5528B82FFD790EF48F019EC21F08B92E4
:10889000899C8B8088EC20F032EC62F00201CA6B7C
:1088A000CB6BCC6BCD6BE66A020EE66E000EE66E0D
:1088B000060EE66E78EC5BF0E552E552E552E552C5
:1088C0008B82898C8B9090EF48F019EC21F08B9281
:1088D000020151A103D00101010EB26F0601240E65
:1088E000006F0601670E016F0601650E026F06013B
:1088F000760E036F0601650E046F0601720E056F9A
:1089000006012C0E066FD7C107F6D8C108F606017E
:108910002C0E096FD80EF66EDE0EF76E0800F5CF3E
:108920000AF6D90EF66EDE0EF76E0800F5CF0BF6DE
:1089300006012C0E0C6FDAC10DF6DBC10EF6060136
:108940002C0E0F6F100EE66E060EE66E0101B25190
:10895000E66EE66A12EC57F0E552E552E552E55252
:1089600006012C0E136F06012A0E146F0601156BFB
:108970000401E05108E1000EE66E060EE66E4CECD6
:1089800068F0E552E552CBEC48F08B82C9D319EC84
:1089900021F08B9281EC5CF00101B56F0601240E91
:1089A000006F0601670E016F0601650E026F06017A
:1089B000630E036F06016C0E046F06016F0E056FE8
:1089C00006012C0E066F070EE66E060EE66E01011E
:1089D000B551E66EE66A12EC57F0E552E552E55203
:1089E000E55206012C0E0A6F06010B6B0401E051E3
:1089F00008E1000EE66E060EE66E4CEC68F0E552FD
:108A0000E552C9DB8B828CD319EC21F08B92E3EC1D
:108A10005BF04EC0D2F24FC0D3F250C0D4F251C07E
:108A2000D5F20601240E006F0601670E016F0601E4
:108A3000650E026F06016D0E036F0601650E046F71
:108A400006016D0E056F06012C0E066F070EE66E11
:108A5000060EE66ED2C24EF0D3C24FF0D4C250F032
:108A6000D5C251F0200E4F5E000E505A000E515AE2
:108A7000100E536E270E546E556A566AA2EC73F0B0
:108A80004E50E66EE66A12EC57F0E552E552E552BA
:108A9000E5520601300E0A6F0601300E0B6F06011B
:108AA000300E0C6F0601300E0D6F06012C0E0E6F8E
:108AB00006010F6B0401E05108E1000EE66E060EA0
:108AC000E66E4CEC68F0E552E55265DB8B8228D30C
:108AD00019EC21F08B927FEC5DF00101B56F06017E
:108AE000240E006F0601670E016F0601650E026F0E
:108AF0000601630E036F0601740E046F0601650E16
:108B0000056F06012C0E066F070EE66E060EE66E6A
:108B10000101B551E66EE66A12EC57F0E552E552F6
:108B2000E552E55206012C0E0A6F06010B6B04019B
:108B3000E05108E1000EE66E060EE66E4CEC68F0C1
:108B4000E552E55228DB8B82EBD219EC21F08B92B7
:108B5000DEEC5CF04EC0D2F24FC0D3F250C0D4F283
:108B600051C0D5F20601240E006F0601670E016F99
:108B70000601650E026F06016D0E036F0601650E9C
:108B8000046F0601740E056F06012C0E066F070EAA
:108B9000E66E060EE66ED2C24EF0D3C24FF0D4C2DD
:108BA00050F0D5C251F0F00E4F5E1F0E505A000E1D
:108BB000515A0A0E536E546A556A566AA2EC73F003
:108BC0004E50E66EE66A12EC57F0E552E552E55279
:108BD000E5520601300E0A6F06012C0E0B6F0601DE
:108BE0000C6B0401E05108E1000EE66E060EE66E25
:108BF0004CEC68F0E552E552CEDA8B8291D219EC5A
:108C000021F08B92000EE66E080EE66EB8EC5AF07C
:108C1000E552E552B4EC62F0F00EE66E1EEC74F034
:108C2000E552000EE66E080EE66E00EC5BF0E552D3
:108C3000E552B1EC13F0E3EC5BF04EC0CAF24FC06A
:108C4000CBF250C0CCF251C0CDF20201CA5106E1C4
:108C5000200ECB1903E1CC5101E1CD510BE0040111
:108C6000E05108E1F50EE66EE70EE66E93EC68F073
:108C7000E552E5520401E05103E035EC4BF0FAD740
:108C80000201CA6B200ECB6FCC6BCD6B0401E0519F
:108C900008E1EE0EE66EE70EE66E93EC68F0E55244
:108CA000E55279DA8B823CD219EC21F08B923BECC5
:108CB0005FF048EC63F0F00EE66E1EEC74F0E552E7
:108CC000F00EE66E1EEC74F0E552F00EE66E1EEC51
:108CD00074F0E5520C012D5142E0DEEC5CF04EC028
:108CE000CEF24FC0CFF250C0D0F251C0D1F202014B
:108CF0001F6B02011F51006E016A340E005C000EF2
:108D0000015829E202011F51040DF3CFE9FFF4CF0E
:108D1000EAFFC10EE9260B0EEA22EECF00F0EECFFD
:108D200001F0EECF02F0EFCF03F002011F51040D6E
:108D3000F3CFE9FFF4CFEAFFF50EE9260B0EEA22A6
:108D400000C0EEFF01C0EEFF02C0EEFF03C0EEFF69
:108D500002011F2BCED70A01A6895CEC1CF0B1ECF6
:108D600013F0E3EC5BF04EC0CAF24FC0CBF250C040
:108D7000CCF251C0CDF219EC21F00401E05108E130
:108D8000E70EE66EE70EE66E93EC68F0E552E5520C
:108D900002DA8B82C5D119EC21F08B9248EC63F09A
:108DA000F00EE66E1EEC74F0E552F00EE66E1EEC70
:108DB00074F0E552F00EE66E1EEC74F0E552F00E23
:108DC000E66E1EEC74F0E552F00EE66E1EEC74F0EA
:108DD000E552F00EE66E1EEC74F0E552B1EC13F0C5
:108DE000E3EC5BF04EC0CAF24FC0CBF250C0CCF205
:108DF00051C0CDF219EC21F00401E05108E1E00E80
:108E0000E66EE70EE66E93EC68F0E552E552C3D9E4
:108E10008B8286D119EC21F08B9232EC62F0F00E4D
:108E2000E66E1EEC74F0E552F00EE66E1EEC74F089
:108E3000E552F00EE66E1EEC74F0E552F00EE66EB2
:108E40001EEC74F0E552F00EE66E1EEC74F0E55286
:108E5000F00EE66E1EEC74F0E552E3EC5BF04EC0F3
:108E6000CAF24FC0CBF250C0CCF251C0CDF20201D9
:108E7000CA5106E1200ECB1903E1CC5101E1CD51DD
:108E80000BE00401E05108E1F50EE66EE70EE66E38
:108E900093EC68F0E552E5520401E05102E0E5DBB5
:108EA000FBD70201CA6B200ECB6FCC6BCD6B0401DC
:108EB000E05108E1EE0EE66EE70EE66E93EC68F028
:108EC000E552E55268D98B822BD119EC21F08B92B7
:108ED00048EC20F060D98B8223D119EC21F08B92E1
:108EE00088EC20F0000EE66E060EE66E00EC5BF0FD
:108EF000E552E552B1EC13F019EC21F00401E05118
:108F000002E0B3DBFBD70401E05108E1D90EE66EC5
:108F1000E70EE66E93EC68F0E552E5523CD98B82A1
:108F2000FFD019EC21F08B92C2800A01AA990101AD
:108F3000240E4B6F0101670E4C6F0101650E4D6FE2
:108F40000101610E4E6F0101640E4F6F0101730E3E
:108F5000506F01012C0E516F520EE66E010EE66E3F
:108F60000A01AB51E66EE66A12EC57F0E552E552A3
:108F7000E552E55201012C0E556F560EE66E010EBC
:108F8000E66E0A01AC51E66EE66A12EC57F0E55265
:108F9000E552E552E55201012C0E596F5A0EE66E6C
:108FA000010EE66E0A01AD51E66EE66A12EC57F06C
:108FB000E552E552E552E55201012C0E5D6F5E0E61
:108FC000E66E010EE66E0A01AE51E66EE66A12EC3E
:108FD00057F0E552E552E552E55201012C0E616F62
:108FE000620EE66E010EE66E0A01AF51E66EE66AAB
:108FF00012EC57F0E552E552E552E55201012C0E14
:10900000656F660EE66E010EE66E0A01B051E66E01
:10901000E66A12EC57F0E552E552E552E5520101DD
:109020002C0E696F6A0EE66E010EE66E0A01B151F2
:10903000E66EE66A12EC57F0E552E552E552E5526B
:1090400001012C0E6D6F6E0EE66E010EE66E0A01CA
:10905000B251E66EE66A12EC57F0E552E552E5527F
:10906000E55201012C0E716F0101780E726F010142
:10907000780E736F0101746B0401E05108E14B0E2F
:10908000E66E010EE66E4CEC68F0E552E55283D8D0
:109090008B8246D0010EE66EB4EC1AF0E5528B904E
:1090A0008B82898CFA0EE66E1EEC74F0E552B2ECFF
:1090B00054F0F8EC0AF0F8EC0AF0F8EC0AF0F8ECEE
:1090C0000AF08B80F8EC0AF0F8EC0AF0F8EC0AF001
:1090D000F8EC0AF08B90F8EC0AF0F8EC0AF0F8ECF7
:1090E0000AF0F8EC0AF08B80F8EC0AF0F8EC0AF0E1
:1090F000F8EC0AF0F8EC0AF08B90F8EC0AF0F8ECD7
:109100000AF0F8EC0AF0F8EC0AF019EC21F0F8ECAF
:109110000AF002015191DAEC3DF08B828B9000D085
:1091200037D06CEC39F0030A2AE00F0A14E00D0A7C
:1091300009E0180A04E0190A01E029D028D061ECFE
:109140003DF025D08B80899C8B80010EE66EB4ECBF
:109150001AF0E5521CD0897C0A010A01DE51020195
:109160005195010B01E05185020151938950400B4B
:1091700001E051830DEC5AF02DEC55F008D00BECCA
:109180001BF00201020E586F0A01A38500D000D027
:1091900047EF3FF012000401E05102E066DAFBD72E
:1091A0000401E05108E1D20EE66EE70EE66E93ECA4
:1091B00068F0E552E5520401E05102E056DAFBD7CF
:1091C0001200D9CFE6FFE1CFD9FF020EE126580EFB
:1091D000DE6E020EDD6E9B8CDFCF00F0DF06010E2F
:1091E000DBCF01F001E2DB060050011001E0F4D713
:1091F0000F0EC1120F0148690F014969ADEC4BF028
:10920000020EE15C02E2E16AE552E16EE552E7CF6F
:10921000D9FF1200D9CFE6FFE1CFD9FFD950FD0F1A
:10922000E96EFF0EDA20EA6EEE50ED1006E0FD0E5C
:10923000DB06FE0E01E2DB06F1D7E552E7CFD9FFF0
:109240001200D9CFE6FFE1CFD9FF020EE126010ED1
:10925000DB6A240EE66E3CEC0AF0E5520A0EE66E7E
:10926000E66AD8DFE552E552DF6ADF50E76EFD0EB1
:10927000DBCFF6FFFE0EDBCFF7FFE750F626000E42
:10928000F7220800F5502A082FE0DF50E76EFD0EA8
:10929000DBCFF6FFFE0EDBCFF7FFE750F626000E22
:1092A000F722010EDBCFE7FF0800F550E71A010EA9
:1092B000E7CFDBFFDF50E76EFD0EDBCFF6FFFE0EE4
:1092C000DBCFF7FFE750F626000EF7220800F55037
:1092D000E66E3CEC0AF0E5520A0EE66EE66A9ADFAC
:1092E000E552E552DF2AC1D72A0EE66E3CEC0AF0C1
:1092F000E5520A0EE66EE66A8DDFE552E552010E92
:10930000DB380F0B0F0B090807E2010EDB380F0BE0
:109310000F0B410FF60F05D0010EDB380F0B0F0BB3
:10932000300FE66E3CEC0AF0E5520A0EE66EE66A95
:1093300071DFE552E552010EDB500F0B090806E222
:10934000010EDB500F0B410FF60F04D0010EDB5066
:109350000F0B300FE66E3CEC0AF0E5520A0EE66E9B
:10936000E66A58DFE552E5520D0EE66E3CEC0AF077
:10937000E5520A0EE66EE66A4DDFE552E5520A0E48
:10938000E66E3CEC0AF0E5520A0EE66EE66A42DF53
:10939000E552E552020EE15C02E2E16AE552E16E5D
:1093A000E552E7CFD9FF1200AD94900EAC6E7E6A05
:1093B0007E86370EB06E010E7F6E9E9A0A0EE66EA6
:1093C0001EEC74F0E5521200240EA86EA884900ED4
:1093D0009C6E7C6A330EAB6E7D6A1200AD84900E7B
:1093E000AC6E7E6A330EB06E7F6A9E9A0A0EE66E8F
:1093F0001EEC74F0E5521200D9CFE6FFE1CFD9FFA1
:10940000020EE126DE6ADD6A240EAD6EAD94900E8A
:10941000AC6EAC987E6A7E86370EB06E010E7F6EA3
:109420009D8A9F8A8B900C0160A302D0D7DFB8D0B1
:10943000E7EC23F06E0E0101B25D2AE202015181D8
:1094400002015193F3EC55F0DE6ADD6ADECF00F0E5
:10945000DDCF01F0640E005C000E015817E2C80E6B
:10946000E66E1EEC74F0E552C80EE66E1EEC74F06B
:10947000E55202015171020151730DEC5AF02DECCD
:1094800055F0DF2A010E01E3DB2AE0D761EC3DF065
:109490000A01A99789DFAC88DE6ADD6ADECF00F0B9
:1094A000DDCF01F00A0E005C000E01580CE2E50E63
:1094B000E66EDF0EE66EC5DEE552E552DF2A010EEE
:1094C00001E3DB2AEBD78ADFFA0EE66E1EEC74F0BE
:1094D000E552FA0EE66E1EEC74F0E552FA0EE66EF8
:1094E0001EEC74F0E552FA0EE66E1EEC74F0E552D6
:1094F000FA0EE66E1EEC74F0E552FA0EE66E1EEC05
:1095000074F0E552FA0EE66E1EEC74F0E552FA0EB7
:10951000E66E1EEC74F0E5520A01A9A7BBD7DE6A1D
:10952000DD6ADECF00F0DDCF01F0030E005C000E3F
:1095300001580AE2FA0EE66E1EEC74F0E552DF2ADC
:10954000010E01E3DB2AEDD749DFFA0EE66E1EECD1
:1095500074F0E552FA0EE66E1EEC74F0E552F40E6D
:10956000E66EDF0EE66E6DDEE552E5520A01A9A752
:1095700002D099EC3BF00A01A9A5F1D7230EE66EC3
:10958000E00EE66E5EDEE552E5520A01A9A702D0C2
:1095900099EC3BF00A01A9A3F1D78B800A01A397AC
:1095A000020EE15C02E2E16AE552E16EE552E7CFCC
:1095B000D9FF1200D9CFE6FFE1CFD9FF040EE12693
:1095C000D880000E04015055C20E5155010E52555F
:1095D000000E535501E23FD050C4D8F451C4D9F421
:1095E00052C4DAF453C4DBF4046A1B0E056EB70EE2
:1095F000066E076A04C04EF005C04FF006C050F07A
:1096000007C051F0D8C453F0D9C454F0DAC455F0AF
:10961000DBC456F0A2EC73F04EC000F04FC001F076
:1096200050C002F051C003F00006000E015A000EB7
:10963000025A000E035A00C0DFFF010E01C0DBFF1B
:10964000020E02C0DBFF030E03C0DBFFDF50B06E73
:10965000010EDB507F6E040EE15C02E2E16AE5522E
:10966000E16EE552E7CFD9FF1200200E0E01E76E42
:109670000019E8AE02D0E73402D0E750005D03E302
:109680006550020B01E002D0DAEC68F01200120023
:1096900012001200120031EC67F01200120091EC7F
:1096A00067F0120065840C01080E616F070E626F8F
:1096B0000C016107000E625B0C0161516211F8E15F
:1096C00065941200D9CFE6FFE1CFD9FFFD0EDBCFC5
:1096D00050F0FE0EDBCF51F0720E501801E15150E8
:1096E00033E0E868501802E17F0E51182BE0740E49
:1096F000501801E1515024E0750E501801E151500D
:109700001DE0730E501801E1515016E0030E501881
:1097100001E151500FE0020E501801E1515008E0F4
:10972000010E501801E1515001E010D0B8DF0FD008
:10973000B5DF0DD0B0DF0BD0ACDF09D0A8DF07D08C
:10974000A7DF05D0A7DF03D0000001D000D0010EB5
:0A97500000D0E552E7CFD9FF120068
:06975A00D9CFE6FFE1CFCC
:10976000D9FFE652A098636A626A0F01160E396F3C
:109770000F019F0E376F0F017B0E366F658C0F0147
:10978000386B030EE66EE66AE66A270EE66E0F0E8B
:10979000E66E29EC72F0006E050EE15E0050659CED
:1097A000DF6ADF50006E016A100E005C000E015887
:1097B00010E2DF50040DF3CFE9FFF4CFEAFF000E13
:1097C000E926040EEA22EE6AEE6AEE6AEE6ADF2A03
:1097D000E8D70F01160E266F62A602D06296FCD75C
:1097E0000E011B6B0E01206B0E01216B226B659825
:1097F000DF6A040EDF5C18E2EA6ADF34FE0BEA3649
:10980000E96E0F0EE9260E0EEA22EE6AED6AEA6AAA
:10981000DF34FE0BEA36E96E070EE9260E0EEA2269
:10982000EE6AED6ADF2AE5D70E01080E0F6F040E0F
:10983000106F0E01016B0E01006BE552E552E7CF90
:10984000D9FF1200D9CFE6FFE1CFD9FFE6520E01D2
:1098500000050AE165BA08D0626A0F0136810F017E
:1098600036890E01020E006F6250040B07E00F01F3
:109870000F013651040B02E06294CDD865A202D0EC
:10988000A19895D06250010B1BE00F010F013651DA
:10989000010B16E062DFD08EA288A088F28E0E0146
:1098A000040E006F0401400E026F040E036F0401EA
:1098B000080E016F0401006B8C0E0401001362900E
:1098C0006250100B07E00F010F013651100B02E040
:1098D0008ED862986250400B15E00F010F0136518F
:1098E000400B10E0010EE66EE66A000EE66EE66AD8
:1098F000730EE66EE66A62EC4BF0006E060EE15EF9
:109900000050629C6250200B06E00F010F0136519F
:10991000200B01E051D86250020B15E00F010F013E
:109920003651020B10E0010EE66EE66A000EE66E9E
:10993000E66AE6687F0EE66E62EC4BF0006E060E9D
:10994000E15E0050636A040E0E01E76E0019E8AE96
:1099500002D0E73402D0E750005D02E2A19827D0A0
:109960000F0136A723D0DF6A040EDF5C1FE262A678
:109970001AD064CF28FE6296780E0E01281502E1F7
:1099800061D810D0000EE66EE66A280EE66E0E0E66
:10999000E66E720EE66EE66A62EC4BF0006E060E44
:1099A000E15E005001D002D0DF2ADED7A198E55257
:1099B000E552E7CFD9FF12000F0126A116D003CE42
:1099C000E9FF04CEEAFFEF5080080DE10FCEE9FF7A
:1099D00010CEEAFFEF50840806E103CEE9FF04CE83
:1099E000EAFF8C0EEF6E0F012691629A12000F01B2
:1099F000368562986582000EE66EE66A000EE66EB7
:109A0000E66A750EE66EE66A62EC4BF0006E060ED4
:109A1000E15E00501200000EE66EE66A000EE66E91
:109A2000E66A740EE66EE66A62EC4BF0006E060EB5
:109A3000E15E005065920F01369562A402D06294F7
:109A4000FCD71200D9CFE6FFE1CFD9FFE652FD0ED9
:109A50000E0128155EE17E0E0E012815E8407F0BF1
:109A6000040DF3CF03FEF4CF04FE000E0E01032716
:109A7000040E0E01042303CE05FE04CE06FE0E01E5
:109A8000057503CEE9FF04CEEAFFEF503C0BE84238
:109A9000E8420D083CE103CEE9FF04CEEAFF020EE6
:109AA000E926000EEA22EECF00F0EFCF01F0480EDB
:109AB000001802E1040E011828E103CEE9FF04CEEC
:109AC000EAFF020EE926000EEA22400EEE6E040EB8
:109AD000ED6EDF6ADF50006E016A080E005C000E5A
:109AE000015813E2DF50EA6A480FE96E040EEA22D9
:109AF000EF50E66EDF50EA6A400FE96E040EEA228C
:109B0000E552E750EF6EDF2AE5D70ED801D033D803
:109B100006D0FD0E0E012815040801E153D8E552C8
:109B2000E552E7CFD9FF12000FCEE9FF10CEEAFFD2
:109B3000EF50800B05E00FCEE9FF10CEEAFFEF6A91
:109B40000E01176B0E01186B0E011C6B1D6B0E01C5
:109B50001B6BC0D8000EE66EE66A000EE66EE66A83
:109B6000030EE66EE66A62EC4BF0006E060EE15EF6
:109B7000005083DA1200020E0E01185D02E1EEDBE6
:109B800020D072D80E0129511AE105CEE9FF06CE88
:109B9000EAFFEE52080EEF6E05CEE9FF06CEEAFFB1
:109BA000020EE926000EEA22400EEE6E040EED6E65
:109BB00005CEE9FF06CEEAFF8C0EEF6E02D00E0155
:109BC000296B1200D9CFE6FFE1CFD9FFE6520FCEC5
:109BD000E9FF10CEEAFFEF50400B01E0010EDF6E0F
:109BE0000E010F75080E0E01005D0DE142C438FF35
:109BF0000F013851000804E20E01100E006F03D06F
:109C00000E01040E006F0E01180528E10FCEE9FFCA
:109C100010CEEAFF020EE926000EEA22480EEE6E92
:109C2000040EED6E04DB020E0E01175D07E10FCE90
:109C3000E9FF10CEEAFF840EEF6E0FD0DF5007E190
:109C40000FCEE9FF10CEEAFFC80EEF6E06D00FCEA2
:109C5000E9FF10CEEAFF880EEF6E01D005D8E5527D
:109C6000E552E7CFD9FF1200D9CFE6FFE1CFD9FF08
:109C7000020EE1260E01186B0FCEE9FF10CEEAFFAF
:109C8000EF6A040E0E010F19006E10CE01F000C035
:109C9000DEFF01C0DDFFDECFE9FFDDCFEAFFEF6AC7
:109CA0000E0120AF0DD00E012351241107E005D085
:109CB00024CEFAFF0E012351F96EFADF0E01209F28
:109CC000020EE15C02E2E16AE552E16EE552E7CFA5
:109CD000D9FF120004014051600BE842E842E8421B
:109CE000E842E842000901E064D0040141510C0A55
:109CF0005FE00B0A4DE00C0A3FE0010A2AE00B0A84
:109D000026E0020A24E0030A20E0080A11E0010A22
:109D10000DE00F0A09E0030A01E04AD00E011B8F93
:109D20000E01080E006F45D0D9D843D0BBDB41D01F
:109D30000E01010E196F0E0E1A6F0E011B810E011E
:109D4000010E1C6F0E011B8F34D02ED932D032D8A9
:109D500030D0040144510E01196F1A6B020E0E012E
:109D600019270E0E0E011A230E011B810E01010E82
:109D70001C6F0E011B8F1DD00E011B8F040144515F
:109D8000EA6A020FE96E0E0EEA2242C4EFFF11D01A
:109D9000000EE66EE66A000EE66EE66A020EE66EFB
:109DA000E66A62EC4BF0006E060EE15E005001D0F8
:109DB00000D01200D9CFE6FFE1CFD9FF040EE12693
:109DC0000401420511E1040140511F0B00090CE19F
:109DD0000E011B8F030E0401415D04E10E01010E13
:109DE000276F02D00E01276B040142516DE104017F
:109DF00040511F0B020868E1040144510F0B000998
:109E000063E00E011B8F040144BF11D004014451D3
:109E10000F0BE96EEA6AD890E936EA36070EE926B2
:109E20000E0EEA22EECFDEFFEDCFDDFF10D00401F3
:109E300044510F0BE96EEA6AD890E936EA360F0E04
:109E4000E9260E0EEA22EECFDEFFEDCFDDFF030E98
:109E50000401415D07E1DECFE9FFDDCFEAFF840EBB
:109E6000EF6E32D0040144510F0B016A260F006ED1
:109E70000F0E0122020E00C0DBFF030E01C0DBFF4C
:109E8000020EDBCFE9FF030EDBCFEAFFEF90040108
:109E900044AF0DD0DECFE9FFDDCFEAFFEF6ADF741C
:109EA000DECFE9FFDDCFEAFF400EEF6E0DD0DECF53
:109EB000E9FFDDCFEAFF880EEF6EDF74DECFE9FF4A
:109EC000DDCFEAFFC80EEF6E040EE15C02E2E16A4C
:109ED000E552E16EE552E7CFD9FF1200800E040192
:109EE000405D61E10E01C00E1B6F04014351030A86
:109EF00035E0010A0DE0030A01E052D00E01860EA2
:109F0000196FE40E1A6F120E0E011C6F1D6B4BD0F1
:109F100004014251F66EF76AD890F636F736470ECE
:109F2000F626E50EF7220900F5CF19FE0A00F5CF57
:109F30001AFE020E0E01F76A1925F66E1A51F72263
:109F40000800F5CF1CFE030E0E01F76A1925F66E08
:109F50001A51F7220800F5CF1DFE25D0030E04018B
:109F6000425D1BE204014251F66EF76AD890F63664
:109F7000F736490EF626E50EF7220900F5CF19FE51
:109F80000A00F5CF1AFE19CEF6FF1ACEF7FF080029
:109F9000F5500E011C6F1D6B02D00E011B6B03D020
:109FA0000E011B6B00D01200D9CFE6FFE1CFD9FF25
:109FB000020EE1260401486B0401496B0401405183
:109FC0001F0B020A12E0030A0DE0010A01E03ED075
:109FD0000E011B8F040148810E01270502E10401D7
:109FE000488334D00E011B8F31D00E011B8F04012A
:109FF00044BF11D0040144510F0BE96EEA6AD890B6
:10A00000E936EA36070EE9260E0EEA22EECFDEFF2B
:10A01000EDCFDDFF10D0040144510F0BE96EEA6A69
:10A02000D890E936EA360F0EE9260E0EEA22EECF78
:10A03000DEFFEDCFDDFFDECFE9FFDDCFEAFFEF5042
:10A04000040B03E00401010E486F00D00E011BAFAA
:10A050000AD00E01480E196F040E1A6F0E011B81F3
:10A060000E01020E1C6F020EE15C02E2E16AE55293
:10A07000E16EE552E7CFD9FF120065980E011BBFD4
:10A080004CD00E0120AF29D00E01020E186F0FCE5A
:10A09000E9FF10CEEAFFEE52EF6A0FCEE9FF10CED5
:10A0A000EAFFC80EEF6E05CEE9FF06CEEAFFEE52DC
:10A0B000080EEF6E05CEE9FF06CEEAFF020EE92696
:10A0C000000EEA22480EEE6E040EED6E05CEE9FF9C
:10A0D00006CEEAFFC80EEF6E1FD005CEE9FF06CE12
:10A0E000EAFFEE52080EEF6E05CEE9FF06CEEAFF5C
:10A0F000020EE926000EEA22400EEE6E040EED6E10
:10A1000005CEE9FF06CEEAFF8C0EEF6E0FCEE9FF1B
:10A1100010CEEAFF840EEF6E89D00E0120BF86D0EC
:10A12000040140AF5BD00E011C510401465D0E01DD
:10A130001D510401475904E246C41CFE47C41DFEDC
:10A1400076D80E01010E186F05CEE9FF06CEEAFFA4
:10A15000EE52080EEF6E05CEE9FF06CEEAFF020EC4
:10A16000E926000EEA22400EEE6E040EED6E05CEDC
:10A17000E9FF06CEEAFF800EEF6E0E01296B03CEDB
:10A18000E9FF04CEEAFFEE52080EEF6E03CEE9FFC0
:10A1900004CEEAFF020EE926000EEA22400EEE6E21
:10A1A000040EED6E03CEE9FF04CEEAFF840EEF6EDF
:10A1B0000E01010E296F0FCEE9FF10CEEAFF020E4D
:10A1C000E926000EEA22480EEE6E040EED6E0FCE6A
:10A1D000E9FF10CEEAFFC80EEF6E28D00E01020E86
:10A1E000186F0FCEE9FF10CEEAFFEE52EF6A0FCEE6
:10A1F000E9FF10CEEAFFC80EEF6E05CEE9FF06CEEE
:10A20000EAFFEE52080EEF6E05CEE9FF06CEEAFF3A
:10A21000020EE926000EEA22480EEE6E040EED6EE6
:10A2200005CEE9FF06CEEAFFC80EEF6E1200D9CFC9
:10A23000E6FFE1CFD9FF020EE1260E01080E1C5DFC
:10A24000000E1D5912E21CCEDEFF1DCEDDFF0E01F9
:10A25000175104E10E01010E176F06D00E0117050C
:10A2600003E10E01020E176F03D0080EDE6EDD6AE9
:10A270000FCEE9FF10CEEAFFEF920FCEE9FF10CE2E
:10A28000EAFFEF900FCEE9FF10CEEAFF010EDB50A0
:10A29000EF120FCEE9FF10CEEAFFEE52DFCFEFFF55
:10A2A000000EDB500E011C5F010EDB500E011D5B2A
:10A2B0000E01480E256F040E266F0E011BB123D030
:10A2C000D9CFE9FFDACFEAFFEE50ED101BE00E0127
:10A2D00019CEF6FF1ACEF7FF192B000E1A2308002D
:10A2E000F550E66E0E0125CEE9FF26CEEAFF252BBE
:10A2F000000E2623E552E750EF6EDF06010E01E265
:10A30000DB06DED721D0D9CFE9FFDACFEAFFEE5066
:10A31000ED101AE00E0119CEE9FF1ACEEAFF192B53
:10A32000000E1A23EF50E66E0E0125CEE9FF26CE71
:10A33000EAFF252B000E2623E552E750EF6EDF06DD
:10A34000010E01E2DB06DFD7020EE15C02E2E16A08
:10A35000E552E16EE552E7CFD9FF1200D9CFE6FF13
:10A36000E1CFD9FF020EE12603CEE9FF04CEEAFFDA
:10A37000EE52EFCFDFFFDFCF00F000500E01215D86
:10A38000000E225902E221CEDFFFDF50006E016A8B
:10A3900000500E01215D0E01216F01500E01225966
:10A3A0000E01226F010EDB6ADF50F36E010EDBCF70
:10A3B000F4FFF350F45C17E2010EDB50EA6A480F39
:10A3C000E96E040EEA22EF50E66E0E011ECEE9FFA2
:10A3D0001FCEEAFF1E2B000E1F23E552E750EF6E43
:10A3E000010EDB2AE1D70E01000ED8802155000EA8
:10A3F000225528E205CEE9FF06CEEAFFEE52080E0E
:10A40000EF6E05CEE9FF06CEEAFF020EE926000E4A
:10A41000EA22480EEE6E040EED6E03CEE9FF04CE86
:10A42000EAFFEF50400B07E105CEE9FF06CEEAFF59
:10A43000C80EEF6E06D005CEE9FF06CEEAFF880E05
:10A44000EF6E26D005CEE9FF06CEEAFFEE52080EEB
:10A45000EF6E05CEE9FF06CEEAFF020EE926000EFA
:10A46000EA22400EEE6E040EED6E05CEE9FF06CE3A
:10A47000EAFF840EEF6E0E012351241107E005D090
:10A4800024CEFAFF0E012351F96EFADF0E01209F50
:10A49000020EE15C02E2E16AE552E16EE552E7CFCD
:10A4A000D9FF1200D9CFE6FFE1CFD9FFE6520E0166
:10A4B0001B8F030EE66EE66AE66A270EE66E0F0E47
:10A4C000E66E29EC72F0006E050EE15E0050DF6A68
:10A4D000DF50006E016A100E005C000E015810E2A1
:10A4E000DF50040DF3CFE9FFF4CFEAFF000EE926B9
:10A4F000040EEA22EE6AEE6AEE6AEE6ADF2AE8D716
:10A50000658C010EE66EE66AE66A020EE66E0E0ED7
:10A51000E66E29EC72F0006E050EE15E0050659C5F
:10A520000E01080E0F6F040E106F0E01000E036F68
:10A53000040E046F03CE05FE04CE06FE42C401FEE7
:10A540000E01015104E10E01100E006F13D0010E37
:10A55000E66EE66A010EE66E0E0EE66E010EE66E21
:10A56000E66A62EC4BF0006E060EE15E00500E01F2
:10A57000200E006FE552E552E7CFD9FF1200D9CF88
:10A58000E6FFE1CFD9FF020EE126000EDE6E040EDB
:10A59000DD6EFD0EDB50E824026EFE0EDB50040D76
:10A5A000F3500224040DF350006E016A020E0F0BEB
:10A5B00005E0D89001320032E806FBE1D890003681
:10A5C0000136D89000360136D9CFE9FFDACFEAFF5D
:10A5D0000050EE260150ED22DECFE9FFDDCFEAFF8D
:10A5E000EF9EFD0EDB500FE1FE0EEA6ADB34FE0B40
:10A5F000EA36E96E070EE9260E0EEA22DECFEEFFFE
:10A60000DDCFEDFF0ED0FE0EEA6ADB34FE0BEA363C
:10A61000E96E0F0EE9260E0EEA22DECFEEFFDDCF49
:10A62000EDFFDECFE9FFDDCFEAFFEF9CDECFE9FFF4
:10A63000DDCFEAFF040EE926000EEA22EF8C020EBF
:10A64000E15C02E2E16AE552E16EE552E7CFD9FF53
:10A650001200D9CFE6FFE1CFD9FF020EE126FE0EB0
:10A66000DB50016A260F006E0F0E012200C0DEFFD4
:10A6700001C0DDFFDECFE9FFDDCFEAFFFD0EDBCF5E
:10A68000EFFFFD0EDBA407D0E66AFE0EDBCFE6FF90
:10A6900076DFE552E552FD0EDBA208D0010EE66E34
:10A6A000FE0EDBCFE6FF6BDFE552E552020EE15C0A
:10A6B00002E2E16AE552E16EE552E7CFD9FF12000E
:10A6C000D9CFE6FFE1CFD9FF020EE126FE0EDB5027
:10A6D00020E105CEE9FF06CEEAFFEE52080EEF6E4E
:10A6E00005CEE9FF06CEEAFF020EE926000EEA22B9
:10A6F000400EEE6E040EED6E05CEE9FF06CEEAFFCB
:10A700008C0EEF6E0FCEE9FF10CEEAFF840EEF6ED7
:10A710003DD0FD0EDB50E824026EFE0EDB50040D32
:10A72000F3500224040DF3CF00F0F4CF01F0000E3B
:10A730000026040E012200C0DEFF01C0DDFF840EF2
:10A74000006EDECFE9FFDDCFEAFF0050EF12FD0E15
:10A75000DB50E824026EFE0EDB50040DF3500224A1
:10A76000010F040DF3CF00F0F4CF01F0000E00262E
:10A77000040E012200C0DEFF01C0DDFF840E006E6A
:10A78000DECFE9FFDDCFEAFF0050EF12020EE15C01
:10A7900002E2E16AE552E16EE552E7CFD9FF12002D
:10A7A000D9CFE6FFE1CFD9FF020EE126FD0EDB5047
:10A7B0000FE0FE0EEA6ADB34FE0BEA36E96E0F0E9E
:10A7C000E9260E0EEA22EECFDEFFEDCFDDFF0ED042
:10A7D000FE0EEA6ADB34FE0BEA36E96E070EE92666
:10A7E0000E0EEA22EECFDEFFEDCFDDFFD9CFE9FF7F
:10A7F000DACFEAFFEE50ED1003E1F36AF46A49D0D4
:10A80000DECFE9FFDDCFEAFF020EE926000EEA22E5
:10A81000FB0EDBCFEEFFFC0EDBCFEDFFDECFE9FF63
:10A82000DDCFEAFFEE52FA0EDBCFEFFF400E006EF7
:10A83000DECFE9FFDDCFEAFF0050EF16880E006E95
:10A84000DECFE9FFDDCFEAFF0050EF12FD0EDB5057
:10A850000CE0FE0EEA6ADB34FE0BEA36E96E0F0E00
:10A86000E9260E0EEA22EF740BD0FE0EEA6ADB3404
:10A87000FE0BEA36E96E070EE9260E0EEA22EF74A9
:10A88000DECF00F0DDCF01F000C0F3FF01C0F4FF28
:10A8900000D0020EE15C02E2E16AE552E16EE552AF
:10A8A000E7CFD9FF1200D9CFE6FFE1CFD9FF65A8E6
:10A8B0004ED0FE0EEA6ADB34FE0BEA36E96E0F0E6E
:10A8C000E9260E0EEA22EE50EFCFEAFFE96E400EC7
:10A8D000EE16EE6AEE6AEE6AFE0EEA6ADB34FE0BF4
:10A8E000EA36E96E0F0EE9260E0EEA22EE50EFCFA1
:10A8F000EAFFE96EEE7CFE0EEA6ADB34FE0BEA3616
:10A90000E96E0F0EE9260E0EEA22EF74400E006E7D
:10A91000FE0EEA6ADB34FE0BEA36E96E0F0EE9261C
:10A920000E0EEA22EE50EFCFEAFFE96E0050EF166E
:10A93000FE0EEA6ADB34FE0BEA36E96E0F0EE926FC
:10A940000E0EEA22EE50EFCFEAFFE96EEF7CE55201
:10A95000E7CFD9FF1200656A0F01366B0E01006B5D
:10A9600000D012000E01005117E1656A0F01366B2D
:10A970000F01160E396F0F019F0E376F0F017B0EFF
:10A98000366FD08EA288A088F28E65B602D065861A
:0AA99000FCD70E01010E006F12004B
:06A99A00D9CFE6FFE1CF7A
:10A9A000D9FFC580C5B0FED7700EE66EF7EC72F029
:10A9B000E552040EF36EFE0EDBCFF4FFF350F45CB1
:10A9C00008E2FE0EDB50F409E66EF7EC72F0E55299
:10A9D00004D0E66AF7EC72F0E552C750040B01E0D0
:10A9E000010E006E1F0EC514001001E0F6D7C584DD
:10A9F000C5B4FED7E552E7CFD9FF1200640EE66E6C
:10AA00006FEC74F0E552C750040B01E0010E006ECC
:10AA10001F0EC514001001E0F6D7640EE66E6FEC51
:10AA200074F0E552C580C5B0FED7700EE66EF7EC47
:10AA300072F0E552480EE66EF7EC72F0E552C75040
:10AA4000040B01E0010E006E1F0EC514001001E0A2
:10AA5000F6D7E66AA2DFE5521200D9CFE6FFE1CFD2
:10AA6000D9FF070EE126DF6ADF50006E016A100E83
:10AA7000005C000E015809E2DF50EA6A310FE96E0E
:10AA8000020EEA22EF6ADF2AEFD7050EDB6A0D0E0F
:10AA9000F36E050EDBCFF4FFF350F45C61E2DF6A86
:10AAA000080EDF5C5AE2050EDB50080DF350DF2480
:10AAB000EA6A600FE96E000EEA22EF380F0BE76ECC
:10AAC000030EE7CFDBFF050EDB50080DF350DF244C
:10AAD000EA6A600FE96E000EEA22EF500F0BE76E94
:10AAE000040EE7CFDBFFDF50EA6AC80FE96E000E05
:10AAF000EA22060EEFCFDBFF060EDBCFE6FF050EE8
:10AB0000DB50EA6A410FE96E020EEA22EF50E5528D
:10AB1000E714006E060EDB50005C1DE1040EDB50F6
:10AB2000EA6AC80FE96E000EEA22EFCF00F0030ECA
:10AB3000DB50EA6A310FE96E020EEA22EF50001094
:10AB4000E66E030EDB50EA6A310FE96E020EEA226E
:10AB5000E552E750EF6EDF2AA3D7050EDB2A97D721
:10AB6000C750040B01E0010E006E1F0EC51400104B
:10AB700001E0F6D7C580C5B0FED7700EE66EF7ECE3
:10AB800072F0E552E66AF7EC72F0E552DF6ADF50E8
:10AB9000006E016A100E005C000E01580DE2DF50DD
:10ABA000EA6A310FE96E020EEA22EF50E66EF7EC28
:10ABB00072F0E552DF2AEBD7C750040B01E0010E1B
:10ABC000006E1F0EC514001001E0F6D7C584C5B491
:10ABD000FED7070EE15C02E2E16AE552E16EE55262
:10ABE000E7CFD9FF1200D9CFE6FFE1CFD9FFE65278
:10ABF000DF6ADF50006E016A100E005C000E015823
:10AC000009E2DF50EA6A410FE96E020EEA22EF6ABA
:10AC1000DF2AEFD7E552E552E7CFD9FF1200D9CFAF
:10AC2000E6FFE1CFD9FFFE0EDB50EA6AD00FE96EF6
:10AC3000000EEA22EFCF41F2FE0EDB50EA6AD00F9F
:10AC4000E96E000EEA22EFCF42F2FE0EDB50EA6A16
:10AC5000D00FE96E000EEA22EFCF43F2FE0EDB507A
:10AC6000EA6AD00FE96E000EEA22EFCF44F2FE0E40
:10AC7000DB50EA6AD00FE96E000EEA22EFCF45F210
:10AC8000FE0EDB50EA6AD00FE96E000EEA22EFCF2B
:10AC900046F2FE0EDB50EA6AD00FE96E000EEA22A1
:10ACA000EFCF47F2FE0EDB50EA6AD00FE96E000EDE
:10ACB000EA22EFCF48F2FE0EDB50EA6AD00FE96ECF
:10ACC000000EEA22EFCF49F2FE0EDB50EA6AD00F07
:10ACD000E96E000EEA22EFCF4AF2FE0EDB50EA6A7E
:10ACE000D00FE96E000EEA22EFCF4BF2FE0EDB50E2
:10ACF000EA6AD00FE96E000EEA22EFCF4CF2FE0EA8
:10AD0000DB50EA6AD00FE96E000EEA22EFCF4DF277
:10AD1000FE0EDB50EA6AD00FE96E000EEA22EFCF9A
:10AD20004EF2FE0EDB50EA6AD00FE96E000EEA2208
:10AD3000EFCF4FF2FE0EDB50EA6AD00FE96E000E45
:10AD4000EA22EFCF50F2FE0EDB50EA6AD00FE96E36
:10AD5000000EEA22EFCF51F2E552E7CFD9FF120001
:10AD6000D9CFE6FFE1CFD9FFFE0EDB50EA6AD00F64
:10AD7000E96E000EEA22EFCF41F2FE0EDB50EA6AE6
:10AD8000D00FE96E000EEA22EFCF42F2FE0EDB504A
:10AD9000EA6AD00FE96E000EEA22EFCF43F2FE0E10
:10ADA000DB50EA6AD00FE96E000EEA22EFCF44F2E0
:10ADB000FE0EDB50EA6AD00FE96E000EEA22EFCFFA
:10ADC00045F2FE0EDB50EA6AD00FE96E000EEA2271
:10ADD000EFCF46F2FE0EDB50EA6AD00FE96E000EAE
:10ADE000EA22EFCF47F2FE0EDB50EA6AD00FE96E9F
:10ADF000000EEA22EFCF48F2FE0EDB50EA6AD00FD7
:10AE0000E96E000EEA22EFCF49F2FE0EDB50EA6A4D
:10AE1000D00FE96E000EEA22EFCF4AF2E552E7CFFB
:10AE2000D9FF1200D9CFE6FFE1CFD9FFE652FB0EE2
:10AE3000DBCFE9FFDB2AFC0EDBCFEAFF01E3DB2AF5
:10AE4000300EEF6EFB0EDBCFE9FFDB2AFC0EDBCF13
:10AE5000EAFF01E3DB2A300EEF6EFB0EDBCFE9FFEA
:10AE6000DB2AFC0EDBCFEAFF01E3DB2A300EEF6EBC
:10AE7000FB0EDBCFE9FFFC0EDBCFEAFFEF6AFD0E36
:10AE8000DB50DF6ED950FD0FE96EFF0EDA20EA6E5F
:10AE90000A0E556E566AEECF50F0EDCF51F035ECFC
:10AEA00074F050C0EEFF51C0EDFFFD0EDB500A0DF7
:10AEB000F350DF5E300EDF24E66EFB0EDB06DBCFE9
:10AEC000E9FFFC0E01E2DB06DBCFEAFFE552E750CB
:10AED000EF6ED950FD0FE96EFF0EDA20EA6EEE50EC
:10AEE000ED10CDE1E552E552E7CFD9FF1200D9CF01
:10AEF000E6FFE1CFD9FFE652BDCB4EF0BECB4FF01F
:10AF0000BFCB50F0C0CB51F0EDEC63F04FC004F07C
:10AF100050C005F051C006F052C007F004C0E6FF73
:10AF200005C0E6FF06C0E6FF07C0E6FF6FEC73F062
:10AF3000E552E552E552E5524EC000F04FC001F037
:10AF400050C002F051C003F0546A5F0E556E6A0E95
:10AF5000566E470E576E00C04FF001C050F002C051
:10AF600051F003C052F01EEC66F0010A47E0B8CB86
:10AF7000E9FFB9CBEAFF640E556E566AE9CF50F08F
:10AF8000EACF51F035EC74F050C0E9FF51C0EAFF50
:10AF9000D00EE926000EEA22EF5080090201456F2B
:10AFA0000A0E006E016ABACB50F0BBCB51F000C064
:10AFB00055F001C056F035EC74F05050DF6EDF50A4
:10AFC000EA6AD00FE96E000EEA22EFCF47F20A0ECE
:10AFD000DF02F350026E036A0B010250BA5D006E8D
:10AFE0000350BB59016E0050DF6EDF50EA6AD00F8C
:10AFF000E96E000EEA22EFCF46F21CD0100EDF6E93
:10B00000DF50EA6AD00FE96E000EEA22EF508009A5
:10B010000201456FDF50EA6AD00FE96E000EEA22A6
:10B02000EFCF46F2DF50EA6AD00FE96E000EEA2257
:10B03000EFCF47F2E552E552E7CFD9FF1200D9CF63
:10B04000E6FFE1CFD9FFE652BDCB4EF0BECB4FF0CD
:10B05000BFCB50F0C0CB51F0EDEC63F04FC004F02B
:10B0600050C005F051C006F052C007F004C0E6FF22
:10B0700005C0E6FF06C0E6FF07C0E6FF6FEC73F011
:10B08000E552E552E552E5524EC000F04FC001F0E6
:10B0900050C002F051C003F0F00E546E7B0E556E9E
:10B0A000120E566E490E576E00C04FF001C050F0A0
:10B0B00002C051F003C052F01EEC66F0010A52E0EB
:10B0C000B8CBE9FFB9CBEAFF640E556E566AE9CFFB
:10B0D00050F0EACF51F035EC74F050C0E9FF51C0A8
:10B0E000EAFFD00EE926000EEA22EF5080090201A5
:10B0F000416F0A0E006E016ABACB50F0BBCB51F023
:10B1000000C055F001C056F035EC74F05050DF6EC1
:10B11000DF50EA6AD00FE96E000EEA22EF50800994
:10B120000201436F0A0EDF02F350026E036A0B0145
:10B130000250BA5D006E0350BB59016E0050DF6EC5
:10B14000DF50EA6AD00FE96E000EEA22EFCF42F23A
:10B150000B01BC51EA6AD00FE96E000EEA22EFCF74
:10B1600044F226D0100EDF6EDF50EA6AD00FE96E8F
:10B17000000EEA22EF5080090201416FDF50EA6AB7
:10B18000D00FE96E000EEA22EFCF42F2DF50EA6AFA
:10B19000D00FE96E000EEA22EF5080090201436FE2
:10B1A000DF50EA6AD00FE96E000EEA22EFCF44F2D8
:10B1B000E552E552E7CFD9FF1200D9CFE6FFE1CF44
:10B1C000D9FF200EE66E020EE66EFE0EDBCFE6FF26
:10B1D000E66A28DEE552E552E552E552300E0201FC
:10B1E000205DEA6AD00FE96E000EEA22EFCF4AF244
:10B1F000300E0201215DEA6AD00FE96E000EEA22EC
:10B20000EFCF49F2300E0201225DEA6AD00FE96EFB
:10B21000000EEA22EFCF48F2070E02014C1520097A
:10B2200002014C6FE552E7CFD9FF1200D9CFE6FFFC
:10B23000E1CFD9FF200EE66E020EE66EFE0EDBCFEA
:10B24000E6FFE66AEFDDE552E552E552E552300EE3
:10B250000201205DEA6AD00FE96E000EEA22EFCF0C
:10B260004AF2300E0201215DEA6AD00FE96E000E4B
:10B27000EA22EFCF49F2300E0201225DEA6AD00FD6
:10B28000E96E000EEA22EFCF48F2070E02014C15DC
:10B29000400902014C6FE552E7CFD9FF1200D9CF28
:10B2A000E6FFE1CFD9FF200EE66E020EE66EFD0E40
:10B2B000DBCFE6FFFE0EDBCFE6FFB4DDE552E55265
:10B2C000E552E552300E0201205DEA6AD00FE96EC8
:10B2D000000EEA22EFCF4AF2300E0201215DEA6A47
:10B2E000D00FE96E000EEA22EFCF49F2300E0201D4
:10B2F000225DEA6AD00FE96E000EEA22EFCF48F233
:10B30000070E02014C15100902014C6FE552E7CF00
:10B31000D9FF1200D9CFE6FFE1CFD9FF200EE66EAC
:10B32000020EE66EFD0EDBCFE6FFFE0EDBCFE6FF84
:10B3300079DDE552E552E552E552300E0201205D1D
:10B34000EA6AD00FE96E000EEA22EFCF4AF2300E21
:10B350000201215DEA6AD00FE96E000EEA22EFCF0A
:10B3600049F2300E0201225DEA6AD00FE96E000E4A
:10B37000EA22EFCF48F2070E02014C15080902013C
:10B380004C6FE552E7CFD9FF1200D9CFE6FFE1CFEE
:10B39000D9FFFE0EDB50080805E2080EF36EFE0E24
:10B3A000F3CFDBFFFE0EDB50080A30E00F0A2AE085
:10B3B000010A24E0030A1EE0010A18E0070A12E06D
:10B3C000010A0CE0030A06E0010A01E022D00201B2
:10B3D0004B6B1FD00201010E4B6F1BD00201030EFD
:10B3E0004B6F17D00201070E4B6F13D002010F0EE7
:10B3F0004B6F0FD002011F0E4B6F0BD002013F0E9F
:10B400004B6F07D002017F0E4B6F03D002014B69D7
:10B4100000D0E552E7CFD9FF1200F80E02014C151B
:10B4200002014C6F020151A105D0010E02014C1125
:10B4300002014C6F020151A305D0020E02014C1112
:10B4400002014C6F020151A505D0040E02014C11FE
:10B4500002014C6F1200D9CFE6FFE1CFD9FFF00E09
:10B4600002014D1502014D6FF60EDB0401E07CD0A8
:10B47000FB0EDBCF4FF0FC0EDBCF50F0FD0EDBCF31
:10B4800051F0FE0EDBCF52F05234000E521809E696
:10B49000D880000E4F54000E5054000E5154000E30
:10B4A000525405E2040E02014D1102014D6FFB0ED4
:10B4B000DBCF4FF0FC0EDBCF50F0FD0EDBCF51F0B9
:10B4C000FE0EDBCF52F05234000E521809E6D8803F
:10B4D000000E4F54000E5054000E5154000E5254A2
:10B4E00005E3080E02014D1102014D6FF70EDBCF8F
:10B4F0004FF0F80EDBCF50F0F90EDBCF51F0FA0E23
:10B50000DBCF52F05234000E521809E6D880000EFC
:10B510004F54000E5054000E5154000E525405E288
:10B52000010E02014D1102014D6FF70EDBCF4FF0FE
:10B53000F80EDBCF50F0F90EDBCF51F0FA0EDBCF77
:10B5400052F05234000E521809E6D880000E4F54C3
:10B55000000E5054000E5154000E525405E3020EDA
:10B5600002014D1102014D6FE552E7CFD9FF1200E4
:10B57000D9CFE6FFE1CFD9FFFD0EDBCFE6FFFE0E10
:10B58000DBCFE6FFE66A020EE66EE66A100EE66EB6
:10B59000E66AE66AA2EC61F0006E080EE15E005019
:10B5A000FD0EDBCFE9FFFE0EDBCFEAFFEF502408F4
:10B5B00021E1010EE76EFD0EDBCFE9FFFE0EDBCFD2
:10B5C000EAFFE750E926000EEA22EF50300812E1C8
:10B5D000020EE76EFD0EDBCFE9FFFE0EDBCFEAFFCA
:10B5E000E750E926000EEA22EF502C0803E1010E95
:10B5F00003D002D0000E00D0E552E7CFD9FF1200F1
:10B60000D9CFE6FFE1CFD9FF020EE12642EC62F08E
:10B61000C80EE66E1EEC74F0E552C80EE66E1EEC27
:10B6200074F0E552C80EE66E1EEC74F0E552C80EDA
:10B63000E66E1EEC74F0E552DE6ADD6ADECF00F0E5
:10B64000DDCF01F0000E005C020E015831E251EC3A
:10B6500060F018EC60F0FD0EDBCF00F0FE0EDBCFEB
:10B6600001F0DE500024E96EDD500120EA6EEF505B
:10B67000E66EDECF02F0DDCF03F0000E0226100EE4
:10B680000322046A056A02C0E6FF03C0E6FF04C0A5
:10B69000E6FF05C0E6FF81EC60F0066E050EE15E98
:10B6A000065051EC60F0DF2A010E01E3DB2AC6D719
:10B6B000020EE15C02E2E16AE552E16EE552E7CF9B
:10B6C000D9FF1200000EE66E060EE66EE66A020E66
:10B6D000E66ECAC2E6FFCBC2E6FFCCC2E6FFCDC231
:10B6E000E6FFA2EC61F0006E080EE15E0050120071
:10B6F000D9CFE6FFE1CFD9FF020EE126DE6ADD6A8F
:10B70000DECF00F0DDCF01F0FB0EDBCF02F0FC0E50
:10B71000DBCF03F00250005C0350015839E251ECDA
:10B7200060F018EC60F0FD0EDBCF00F0FE0EDBCF1A
:10B7300001F0DE500024E96EDD500120EA6EEF508A
:10B74000E66EDECF02F0DDCF03F0046A056ACA0EB2
:10B75000E96E020EEA6EEE500226EE500322EE5023
:10B760000422EE50052202C0E6FF03C0E6FF04C03B
:10B77000E6FF05C0E6FF81EC60F0066E050EE15EB7
:10B78000065051EC60F0DF2A010E01E3DB2AB8D746
:10B79000FB0EDBCF00F0FC0EDBCF01F00001005010
:10B7A0000201CA27000101500201CB23000ECC2365
:10B7B000CD23020EE15C02E2E16AE552E16EE55260
:10B7C000E7CFD9FF12000A01816B200E826F836BD5
:10B7D000846B0A018569EF0E866F1F0E876F886B79
:10B7E000E66A020EE66EE66A000EE66E060EE66E8B
:10B7F00029EC72F0006E050EE15E0050810EE96EDC
:10B800000A0EEA6E0A018551EE5C0A018651EE5875
:10B810000A018751EE580A018851EE5868E2000E7D
:10B82000E66E060EE66E100EE66EE66A81CAE6FF6A
:10B8300082CAE6FF83CAE6FF84CAE6FFA2EC61F093
:10B84000006E080EE15E0050FF0E0601005D45E14E
:10B85000FF0E0601015D41E1FF0E0601025D3DE1C3
:10B86000FF0E0601035D39E1FF0E0601045D35E1BF
:10B87000FF0E0601055D31E1FF0E0601065D2DE1BB
:10B88000FF0E0601075D29E1FF0E0601085D25E1B7
:10B89000FF0E0601095D21E1FF0E06010A5D1DE1B3
:10B8A000FF0E06010B5D19E1FF0E06010C5D15E1AF
:10B8B000FF0E06010D5D11E1FF0E06010E5D0DE1AB
:10B8C000FF0E06010F5D09E181CA4EF082CA4FF0FA
:10B8D00083CA50F084CA51F013D0020E0A018227A5
:10B8E000000E0A018323000E0A01842387D781CA30
:10B8F0004EF082CA4FF083CA50F084CA51F000D093
:10B900001200D9CFE6FFE1CFD9FFE652DF6A5BDF55
:10B910004EC085FA4FC086FA50C087FA51C088FAE7
:10B920000A01816B200E826F836B846B810EE96E3E
:10B930000A0EEA6E0A018551EE5C0A018651EE5844
:10B940000A018751EE580A018851EE5830E2000E84
:10B95000E66E060EE66E100EE66EE66A81CAE6FF39
:10B9600082CAE6FF83CAE6FF84CAE6FFA2EC61F062
:10B97000006E080EE15E0050240E0601005D0DE130
:10B98000360E0601015D09E1460E0601025D05E184
:10B990002C0E0601035D01E1DF2A020E0A01822757
:10B9A000000E0A018323000E0A018423BFD7DF5053
:10B9B00000D0E552E552E7CFD9FF12000A01816BB2
:10B9C000F00E826F1F0E836F846B0A018569866992
:10B9D0001F0E876F886B500EE66EE66AE66A4B0EA6
:10B9E000E66E010EE66E29EC72F0006E050EE15E69
:10B9F0000050810EE96E0A0EEA6E0A018551EE5C76
:10BA00000A018651EE580A018751EE580A01885101
:10BA1000EE586BE24B0EE66E010EE66E100EE66E11
:10BA2000E66A81CAE6FF82CAE6FF83CAE6FF84CAE5
:10BA3000E6FFA2EC61F0006E080EE15E0050FF0E22
:10BA400001014B5D45E1FF0E01014C5D41E1FF0E3F
:10BA500001014D5D3DE1FF0E01014E5D39E1FF0E3B
:10BA600001014F5D35E1FF0E0101505D31E1FF0E37
:10BA70000101515D2DE1FF0E0101525D29E1FF0E33
:10BA80000101535D25E1FF0E0101545D21E1FF0E2F
:10BA90000101555D1DE1FF0E0101565D19E1FF0E2B
:10BAA0000101575D15E1FF0E0101585D11E1FF0E27
:10BAB0000101595D0DE1FF0E01015A5D09E181CAE5
:10BAC0004EF082CA4FF083CA50F084CA51F016D0AB
:10BAD000340E0A018127000E0A018223000E0A019A
:10BAE0008323000E0A01842384D781CA4EF082CAC0
:10BAF0004FF083CA50F084CA51F000D01200D9CF61
:10BB0000E6FFE1CFD9FF050EE12658DF4EC0DEFF8C
:10BB10004FC0DEFF50C0DEFF51C0DDFFDD52DD5201
:10BB20000A01816BF00E826F1F0E836F846BD9CF79
:10BB3000E9FFDACFEAFFEE500A0181190CE1EE507D
:10BB40000A01821908E1EE500A01831904E1EE505E
:10BB50000A01841900E102E1000E46D0D9CFE9FFC5
:10BB6000DACFEAFF0A018151EE5E0A018251EE5AF4
:10BB70000A018351EE5A0A018451EE5AD9CFE9FFE6
:10BB8000DACFEAFFEECF04F0EECF05F0EECF06F00D
:10BB9000EFCF07F004C04EF005C04FF006C050F0E4
:10BBA00007C051F0EBEC63F04FC000F050C001F063
:10BBB00051C002F052C003F0546A556A500E566EDE
:10BBC000420E576E00C04FF001C050F002C051F05D
:10BBD00003C052F09DEC64F091EC65F0040E51C08E
:10BBE000DBFF040EDB5000D0006E050EE15C02E2CC
:10BBF000E16AE552E16E0050E552E7CFD9FF12004D
:10BC0000D9CFE6FFE1CFD9FFFE0EDB06006A800E3A
:10BC1000016E0268490E036E086A096A500E0A6EC8
:10BC2000420E0B6EFE0EDBCF10F010C051F0C5ECD3
:10BC300063F04FC00CF050C00DF051C00EF052C078
:10BC40000FF00CC054F00DC055F00EC056F00FC0F0
:10BC500057F008C04FF009C050F00AC051F00BC0B7
:10BC600052F0F0EC64F04FC004F050C005F051C049
:10BC700006F052C007F004C054F005C055F006C0ED
:10BC800056F007C057F000C04FF001C050F002C09E
:10BC900051F003C052F007EC64F0E7EC65F04EC0E1
:10BCA00081FA4FC082FA50C083FA51C084FA4B0E19
:10BCB000E66E010EE66E340EE66EE66A81CAE6FFB7
:10BCC00082CAE6FF83CAE6FF84CAE6FFA2EC61F0FF
:10BCD000006E080EE15E0050340EE66EE66A4B0E12
:10BCE000E66E010EE66EF50EE66E0B0EE66EDBEC12
:10BCF00071F0006E060EE15E0050010E00D0E552BC
:10BD0000E7CFD9FF1200D9CFE6FFE1CFD9FF040E6C
:10BD1000E126DE6ADE6ADE6ADD6ADD52DD52FE0E93
:10BD2000DB06006A800E016E0268490E036E086A27
:10BD3000096A500E0A6E420E0B6EFE0EDBCF10F03B
:10BD400010C051F0C5EC63F04FC00CF050C00DF0C6
:10BD500051C00EF052C00FF00CC054F00DC055F0A1
:10BD60000EC056F00FC057F008C04FF009C050F099
:10BD70000AC051F00BC052F0F0EC64F04FC004F078
:10BD800050C005F051C006F052C007F004C054F096
:10BD900005C055F006C056F007C057F000C04FF080
:10BDA00001C050F002C051F003C052F007EC64F043
:10BDB000E7EC65F04EC081FA4FC082FA50C083FABA
:10BDC00051C084FA4B0EE66E010EE66E040EE66E6E
:10BDD000E66A81CAE6FF82CAE6FF83CAE6FF84CA32
:10BDE000E6FFA2EC61F0006E080EE15E0050040E6A
:10BDF000E66EE66A4B0EE66E010EE66ED9CFE6FF02
:10BE0000DACFE6FFDBEC71F0006E060EE15E00506B
:10BE1000DECF4EF0DECF4FF0DECF50F0DDCF51F071
:10BE2000DD52DD5200D0040EE15C02E2E16AE5522F
:10BE3000E16EE552E7CFD9FF1200D9CFE6FFE1CF9F
:10BE4000D9FFFE0EDBCFE6FFDBDEE552000906E19F
:10BE50004E6A4F6A506A516A0AD009D0F5CB4EF04B
:10BE6000F6CB4FF0F7CB50F0F8CB51F000D0E552C5
:10BE7000E7CFD9FF1200D9CFE6FFE1CFD9FF070EF8
:10BE8000E126010EDF6E3BDEE76E060EE7CFDBFF3D
:10BE90000C012D6B0B01C00EC16F270EC26F090E76
:10BEA000C36FC46B010EDF6E0D0EDF5C12E2DF505C
:10BEB000040DF3CFE9FFF4CFEAFFC10EE9260B0E24
:10BEC000EA22600EEE6EEA0EEE6EEE6AEE6ADF2A8F
:10BED000EBD7060EDB5002E1000E55D0010EDF6EEF
:10BEE000060EDB50D880DF544CE3DFCFE6FF88DE60
:10BEF000E552F50EE96E0B0EEA6E0B01C151EE5CD8
:10BF00000B01C251EE580B01C351EE580B01C45145
:10BF1000EE5835E2010EDB6A0D0EF36E010EDBCF3B
:10BF2000F4FFF350F45C29E2010EDB50040DF3CF73
:10BF3000E9FFF4CFEAFFF50EE9260B0EEA22EECF79
:10BF400000F0EECF01F0EECF02F0EFCF03F0010EE4
:10BF5000DB50040DF3CFE9FFF4CFEAFFC10EE92671
:10BF60000B0EEA2200C0EEFF01C0EEFF02C0EEFFA2
:10BF700003C0EEFF010EDB2ACFD7DFCF2DFCDF2A77
:10BF8000AFD7DF5000D0006E070EE15C02E2E16A3D
:0EBF9000E552E16E0050E552E7CFD9FF1200F6
:02BF9E0073A08E
:10BFA000FED7756A72AE02D073A0FED71200D9CF49
:10BFB000E6FFE1CFD9FFE6528C9E900EE66E4BEC89
:10BFC00074F0E552E66A4BEC74F0E552E66A4BEC2D
:10BFD00074F0E552FE0EDBCFE6FF4BEC74F0E55259
:10BFE0005EEC74F0DF6E8C8EDF5000D0E552E552CF
:10BFF000E7CFD9FF12008C9E500EE66E4BEC74F02A
:10C00000E5528C8E1200D9CFE6FFE1CFD9FF8C9E8E
:10C01000010EE66E4BEC74F0E552FE0EDBCFE6FF50
:10C020004BEC74F0E5528C8EE552E7CFD9FF12004D
:10C030008C9E060EE66E4BEC74F0E5528C8E120070
:10C040008C9E040EE66E4BEC74F0E5528C8E120062
:10C050008C9E800EE66E4BEC74F0E5528C8E1200D6
:10C060008C9E050EE66E4BEC74F0E5525EEC74F0BF
:10C070000401FB6F8C8E0401FB5100D01200D9CF5C
:10C08000E6FFE1CFD9FFE652EBDFDF6E000EDF14F3
:10C0900003E0E6DFDF6EFAD7E552E552E7CFD9FFDE
:10C0A0001200D9CFE6FFE1CFD9FFE652640EDF6E72
:10C0B000D7DF010B010802E1D3DFFAD7E552E552E1
:10C0C000E7CFD9FF1200D9CFE6FFE1CFD9FFE65283
:10C0D000190EDF6EDF5002E0DF06FCD7E552E552B5
:10C0E000E7CFD9FF1200D9CFE6FFE1CFD9FFFE0E8F
:10C0F000DB50756E73A0FED700D0E552E7CFD9FFB5
:10C100001200D9CFE6FFE1CFD9FF8C9E020EE66E7A
:10C11000EADFE552006801680268036AD950FB0F44
:10C12000E96EFF0EDA20EA6EEE500016EE500116B0
:10C13000EE500216EE500316100ED8900332023263
:10C1400001320032E806F9E10050E66ECCDFE5523C
:10C1500000680168026A036AD950FB0FE96EFF0E9E
:10C16000DA20EA6EEE500016EE500116EE5002167E
:10C17000EE500316080ED89003320232013200321C
:10C18000E806F9E10050E66EAEDFE552FB0EDBCFCC
:10C1900000F0FC0EDBCF01F0FD0EDBCF02F0FE0E57
:10C1A000DBCF03F00050E66E9EDFE552FA0EDBCFE8
:10C1B000E6FF99DFE5528C8E86DFE552E7CFD9FFA7
:10C1C0001200D9CFE6FFE1CFD9FF020EE126DE6AE9
:10C1D000DD6ADE6ADD6ADECF00F0DDCF01F0F70E4A
:10C1E000DBCF02F0F80EDBCF03F00250005C03500F
:10C1F000015835E21DDFF90EDBCF00F0FA0EDBCF80
:10C2000001F0DE500024E96EDD500120EA6EEF50AF
:10C21000E66EDECF02F0DDCF03F0046A056AD95086
:10C22000FB0FE96EFF0EDA20EA6EEE500226EE50AA
:10C230000322EE500422EE50052202C0E6FF03C0A6
:10C24000E6FF04C0E6FF05C0E6FF5BDF066E050EF5
:10C25000E15E0650DF2A010E01E3DB2ABCD7F0DEE7
:10C2600020DF020EE15C02E2E16AE552E16EE55296
:10C27000E7CFD9FF1200D9CFE6FFE1CFD9FF040104
:10C28000FB698C9E030EE66E4BEC74F0E552006881
:10C2900001680268036AD950FB0FE96EFF0EDA20CD
:10C2A000EA6EEE500016EE500116EE500216EE50F9
:10C2B0000316100ED8900332023201320032E80623
:10C2C000F9E10050E66E4BEC74F0E552006801684D
:10C2D000026A036AD950FB0FE96EFF0EDA20EA6E9C
:10C2E000EE500016EE500116EE500216EE500316F8
:10C2F000080ED8900332023201320032E806F9E12A
:10C300000050E66E4BEC74F0E552FB0EDBCF00F014
:10C31000FC0EDBCF01F0FD0EDBCF02F0FE0EDBCF1B
:10C3200003F00050E66E4BEC74F0E5525EEC74F0F6
:10C330000401FB6F8C8E0401FB5100D0E552E7CF66
:10C34000D9FF1200D9CFE6FFE1CFD9FF020EE126D7
:10C35000DE6ADD6A8C9E030EE66E4BEC74F0E552ED
:10C36000006801680268036AD950FB0FE96EFF0E8E
:10C37000DA20EA6EEE500016EE500116EE5002166C
:10C38000EE500316100ED890033202320132003202
:10C39000E806F9E10050E66E4BEC74F0E5520068F7
:10C3A0000168026A036AD950FB0FE96EFF0EDA20BA
:10C3B000EA6EEE500016EE500116EE500216EE50E8
:10C3C0000316080ED8900332023201320032E8061A
:10C3D000F9E10050E66E4BEC74F0E552FB0EDBCF5A
:10C3E00000F0FC0EDBCF01F0FD0EDBCF02F0FE0E05
:10C3F000DBCF03F00050E66E4BEC74F0E552DE6AE2
:10C40000DD6ADECF00F0DDCF01F0F90EDBCF02F008
:10C41000FA0EDBCF03F00250005C0350015817E224
:10C420005EEC74F0E66EF70EDBCF00F0F80EDBCFBB
:10C4300001F0DE500024E96EDD500120EA6EE55285
:10C44000E750EF6EDF2A010E01E3DB2ADAD78C8E8C
:10C45000020EE15C02E2E16AE552E16EE552E7CFED
:10C46000D9FF1200E5DD1DDE8C9E600EE66E4BEC02
:10C4700074F0E5528C8EF00EE66E1EEC74F0E55210
:10C4800010DE1200D9CFE6FFE1CFD9FF040EE1267E
:10C49000DE6A100EDE6EDE6ADD6ADD52DD52C8DD58
:10C4A00000DEEDDD8C9E200EE66E4BEC74F0E55266
:10C4B000006801680268036AD9CFE9FFDACFEAFFB2
:10C4C000EE500016EE500116EE500216EE50031616
:10C4D000100ED8900332023201320032E806F9E140
:10C4E0000050E66E4BEC74F0E55200680168026A99
:10C4F000036AD9CFE9FFDACFEAFFEE500016EE501B
:10C500000116EE500216EE500316080ED8900332B4
:10C51000023201320032E806F9E10050E66E4BECDF
:10C5200074F0E552D9CFE9FFDACFEAFFEECF00F0A1
:10C53000EECF01F0EECF02F0EFCF03F00050E66E49
:10C540004BEC74F0E5528C8EACDD780EE66E1EEC92
:10C5500074F0E552040EE15C02E2E16AE552E16E3C
:10C56000E552E7CFD9FF1200D9CFE6FFE1CFD9FFDF
:10C57000040EE126DE6ADE6ADE6ADD6ADD52DD5225
:10C5800057DD8FDD7CDDDE6A200EDE6EDE6ADD6A61
:10C59000DD52DD52D9CFE9FFDACFEAFFFF0EEE5CC4
:10C5A000EF0EEE581F0EEE58000EEE5866E28C9E0F
:10C5B000200EE66E4BEC74F0E552006801680268EC
:10C5C000036AD9CFE9FFDACFEAFFEE500016EE504A
:10C5D0000116EE500216EE500316100ED8900332DC
:10C5E000023201320032E806F9E10050E66E4BEC0F
:10C5F00074F0E55200680168026A036AD9CFE9FF66
:10C60000DACFEAFFEE500016EE500116EE50021699
:10C61000EE500316080ED890033202320132003277
:10C62000E806F9E10050E66E4BEC74F0E552D9CF24
:10C63000E9FFDACFEAFFEECF00F0EECF01F0EECF68
:10C6400002F0EFCF03F00050E66E4BEC74F0E552D1
:10C650008C8E1E0EE66E1EEC74F0E552E9DC21DDD8
:10C660000EDDD9CFE9FFDACFEAFFEE52100EEE264B
:10C67000000EEE22000EEE228DD713DD040EE15CDB
:10C6800002E2E16AE552E16EE552E7CFD9FF12001E
:10C69000D9CFE6FFE1CFD9FF040EE126DE6AF00E26
:10C6A000DE6E1F0EDE6EDD6ADD52DD52C1DCF9DCAE
:10C6B000E6DC8C9E200EE66E4BEC74F0E5520068D2
:10C6C00001680268036AD9CFE9FFDACFEAFFEE50CA
:10C6D0000016EE500116EE500216EE500316100E24
:10C6E000D8900332023201320032E806F9E10050FC
:10C6F000E66E4BEC74F0E55200680168026A036A6A
:10C70000D9CFE9FFDACFEAFFEE500016EE5001165E
:10C71000EE500216EE500316080ED8900332023285
:10C7200001320032E806F9E10050E66E4BEC74F09D
:10C73000E552D9CFE9FFDACFEAFFEECF00F0EECF36
:10C7400001F0EECF02F0EFCF03F00050E66E4BECBD
:10C7500074F0E5528C8EA5DC780EE66E1EEC74F05B
:10C76000E552040EE15C02E2E16AE552E16EE55257
:10C77000E7CFD9FF12003FDCE66A45DCE55258DC22
:0AC7800090DC7DDC8EDC8DDC120005
:06C78A00499E05D0499E06
:10C7900051AE02D0516C498E51C04BF04A6A5B6A6F
:10C7A0005A6A860E4C6E4D6AA1EF66F0499E08D01B
:10C7B000499E51AE05D0506C511EE86A5122498EF7
:10C7C00051C04BF050C04AF05B6A5A6A8E0E4C6EF4
:10C7D0004D6AA1EF66F0499E0CD0499E51AE09D03A
:10C7E0004E6C4F1E501E511EE86A4F22502251229D
:10C7F000498E51C04BF050C04AF04FC05BF04EC064
:10C800005AF09E0E4C6E4D6AA1EF66F0577E496A53
:10C81000DDEC66F0F5EC66F049B685EF66F049A20E
:10C820000AD049AA03D049BE85EF66F049A491EF2A
:10C8300066F08EEF66F049AA05D049AC91EF66F03C
:10C840008EEF66F049A00AD049A808D049BE04D0AE
:10C8500049A402D09AEF66F09EEF66F05A6A4D6ADC
:10C860005750525C596E10E34FC05BF050C04AF015
:10C8700051C04BF052C058F054C04FF055C050F06A
:10C8800056C051F0493A09D054C05BF055C04AF047
:10C8900056C04BF057C058F0596C499E49BC498E60
:10C8A00058C04CF049B0CDEF66F01A0E5960CDEF8C
:10C8B00066F04C6A526A49A408D04F6C501E511E53
:10C8C000521EE86A50225122522249AC08D05B6CB9
:10C8D0004A1E4B1E4C1EE86A4A224B224C224E6ACC
:10C8E000595207E05234513250324F324E32592EA3
:10C8F000F9D74F505B2650504A2251504B2252508C
:10C900004C224EC05AF0499E4CAE0BD05A6C5B1E66
:10C910004A1E4B1E4C1EE86A5B224A224B224C22C6
:10C92000498E4CA006D0D8804B324A325B325A3204
:10C93000582A58C04CF0A1EF66F0496ADDEC66F069
:10C94000F5EC66F049B685EF66F049A205D049BA24
:10C9500085EF66F08CEF66F049BA98EF66F049A073
:10C9600005D049B885EF66F098EF66F049B88CEFCE
:10C9700066F04D6A7F0E52244C6EE86A4D22575085
:10C980004C5EE86A4D5A1A0E586E526A5A6A5B6AD1
:10C990004A6A4B6A54504F5E5550505A5650515A3D
:10C9A000000E525A09E754504F2655505022565007
:10C9B0005122000E522201D05A8AD8904F3650365A
:10C9C00051365236D8905A365B364A364B36582E48
:10C9D000E1D7515050104F10D8A45A8AA1EF66F0F9
:10C9E000496ADDEC66F0F5EC66F049B685EF66F075
:10C9F00049A205D049B885EF66F08CEF66F049AAE8
:10CA000005D049B085EF66F08CEF66F049B002D0F2
:10CA100049A802D098EF66F04D6A575052244C6EE8
:10CA2000E86A4D227E0E4C5EE86A4D5A5A6A5B6A8D
:10CA30004A6A4B6A56505102F4CF4BF0F3CF4AF09A
:10CA400055505102F3505B26F4504A22000E4B22FF
:10CA500056505002F3505B26F4504A22000E4B22EF
:10CA600054505102F3505A26F4505B22000E4A22D1
:10CA70004B2255505002F3505A26F4505B22000EC0
:10CA80004A224B2256504F02F3505A26F4505B2252
:10CA9000000E4A224B2254505002F4505A26000EE7
:10CAA0005B224A224B2255504F02F4505A26000E68
:10CAB0005B224A224B22A1EF66F0486AE86A56AE32
:10CAC0006AEF65F0536C541E551E561E54225522B3
:10CAD0005622481E51AE75EF65F04E6C4F1E501E2B
:10CAE000511E4F2250225122481EA2EC73F051BE1B
:10CAF0008CEF65F048AE000C4E6C4F1E501E511E60
:10CB0000E86A4F22502251224A6C4B1E4C1E4D1E89
:10CB10004B224C224D22000C48BE7CEF65F0498828
:10CB2000FF0C496ADDEC66F049B69BEF65F049A25F
:10CB30000AD049B403D07F0E516E19D0800E516EC9
:10CB400016D0516A14D049B0FCD7870E5260F1D785
:10CB50007E0E5264F6D7860E525C04E0D8905132B5
:10CB6000522AF9D749A403D0516C51AEEAD712002A
:10CB7000496ADDEC66F049B6C2EF65F049A20ED015
:10CB800049B405D07F0E516EFF0E506E1FD0800E3F
:10CB9000516E506A1BD0516A506A18D049B0FBD709
:10CBA0008F0E5260EDD77E0E5264F5D78E0E525C1A
:10CBB00005E0D89051325032522AF8D749A406D015
:10CBC000506C511EE86A512251AEE5D71200496AF5
:10CBD000DDEC66F049B6F1EF65F049A20FD049B43B
:10CBE00007D07F0E516EFF0E506E4F6E4E6E25D0E9
:10CBF000800E516E01D0516A000EF6D749B0FBD7B6
:10CC00004E6A9F0E5260EBD77E0E5264F4D79E0E92
:10CC1000525C07E0D890513250324F324E32522A95
:10CC2000F6D749A40AD04E6C4F1E501E511EE86A1A
:10CC30004F225022512251AEDED7120030EC66F066
:10CC400049B6000C49B0000C49B4000C010C30ECA2
:10CC500066F049B6000C49B0000C49A4000C010C68
:10CC6000496ADDEC66F0F5EC66F049B6120049AEB3
:10CC700008D049A004D049A802D0498012004990A8
:10CC800012005750525C0BE15650515C08E1555070
:10CC9000505C05E154504F5C02E149801200D8A07D
:10CCA00002D0498E10D0525057C052F0576E51509A
:10CCB00056C051F0566E505055C050F0556E4F5002
:10CCC00054C04FF0546E5750525C10E0FF0F09E013
:10CCD000499049B403D049AE4984120049AE499401
:10CCE0001200572AD89056325532543254504F5E63
:10CCF0005550505A5650515A51BEEAD7D8904F36D7
:10CD000050365136522EF8D7C8D77F0E526EFF0ECE
:10CD1000516E506E4F6E12007F0E49BEFF0E526E66
:10CD200002D07F0E526E800E516E506A4F6AF3D75A
:10CD300049AE04D0800E526E516AF7D7526A516ADA
:10CD4000F4D74B504A105B105A10F8E04DBEF0D7A4
:10CD50004BBE0CD04C504D10EBE0D8905A365B36A1
:10CD60004A364B364C06D8A04D06F2D74D50D4E18A
:10CD70004C28D2E05AAE11D07F0E5A1402E15BA0CB
:10CD80000CD05B2AE86A4A224B2207E3D8804B3258
:10CD90004A325B324C2A4C28BFE04C50C9E05BC0A1
:10CDA0004FF04AC050F04B34516E4C30526E5132FD
:10CDB000529E49BE528E8BEF66F05136523602E3D8
:10CDC0004984497E06E14980526A516A506A4F6A35
:10CDD0001200522803E0D88051321200D89051320C
:10CDE00002E149821200498612005636573602E3A4
:10CDF000498C497E06E14988576A566A556A546AE1
:10CE00001200572803E0D88056321200D8905632CC
:10CE1000EAE1498A1200486A56AE14EF67F0556C91
:10CE2000561EE86A5622481E51AE1CEF67F0506C41
:10CE3000511EE86A5122481E35EC74F051BE2CEFA9
:10CE400067F048AE000C506C511EE86A51224C6CE1
:10CE50004D1EE86A4D22000C48BE23EF67F049885A
:02CE6000FF0CC5
:0ECE6200040140511F0B010801E059D00401EA
:10CE70004051600BE842E842E842E842E8420108DB
:10CE800001E04ED00401445104E00401440501E0F6
:10CE900047D004014151220A3DE0030A2EE0010A75
:10CEA0001BE0210A11E0010A01E039D00E01F00E69
:10CEB000196F040E1A6F080E0E011C6F1D6B0E0108
:10CEC0001B810E011B8F2CD00E01F00E196F040E6A
:10CED0001A6F0E011B8F24D046C421FE47C422FEC8
:10CEE0000E01500E1E6F040E1F6F0E01B40E236F45
:10CEF000950E246F0E01208F13D00E01D80E196FDE
:10CF0000040E1A6F070E0E011C6F1D6B0E01C10E71
:10CF10001B6F06D042C4EBF40E011B8F01D000D072
:10CF200012000401D86B4B0ED96FDA6BDB6B040176
:10CF3000DC6B0401DD6B0401080EDE6F0401E06BA5
:10CF40000401DF6B1A0EE66E020EE66E29EC53F05A
:10CF5000E552E5521E0EE66E030EE66E29EC53F026
:10CF6000E552E552400EE66E580EE66E040EE66E91
:10CF7000E66A030EE66ED0EC53F0006E050EE15E3D
:10CF80000050F3CFE7F4F4CFE8F40401E96BEA6B67
:10CF90001200D9CFE6FFE1CFD9FF0401DF6B040116
:10CFA000E751E81102E1000E08D0E7C4E9FFE8C448
:10CFB000EAFFEF50800B01E0010E00094AE1FC0E90
:10CFC000DBCF00F0E7C4E9FFE8C4EAFFEE52EF5020
:10CFD000D880005408E2E7C4E9FFE8C4EAFFEE5253
:10CFE000FC0EEFCFDBFF0401DF6BFC0EDB50040116
:10CFF000DF5D1CE20401DF51EA6A580FE96E040E9E
:10D00000EA22EF50E66E0401DF51E76EFD0EDBCF42
:10D01000E9FFFE0EDBCFEAFFE750E926000EEA2229
:10D02000E552E750EF6E0401DF2BDFD7400EE66ECE
:10D03000580EE66E040EE66EE66A030EE66ED0EC5F
:10D0400053F0006E050EE15E0050F3CFE7F4F4CF2D
:10D05000E8F40401DF5100D0E552E7CFD9FF120018
:10D06000D9CFE6FFE1CFD9FFA0980401E0510FE14D
:10D07000FD0EDBCFE1F4FE0EDBCFE2F4FC0EDBCFE6
:10D08000E5F40401010EE66F0401010EE06FA088D3
:10D09000E552E7CFD9FF1200D9CFE6FFE1CFD9FFA4
:10D0A000030EE126A0980401E05102E0A08831D0EF
:10D0B000DF6AFD0EDBCF50F0FE0EDBCF51F0DE520B
:10D0C00050C0DEFF51C0DDFFDD52DF2ADF50006EB1
:10D0D000016AFF0E001801E1015001E10BD0010EC1
:10D0E000DBCFE9FFDB2A020EDBCFEAFF01E3DB2A1D
:10D0F000EF50EBE1FD0EDBCFE1F4FE0EDBCFE2F40F
:10D10000DFCFE5F40401010EE66F0401010EE06FCC
:10D11000A088030EE15C02E2E16AE552E16EE552AD
:10D12000E7CFD9FF1200D9CFE6FFE1CFD9FF030E39
:10D13000E126A0980401E05102E0A08831D0DF6A26
:10D14000FD0EDBCF50F0FE0EDBCF51F0DE5250C0B3
:10D15000DEFF51C0DDFFDD52DF2ADF50006E016AC5
:10D16000FF0E001801E1015001E10CD0010EDBCFF0
:10D17000F6FFDB2A020EDBCFF7FF01E3DB2A080014
:10D18000F550EAE1FD0EDBCFE1F4FE0EDBCFE2F479
:10D19000DFCFE5F40401E66B0401010EE06FA08827
:10D1A000030EE15C02E2E16AE552E16EE552E7CF8F
:10D1B000D9FF1200D9CFE6FFE1CFD9FF020EE12659
:10D1C000A0980401E951EA1102E1000E08D0E9C477
:10D1D000E9FFEAC4EAFFEF50800B01E0010E00090D
:10D1E00002E0A0889AD0030E0401E05D02E1040190
:10D1F000E06B0401E05102E1A0888FD0020E04012F
:10D20000E05D16E1E66A000EE66EE66A010EE66E85
:10D21000030EE66ED0EC53F0006E050EE15E00509A
:10D22000F3CFE9F4F4CFEAF40401030EE06F74D015
:10D230000401E00571E1400E006E016A0401E55150
:10D24000005C000E015803E2400EDF6E02D0E5C420
:10D25000DFFFDF500401E55D0401E56F0401980E76
:10D26000E36F040EE46F010EDFCFDBFF0401E65134
:10D270001AE1010EDB5016E0E1C4F6FFE2C4F7FF4D
:10D280000800F550E3C4E9FFE4C4EAFFEF6E0401CF
:10D29000E32B000EE4230401E12B000EE223010E38
:10D2A000DB06E7D718D0010EDB5015E0E1C4E9FF3B
:10D2B000E2C4EAFFEF50E3C4E9FFE4C4EAFFEF6E23
:10D2C0000401E32B000EE4230401E12B000EE22312
:10D2D000010EDB06E8D70401E5510AE1400EDF5CF0
:10D2E00004E10401020EE06F03D00401030EE06FBD
:10D2F000DFCFE6FF980EE66E040EE66E010EE66ED8
:10D30000030EE66ED0EC53F0006E050EE15E0050A9
:10D31000F3CFE9F4F4CFEAF4A088020EE15C02E274
:0ED32000E16AE552E16EE552E7CFD9FF120057
:02D32E00FF0EF0
:10D33000E3CFEAFFE552FF0EE3CFE9FFE552E66AED
:10D34000D9CFE6FFDACFE6FFFD0EE124D96EFF0E5E
:10D35000E220DA6EE66AE66A200EEF5C06E0090E6D
:10D36000EF5C03E0EF6603D02CD0EE50F5D72D0E26
:10D37000EF5C03E1FF0EE32A03D02B0EEF5C01E12B
:10D38000EE502F0EEF6416D03A0EEF6013D0D89007
:10D39000FB0EE336FE0EDFCFE3FFD890FB0EE33645
:10D3A000D890FB0EE336FE0EE350DF26300EEE5C27
:10D3B000DF26E7D7FF0EE3CFE8FFE85202E0DF1EEB
:10D3C000DF2AE552E552FF0EE3CFDAFFE552FF0E0A
:10D3D000E3CFD9FFE552FF0EE3CFE8FFE65212009C
:10D3E000FF0EE3CFEAFFE552FF0EE3CFE9FFE55280
:10D3F000E66AE66AD9CFE6FFDACFE6FFFC0EE12463
:10D40000D96EFF0EE220DA6EE66AE66AE66A200E60
:10D41000EF5C06E0090EEF5C03E0EF6603D03FD05F
:10D42000EE50F5D72D0EEF5C03E1FF0EE32A03D09B
:10D430002B0EEF5C01E1EE502F0EEF6424D03A0E7C
:10D44000EF6021D0D890F90EE336FA0EE336FD0EE8
:10D45000DECFE3FFFE0EDDCFE3FFD890F90EE3361B
:10D46000FA0EE336D890F90EE336FA0EE336FD0EE7
:10D47000E350DE26FE0EE350DD22300EEE5CDE26AB
:10D48000000EDD22D9D7FF0EE3CFE8FFE85207E018
:10D49000F90EE31EE32AFA0ED8B4E306E31EE552C2
:10D4A000E552E552FF0EE3CFDAFFE552FF0EE3CF80
:10D4B000D9FFE552E1CFE9FFE2CFEAFFED52ED52AD
:10D4C000EECFF3FFEFCFF4FF1200FF0EE3CFEAFF42
:10D4D000E552FF0EE3CFE9FFE552E66AE66AE66A47
:10D4E000E66AD9CFE6FFDACFE6FFFA0EE124D96E7D
:10D4F000FF0EE220DA6EE66AE66AE66AE66AE66A45
:10D50000200EEF5C06E0090EEF5C03E0EF6603D04F
:10D510006BD0EE50F5D72D0EEF5C03E1FF0EE32A42
:10D5200003D02B0EEF5C01E1EE502F0EEF6444D0E0
:10D530003A0EEF6041D0D890F50EE336F60EE336A2
:10D54000F70EE336F80EE336FB0EDECFE3FFFC0EFC
:10D55000DECFE3FFFD0EDECFE3FFFE0EDDCFE3FF08
:10D56000DD52DD52D890F50EE336F60EE336F70EB7
:10D57000E336F80EE336D890F50EE336F60EE336D2
:10D58000F70EE336F80EE336FB0EE350DE26FC0E14
:10D59000E350DE22FD0EE350DE22FE0EE350DD22DC
:10D5A000DD52DD52300EEE5CDE26000EDE22DE2283
:10D5B000DD22DD52DD52B9D7FF0EE3CFE8FFE8529E
:10D5C00013E0F50EE31EF60EE31EF70EE31EF80E53
:10D5D000E31EF50EE32A08E1F60EE32A05E1F70E55
:10D5E000E32A02E1F80EE32AE552E552E552E5525C
:10D5F000E552D9CFE9FFDACFEAFFEECF4EF0EECF1A
:10D600004FF0EECF50F0EFCF51F0FF0EE3CFDAFF47
:10D61000E552FF0EE3CFD9FFE552E552E552120085
:10D62000D9CFE6FFDACFE6FFE66AE66AE66AE66A9F
:10D63000E66AE66AE66AE66AE66AE66AF20EE3CF58
:10D64000E9FFF30EE3CFEAFF200EEF5C06E0090EE0
:10D65000EF5C03E0EF6603D07BD0EE50F5D72D0EE4
:10D66000EF5C03E1FF0EE38003D02B0EEF5C01E1E2
:10D67000EE50FA0EE124D96EFF0EE220DA6E2E0E85
:10D68000EF5C04E1FF0EE382EE52F9D72F0EEF6458
:10D6900049D03A0EEF6046D0D890FA0EE336FB0E32
:10D6A000E336FC0EE336FD0EE336F60EDECFE3FF87
:10D6B000F70EDECFE3FFF80EDECFE3FFF90EDDCF8E
:10D6C000E3FFDD52DD52D890FA0EE336FB0EE3366F
:10D6D000FC0EE336FD0EE336D890FA0EE336FB0E71
:10D6E000E336FC0EE336FD0EE336F60EE350DE269F
:10D6F000F70EE350DE22F80EE350DE22F90EE3507F
:10D70000DD22DD52DD52300EEE5CDE26000EDE2222
:10D71000DE22DD22DD52DD52FF0EE3A2B0D7FE0E87
:10D72000E306ADD7FF0EE3A013D0FA0EE31EFB0E07
:10D73000E31EFC0EE31EFD0EE31EFA0EE32A08E1D3
:10D74000FB0EE32A05E1FC0EE32A02E1FD0EE32ACB
:10D75000F20EE9CFE3FFF30EEACFE3FFEE0EE3CFE5
:10D76000D9FFEF0EE3CFDAFFFA0EE3CFDEFFFB0EB9
:10D77000E3CFDEFFFC0EE3CFDEFFFD0EE3CFDDFFE8
:10D78000DD52DD52F00EE3CFD9FFF10EE3CFDAFF29
:10D79000FE0EE3CFDFFFF20EE124E96EFF0EE22082
:10D7A000EA6EF60EE126FF0EE222FF0EE3CFDAFF6D
:10D7B000E552FF0EE3CFD9FFE552EECFF3FFEFCFF7
:04D7C000F4FF120060
:0CD7C400D9CFE6FFDACFE6FFE1CFD9FFB6
:10D7D000E2CFDAFF240EE12402E3E168E652E16ED3
:10D7E000D950FA0FE96EFF0EDA20EA6E020EEECF84
:10D7F000DBFF030EEECFDBFF040EEECFDBFF050EEB
:10D80000EECFDBFFE8D9F2D9C0EC70F0006E060E67
:10D81000E15C02E2E16AE552E16E0050E76E0D0E56
:10D82000E7CFDBFFDB50800815E0A0D9546A556ACA
:10D83000566A576A00C04FF001C050F002C051F064
:10D8400003C052F027EC66F0010A10E1210E04013A
:10D85000F86FF96B020EDB68030EDB68040EDB6801
:10D860007F0EF36E050EF3CFDBFF66D10D0EDB509E
:10D87000050B01E061D10A0EDBCF00F00B0EDBCF10
:10D8800001F0830E0026FF0E012200C0DEFF01C062
:10D89000DDFFD950060F65D976D9DF50010B0FE0B7
:10D8A000DF06010E01E2DB06D950180F5AD9D890D5
:10D8B000EF36010EEB36020EEB36030EEB36D9CF08
:10D8C000E9FFDACFEAFF020E556E566AEECF50F04E
:10D8D000EDCF51F00BEC67F050C0EEFF51C0EDFF03
:10D8E000140EDB6A150EDB6A160EDB6A170EDB6A96
:10D8F0001C0EDB6A1D0EDB6A1E0EDB6A010EF36E68
:10D900001F0EF3CFDBFF010EF36E0E0EF3CFDBFF26
:10D910000F0EDB6A0E0EDBCF00F00F0EDBCF01F037
:10D92000D890015004E61A0E005C000E015801E385
:10D9300098D0180EDBCF00F0190EDBCF01F01A0ED5
:10D94000DBCF02F01B0EDBCF03F0010E1F0B07E055
:10D95000D8900036013602360336E806F9E1180E93
:10D9600000C0DBFF190E01C0DBFF1A0E02C0DBFF97
:10D970001B0E03C0DBFF140EDBCF08F0150EDBCF50
:10D9800009F0160EDBCF0AF0170EDBCF0BF0010EFD
:10D990001F0B07E0D890083609360A360B36E80622
:10D9A000F9E1D9501C0FDDD80850EE24046E09505F
:10D9B000EE20056E0A50EE20066E0B50EE20076E2C
:10D9C000D950180FCED80450EE5C006E0550EE58BA
:10D9D000016E0650EE58026E0750EE58036E200E90
:10D9E00000C0DBFF210E01C0DBFF220E02C0DBFF07
:10D9F000230E03C0DBFF200EDBCF4FF0210EDBCF69
:10DA000050F0220EDBCF51F0230EDBCF52F0523418
:10DA1000000E521809E6D880000E4F54000E5054E4
:10DA2000000E5154000E525411E2D950200F99D8D3
:10DA3000AAD8D8D81C0EDB50EE121D0EDB50EE1209
:10DA40001E0EDB50EE121F0EDB50EE12D9501C0FD3
:10DA500088D8AFD80E0EDB2A0F0E01E25BD7DB2A87
:10DA600059D7C9D8100E00C0DBFF110E01C0DBFF73
:10DA7000180EDBCF50F0190EDBCF51F0120E50C054
:10DA8000DBFF130E51C0DBFFADD893D8D950100F78
:10DA900068D8EE50ED1012E0D950120F62D8EE5057
:10DAA000ED1006E1A8D8005001100210031006E0A6
:10DAB00099D8EE2A000EEE22EE22EE220C0EDB6A40
:10DAC00091D8060EEECFDBFF070EEECFDBFF080E80
:10DAD000EECFDBFF090EEECFDBFF7E0EF36E0A0EFC
:10DAE000F3CFDBFF0B0EDB6AD950020FE66E000EA0
:10DAF000DA20E66E70D84EEC71F0E552E552E55250
:10DB0000E552DECFE6FFDDCFE6FF70D824EC70F003
:10DB1000006E060EE15C02E2E16AE552E16E005041
:10DB2000020E4EC0DBFF030E4FC0DBFF040E50C0E1
:10DB3000DBFF050E51C0DBFF19D800C04EF001C05D
:10DB40004FF002C050F003C051F0240EE15C02E23D
:10DB5000E16AE552E16EE552E5CFDAFFE7CFD9FFA2
:10DB60001200E96E000EDA20EA6E1200020EDBCF20
:10DB700000F0030EDBCF01F0040EDBCF02F0050E48
:10DB8000DBCF03F01200180EEECFDBFF190EEECF45
:10DB9000DBFF1A0EEECFDBFF1B0EEECFDBFF12001A
:10DBA000EECFE6FFEECFE6FFEECFE6FFEFCFE6FFEC
:10DBB0001200D890030EEB32020EEB32010EEB3264
:10DBC000EF321200EE500016EE500116EE50021623
:10DBD000EE5003161200D950060FE66E000EDA2042
:10DBE000E66E1200D950140FB1EF6DF0D950020F4C
:10DBF000B8DFD0EF6DF0010E006E016A026A036AB1
:06DC0000F1DFE2EF6DF020
:0ADC0600D9CFE6FFDACFE6FFE1CF49
:10DC1000D9FFE2CFDAFF100EE12402E3E168E65219
:10DC2000E16E0F0EDB6AD950020FE66E000EDA20AD
:10DC3000E66ED950060FE66E000EDA20E66EFC0E98
:10DC4000DBCFE6FFFD0EDBCFE6FF10EC6BF0006EE6
:10DC5000060EE15C02E2E16AE552E16E0050F3CFAC
:10DC6000DEFFF4CFDDFFDECFE9FFDDCFEAFFEF50CF
:10DC7000DF0B450814E1DF2A010E01E3DB2ADECFCA
:10DC8000E6FFDDCFE6FFF0EC69F0E552E552060E67
:10DC9000DBCFE7FFF350E726060EE7CFDBFF020EF0
:10DCA000DBCF00F0030EDBCF01F0040EDBCF02F080
:10DCB000050E03D9EDEC63F0F3D8060EDB5001E15D
:10DCC00090D006D900340BE3010EF36E0F0EF3CFA4
:10DCD000DBFF060EDB50FF0D060EF3CFDBFF0B0E56
:10DCE000DB6A0C0EDB6A800EF36E0D0EF3CFDBFFEA
:10DCF0003F0EF36E0E0EF3CFDBFFEAD8140EE76E85
:10DD00000018E8AE02D0E73402D0E750005C0BE325
:10DD100097D8EC0E546E780E556EAD0E566E600EA2
:10DD200077D8140EB3D8D4D80A0EE76E0018E8AE30
:10DD300002D0E73402D0E750005C0BE381D8F90E43
:10DD4000546E020E556E150E566E500E61D80A0EA8
:10DD50009DD8BED8050EE76E0018E8AE02D0E734B5
:10DD600002D0E750005C0AE36BD8546A500E556E3F
:10DD7000C30E566E470E4CD8050E88D8A9D8020E91
:10DD8000E76E0018E8AE02D0E73402D0E750005C3E
:10DD900009E356D8546A556AC80E566E420E38D8F2
:10DDA000020EEBD795D8010EE76E0018E8AE02D050
:10DDB000E73402D0E750005C09E342D8546A556A60
:10DDC000200E566E410E24D8060EDB060F0EDB50D9
:10DDD00004E043D89DEC64F003D03FD8F0EC64F04D
:10DDE0005FD8070EDBCF00F0080EDBCF01F0090E85
:10DDF000DBCF02F00A0E61D8100EE15C02E2E16AAC
:10DE0000E552E16EE552E5CFDAFFE7CFD9FF120028
:10DE1000576E00C04FF001C050F002C051F003C077
:10DE200052F0F0EC64F00B0E4FC0DBFF0C0E50C054
:10DE3000DBFF0D0E51C0DBFF0E0E52C0DBFF1200E8
:10DE40000B0EDBCF00F00C0EDBCF01F00D0EDBCFA5
:10DE500002F00E0EDBCF03F01200070EDBCF4FF007
:10DE6000080EDBCF50F0090EDBCF51F00A0EDBCFEE
:10DE700052F00B0EDBCF54F00C0EDBCF55F00D0E35
:10DE8000DBCF56F00E0EDBCF57F01200006E060E01
:10DE9000DBCFE7FF0050E75E060EE7CFDBFF1200A7
:10DEA000070E4FC0DBFF080E50C0DBFF090E51C04C
:10DEB000DBFF0A0E52C0DBFF1200DBCF03F000C015
:10DEC0004EF001C04FF002C050F003C051F01200FC
:08DED000060EDBCF00F012008A
:08DED80031340024302C462CEB
:10DEE000313030302C2A0024312C70696C6F746F03
:10DEF0002C70697374612C2A0024322C352C302C40
:10DF0000352C302C352C302C352C302C352C302C1D
:10DF1000352C302C352C302C352C302C2A00243349
:10DF20002C302C2A0024342C312C312C312C2A007A
:10DF300024352C322C322C322C2A0024362C332C33
:10DF4000332C312C2A0024372C332C2A0024382C53
:10DF5000322C2A0024392C35383533323831302CE4
:10DF600033343733353732302C362C313136382C88
:10DF7000313936332C333332302C313237382C337D
:10DF80003138322C313534382C333534372C313963
:10DF900031382C323230302C313435352C31383464
:10DFA000332C313730322C65766974612E70617292
:10DFB0002C302C2A002431302C322C323030302CB2
:10DFC0002A002431312C36302C2A002431322C32D4
:10DFD0002C2A000D0A5B444154415D002447504502
:10DFE0004E440D0A00504D544B3235312C353736E6
:10DFF00030302A00504D544B3331342C302C312CDE
:10E00000302C302C302C302C302C302C302C302C30
:10E01000302C302C302C302C302C302C302C302C20
:10E02000302A00504D544B3232302C3130302A00DF
:10E03000504D544B3136312C302A00313433312C91
:07E0400031383034313600A5
:08E0480096D8E1CFD9FFE2CF29
:10E05000DAFF0C0EE12402E3E168E652E16ED950EA
:10E06000FA0FE96EFF0EDA20EA6E080EEECFDBFF44
:10E07000090EEECFDBFF0A0EEECFDBFF0B0EEECF6D
:10E08000DBFF79D8D950080FE96E000EDA20EA6E6E
:10E09000EECFE6FFEECFE6FFEECFE6FFEFCFE6FFF7
:10E0A000C0EC70F0006E060EE15C02E2E16AE5523F
:10E0B000E16E0050E76E070EE7CFDBFFDB50840B0D
:10E0C0003AE1070EDB041AE1060EDB5006E0006AB7
:10E0D000016A026A800E036E04D0006A016A026A55
:10E0E000036A080E00C0DBFF090E01C0DBFF0A0E49
:10E0F00002C0DBFF0B0E03C0DBFF1DD0F80EDBCF31
:10E1000000F0F90EDBCF01F0D950040FE96E000EDC
:10E11000DA20EA6E0050EE260150ED22D950080FA9
:10E12000E66E000EDA20E66E26D84EEC71F0E5526F
:10E13000E552E552E552080EDBCF00F0090EDBCFC9
:10E1400001F00A0EDBCF02F00B0EDBCF03F000C0B4
:10E150004EF001C04FF002C050F003C051F00C0E61
:10E16000E15C02E2E16AE552E16EE552E5CFDAFFF9
:10E17000E7CFD9FF1200D9CFE6FFDACFE6FF1200D2
:10E18000D9CFE6FFDACFE6FFE1CFD9FFE2CFDAFF62
:10E19000E652006801687F0E026E036AD950FA0FDA
:10E1A000E96EFF0EDA20EA6EEE500016EE50011610
:10E1B000EE500216EE5003166AD800C0EEFF01C002
:10E1C000EEFF02C0EEFF03C0EEFFFD0EDB50800B42
:10E1D00002E0010E01D0000EE66E59D8060EE926C7
:10E1E000000EEA22E552E750EF6EFC0EDBCF00F0A6
:10E1F000FD0EDBCF01F0D89000360136FC0E00C0DA
:10E20000DBFFFD0E01C0DBFFDB50E66E40D8040EE5
:10E21000E926000EEA22E552E750EE6EED6AFD0EA9
:10E22000DB50006E016AFF0E001818E1015016E184
:10E230002ED8EECF00F0EECF01F0EECF02F0EFCF10
:10E2400003F0005001100210031006E0210E04013B
:10E25000F86FF96B800E0BD0040E09D0FD0EDB5069
:10E2600008E115D8EE6AEE6AEE6AEE6A010EDF6E1C
:10E2700006D0020EDF6E0BD8EE52EE52EE8EDF505D
:10E28000E552E552E5CFDAFFE7CFD9FF1200F80EED
:0CE29000DBCFE9FFF90EDBCFEAFF120044
:04E29C00D9CFE6FFF1
:10E2A000DACFE6FFE1CFD9FFE2CFDAFF5BD8013466
:10E2B00011E20050FE08000E01540CE276D805E091
:10E2C0006CD8800EEE6EEE6847D067D8800EEE6E8A
:10E2D0007F0E0ED047D8D890015004E6010E005CA6
:10E2E000000E01580BE261D805E057D8EE6A800EA7
:10E2F000EE6E32D052D8EE6AEE6A2ED047D8EECF0C
:10E3000000F0EECF01F0EECF02F0EFCF03F032D805
:10E3100000C0EEFF01C0EEFF02C0EEFF03C0EEFF43
:10E3200021D80050010B05E025D8020E3AD8EF8E17
:10E3300004D020D8020E35D8EF9E14D8D8900132E0
:10E34000003218D8030E2DD800C0EFFF1AD804E011
:10E3500011D8030E26D8EF8EE552E5CFDAFFE7CFCE
:10E36000D9FF120013D8040E1CD8EECF00F0EFCF67
:10E3700001F01200FA0EDBCFE9FFFB0EDBCFEAFF64
:10E38000120004D8060E0DD8EF501200FC0EDBCFA1
:10E39000E9FFFD0EDBCFEAFF1200ECDFEE6AEE6A6A
:10E3A0001200E926000EEA221200220E0401F86F84
:06E3B000F96BC1EF71F0F2
:0AE3B600D9CFE6FFDACFE6FFFA0E3A
:10E3C000E3CFD9FFFB0EE3CFDAFFFC0EE3CFE9FF8B
:10E3D000FD0EE3CFEAFFE9CFF3FFEACFF4FFF80E3B
:10E3E000E35003E1F90EE35008E0F80EE30602E221
:10E3F000F90EE306DECFEEFFF2D7FF0EE3CFDAFF32
:10E40000E552FF0EE3CFD9FFE5521200FB0EE3CF3A
:10E41000F6FFFC0EE3CFF7FFFD0EE3CFF8FFFE0E95
:10E42000E3CFE9FFFF0EE3CFEAFFE9CFF3FFEACF47
:10E43000F4FFF90EE35003E1FA0EE35009E0F90EA0
:10E44000E30602E2FA0EE3060900F5CFEEFFF1D78C
:10E450001200FE0EE3CFE9FFFF0EE3CFEAFFE9CFA4
:10E46000F3FFEACFF4FFFB0EE35003E1FC0EE350B1
:10E4700009E0FB0EE30602E2FC0EE306FD0EE350AC
:06E48000EE6EF1D7120060
:0AE486001201000202000008FF0F5F
:10E49000FF0F00010102000109024300020100C058
:10E4A00032090400000102020100052400100104E9
:10E4B000240202052406000105240100010705824B
:10E4C0000308000209040100020A00000007050316
:10E4D00002400000070583024000000403090434E1
:10E4E000034D006900630072006F007400650078DE
:10E4F00000200046006900720065004C006F006754
:10E50000000000000000000000000000000000000B
:10E510000000003403430044004300200052005335
:10E52000002D00320033003200200045006D0075E0
:10E53000006C006100740069006F006E00200044F0
:0FE540000065006D006F0098E4DBE4DFE413E595
:10E550001E0EF66E100EF76E000EF86E000109002A
:10E56000F550E66F0900F550E76F03E1E66701D06B
:10E570003DD00900F550E16F0900F550E26F090048
:10E58000F550E36F09000900F550E96E0900F550F8
:10E59000EA6E090009000900F550E46F0900F55022
:10E5A000E56F09000900F6CFE8F0F7CFE9F0F8CF02
:10E5B000EAF0E1C0F6FFE2C0F7FFE3C0F8FF0001B8
:10E5C000E45302E1E55307E00900F550EE6EE4077D
:10E5D000F8E2E507F9D7E8C0F6FFE9C0F7FFEAC0BF
:0EE5E000F8FF0001E607000EE75BBFD7120050
:02E5EE00D9CF83
:10E5F000E6FFDACFE6FFE1CFD9FFE2CFDAFFFD0E8B
:10E60000DB50C96EC6AE02D0FF0E2BD00F0EC61463
:10E6100008080FE00F0EC6140B080BE0C6889EA674
:10E62000FED7C750040B03E1C750010B17E0000EE3
:10E6300018D00F0EC614080804E00F0EC6140B08FD
:10E6400010E1C7B0FED7C750040B01E0010E006E09
:10E650001F0EC5140010F7E1C5AC02D0FE0E01D0AC
:0EE66000000EE552E5CFDAFFE7CFD9FF12003A
:02E66E004E500C
:10E670005302F3CF4AF0F4CF4BF05402F3504B2641
:10E68000000EF4204C6E4E505502F3504C26000EF6
:10E69000F4204D6E4E505602F3504D264F5053020B
:10E6A000F3504B26F4504C22000E4D224F50540292
:10E6B000F3504C26F4504D224F505502F3504D2646
:10E6C00050505302F3504C26F4504D2250505402F7
:0EE6D000F3504D2651505302F3504D261200C8
:02E6DE00D9CF92
:10E6E000E6FFDACFE6FFE1CFD9FFE2CFDAFFE6526D
:10E6F000E652D950FD0F006EFF0EDA2000C0DEFF9B
:10E70000DD6EDECFE9FFDDCFEAFFEF9EFA0EDBCF55
:10E7100000F0FB0EDBCF01F0FC0EDBCF02F0FD0EB4
:10E72000DBCF03F000C04EF001C04FF002C050F04C
:10E7300003C051F0E552E552E552E5CFDAFFE7CFED
:04E74000D9FF1200EB
:0CE744004D6A4C6A4B6A4A6A200EE76E70
:10E75000D8904E364F36503651364A364B364C36B8
:10E760004D3653504A5C54504B5855504C585650A7
:10E770004D5809E353504A5E54504B5A55504C5A29
:0CE7800056504D5A4E2AE72EE4D71200E6
:04E78C00D9CFE6FFFC
:10E79000E1CFD9FF3F0E7316726AFE0EDB50721284
:10E7A000FC0EDB507312FD0EDB50030A0AE0010A77
:10E7B00005E0020A01E007D0738C06D0738C7288E2
:10E7C00003D0728801D000D0728AE552E7CFD9FF1A
:02E7D000120035
:0EE7D200244750454E4400247365636E660074
:10E7E000246770636C7400246770636C6D00246729
:10E7F00070636C7200246770636C724552524F52A2
:09E800002100246770636F6E00B3
:06E80A00D9CFE6FFDACFD2
:10E81000E6FFE1CFD9FFE2CFDAFF3F0EC716C66AA7
:10E82000C56AFD0EDB50C612FC0EDB50C712C68A4D
:0CE83000E552E5CFDAFFE7CFD9FF120078
:04E83C00FF0EE35098
:10E840005F6EEF0E01D0F30EE76EE72E25EF74F04A
:10E850000C0E5E6EE76AE72E2BEF74F05E2E2AEF49
:0AE8600074F05F2E23EF74F0120035
:06E86A004D6A4C6A100E1D
:10E87000E76ED890503651364C364D3655504C5C7C
:10E8800056504D5805E355504C5E56504D5A502A3F
:06E89000E72EF0D7120094
:0AE89600D9CFE6FFE1CFD9FFE6522B
:10E8A0007550DF6EFE0EDB50756E73A0FED7000E46
:0CE8B00000D0E552E552E7CFD9FF12007E
:04E8BC00D9CFE6FFCB
:10E8C000E1CFD9FFE6527550DF6E756A73A0FED7AF
:0EE8D000755000D0E552E552E7CFD9FF120097
:02E8DE00FF0E2B
:10E8E000E3505F6E480E01D04C0EE76EE72EFED768
:0EE8F000E76AE72EFED75F2EF7D70000120072
:02E8FE00C00E4A
:10E90000F36E00EE00F00E0E01D81200EA6002D0A5
:0EE91000EE6AFCD7F350E9601200EE6AFCD705
:02E91E001DEEEC
:10E9200000F02DEE00F0F86A499CA8EC72F003ECC0
:0AE9300008F066EC3EF0FBD7120081
:06E93A00FF0EE350E84E61
:10E940001200000000D000D000D0E82EFAD712004C
:10E9500000000000000000000000000000000000B7
:10E9600000000000000000000000000000000000A7
:10E970000000000000000000000000000000000097
:10E980000000000000000000000000000000000087
:10E990000000000000000000000000000000000077
:10E9A0000000000000000000000000000000000067
:10E9B0000000000000000000000000000000000057
:10E9C0000000000000000000000000000000000047
:10E9D0000000000000000000000000000000000037
:10E9E0000000000000000000000000000000000027
:10E9F0000000000000000000000A0A0A00000000F9
:10EA000000000000000010DE0AFF0A0E0B0C0B00D5
:10EA100000000000000000000000000000000000F6
:0EEA20000000000000000041410048480000D6
:02EA2E0054563C
:10EA3000555743424140444645473332310034360E
:10EA40003537232221202426252713121100535164
:10EA50005250666765646361626076777574B3B1BE
:10EA6000B2B0C6C7C500D7D5D6D4D2D3D100E7E55A
:10EA7000E6E4E2E3E100F7F5F6F4F2F3F100000278
:10EA8000010307050604141615C3C1C2C000101700
:10EA9000E0D00000000001020408102040803F0682
:0FEAA0005B4F666D7D077F6F01020408102040F9
:01FFF800AC5C
:01FFF900F710
:01FFFA001AEC
:01FFFB00FF06
:01FFFC0063A1
:01FFFD00F80B
:01FFFE008181
:01FFFF00F110
:00000001FF
